:020000040800F2
:1000000000000110A5D70308C523030849F800081C
:10001000A9D80308A9D80308A9D80308000000003C
:10002000000000000000000000000000112A03088A
:100030000D2A030800000000092A0308450D0108E5
:10004000A9D80308A9D80308A9D80308A9D8030880
:10005000A9D80308A9D80308E5B5010811B7010814
:10006000D5B6010899B601085DB6010809BD0008BA
:10007000F9BC0008E9BC0008D9BC0008C9BC0008EC
:10008000B5BC0008A1BC0008A9D80308A9D803087A
:10009000A9D80308A9D80308A9D8030821B60108DC
:1000A00099040108A9D80308A9D80308A9D8030806
:1000B000E9040108D9040108A9D80308F1C400081B
:1000C000F9C40008E5C40008EDC40008A9D8030875
:1000D000A9D80308110F0108A9D80308710E010857
:1000E000ABB50108A9D803082D2B03088904010822
:1000F000A9040108A9D80308B90401088DBC0008A7
:10010000A9D80308A9D80308C9040108A9D8030875
:10011000A9D80308A9D80308E5580208C958020855
:1001200079BC000865BC000851BC00083DBC000853
:1001300029BC0008A9D80308A9D80308A9D803082E
:10014000A9D80308A9D80308A9D80308C923030814
:1001500015BC000801BC0008EDBB0008D10D01086A
:10016000D9C40008E1C40008A9D80308A9D8030825
:10017000A9D80308A9D80308A9D80308A9D803084F
:08018000A9D80308A9D803085F
:080188003CD30300010000005C
:1001900002020300AC1E0020A81E00200000000088
:1001A000000000000E020200A41E0020B01E00206D
:1001B000000000001806000816000800D4210020E6
:1001C000EC210020000000001A0600081D000100BC
:1001D000B02300203C24002000000000220600087C
:1001E00027000400D023002040240020000000004D
:1001F000240600082C0010005C2A00204C2A002055
:1002000000000000A9F301082B002400902A002020
:100210006C2A00200000000079F30108290050003A
:1002200080290020B42A0020000000000000000007
:10023000051006003A2C0020842D0020000000004C
:10024000280600080E20EA001A2B00208C2D002022
:10025000000000001D5A020802010300072B0020C5
:10026000782E00200000000021D4020814000200B3
:10027000203100202431002000000000300600085A
:10028000130004001031002028310020000000007D
:1002900034060008100003000C3100202C3100202F
:1002A000000000003806000828001000FC30002084
:1002B0003031002000000000A97502082300100062
:1002C000EC3000204031002000000000C175020821
:1002D00019000500E430002050310020000000002B
:1002E0003C060008F8110100E030002058310020E1
:1002F000000000004206000800010400DC3000207D
:100300005C31002000000000440600082F001100AE
:10031000C8300020603100200000000048060008BE
:100320000A020A0090320020A032002000000000E3
:100330005A06000803000100603400203C39002008
:100340000000000000000000031233007F40002086
:100350004C400020000000006406000825005A0000
:10036000983F0020F23F0020000000000000000045
:10037000F6110C008C3F0020803F002000000000A0
:100380009806000815007000A03E0020103F0020D5
:1003900000000000000000002A006000E03D002096
:1003A000403E002000000000F559020803010A0049
:1003B000504100205C41002000000000A40600081D
:1003C0000120080094420020C042002000000000EC
:1003D000AE0600081A00080078420020C84200203B
:1003E00000000000B60600080101040010430020D0
:1003F0002852002000000000000000000802090050
:10040000505100202C5200200000000029AB0108B0
:1004100006020C00C85100203852002000000000E5
:100420002DAC010807020200FC51002044520020BC
:1004300000000000BE06000802000C00D45100209D
:10044000485200200000000000000000F7010600F4
:10045000445100205452002000000000C006000853
:10046000FA01020054540020805A002000000000CD
:10047000F1F20008FE01090030540020845A0020E7
:1004800000000000DDF20008FB010100F464002020
:10049000B865002000000000D5F20008FC0109004A
:1004A000C0630020BC65002000000000A1F200082D
:1004B0000A101200B85B0020C86500200000000090
:1004C000C606000834001000E45A0020DC65002055
:1004D00000000000AD59020818102C00905A0020AE
:1004E000EC65002000000000B9FB01080D002400AD
:1004F000BC5A00201866002000000000E5B3030885
:1005000004008000487900204C7A002000000000A0
:1005100000000000F9010400647E00201C87002018
:100520000000000011AB0108FD011E00447E002008
:100530002087002000000000A1AA01080600160084
:10054000CC7A0020408700200000000031B502086E
:100550001E00040058870020AC8B00200000000023
:10056000D806000822000C00C88A0020B08B0020AA
:1005700000000000DC06000826000E00CC8B0020E6
:10058000BC8B0020000000001D4203080B2010005F
:10059000308E0020808F002000000000E806000858
:1005A0001F000E00E89000202491002000000000B1
:1005B000F806000805020100D090002034910020C8
:1005C00000000000060700080902010095910020C4
:1005D000AC910020000000000807000812200C0069
:1005E0009C92002030930020000000000A070008C1
:1005F0000C002400A89200203C9300200000000082
:1006000095440208000205007C92002060930020BF
:080610000000000000000000E2
:100618000000C40900001901282800002003000078
:100628002000030100000000030000000800000093
:1006380000010500000028010000020090010000F0
:1006480000000000000000000000000000000000A2
:10065800000000004A01B400D601000000000000BC
:100668000000000000000000000000000000000082
:100678000000000000000000000000000000000072
:100688000000000000000000000000000000010061
:10069800000000000000000000000000040101004C
:1006A8006C1600000000E8036400040A00017E05DF
:1006B800EA05B4053200013C3901000000000030B1
:1006C8000400005A0000000090012C01C8006400DA
:1006D80000000100C800141E010064002C0128005D
:1006E8002B21231E64000200000001000A012900DA
:1006F80000000000000001000000000500000000EC
:0E070800370000000001000553504B32000086
:100716005001000007000000020000000000000079
:100726000000000001020304060708090101000099
:10073600EC210408BC56040800000000000000007C
:10074600FC21040804220408000000000120000027
:1007560008220408102204080000000001400000DE
:1007660014220408003004080000000001200000E4
:10077600202204082C2204080000000004000000C7
:10078600302204083C220408000000000400000097
:100796004022040830550408000000000100000053
:1007A600020100000000803F0000803F00000000C2
:1007B60000000000000000000000803FFF00000075
:1007C6000101D60161ED01080000000000000000F3
:1007D60020700020702D7200000000000000000054
:1007E600F80D0020FFFFFFFFFA00000001000000E7
:1007F60001000000FC2804080000000000000000C2
:100806000000000000000000E828040804000000C2
:10081600C786030800000000000000000429040841
:1008260001000000000000000000000000000000C1
:10083600000000000D0000000000000000000000A5
:1008460000000000FA7900200100C4090000000041
:10085600F87900200100C40900000000F6790020A4
:100866000100C40900000000F47900200100C40959
:1008760000000000F07900200100C409000000001B
:10088600F27900200100C40900000000EE79002082
:100896000100C40900000000EC7900200100C40931
:1008A600000000000000000000000000E40000203E
:1008B6008C9000209CFF2C0100000000DC1600201C
:1008C6000A000000F4F4030838910020E0150C1724
:1008D60000000000DE160020080000001C1B0408B3
:1008E600DD16002005000000701E04083A91002065
:1008F600020000000CF50308402C00200100FF7FD9
:1009060001000000392C00200200000018F5030841
:100916000E2B00200300000028F503080D2B0020F5
:100926000300000028F503080C2C00200000F40149
:10093600010000000A2C00200000F4010100000064
:10094600082C00200000F40101000000062C002005
:100956000000F40101000000042C002000FF01004B
:10096600242C0020E803D0070A000000222C0020D7
:10097600006401000A0000001E2C00200064010033
:100986001D2C002000640100232C002000640100BF
:100996000A0000001C2C0020006401000A00000070
:1009A600212C0020006401000A000000202C0020F9
:1009B600006401000A0000001F2C002000640100F2
:1009C6000A0000001B2C002000FF01000A000000A6
:1009D6001A2C002000FF01000A000000162B002040
:1009E6000000F40101000000142B00200000F401B7
:1009F60001000000122B00200000F401010000009D
:100A0600102B00200000F40101000000162C00202D
:100A16001400E80301000000142C0020E8033075E0
:100A260001000000132C002000C80100122C002039
:100A360000C80100112C002000C80100102C002065
:100A4600006401000A0000000F2C002000FF0100D6
:100A56000A0000002F2C002000C801002E2C0020C8
:100A660000C801002D2C002000C801002C2C0020FD
:100A760000C801002B2C002000C801002A2C0020F1
:100A860000C80100292C002000C80100282C0020E5
:100A960000C80100272C002000C8010044290408D2
:100AA6000000000000000000000000000000000040
:100AB60054290408090000000000000088010020F5
:100AC600040000005C290408090000000000000082
:100AD6007C01002004000000582D040809000000D5
:100AE60000000000700100200400000064290408D2
:100AF600090000000000000064010020040000005E
:100B060068290408090000000000000058010020C0
:100B1600040000007029040809000000000000001D
:100B26004C01002004000000782904080900000098
:100B36000000000040010020040000008029040895
:100B4600090000000000000034010020040000003D
:100B56000429040801000000000000000000000055
:100B660000000000000000000D0000000000000072
:100B76000000000000000000C02A04080000000079
:100B8600000000000000000000000000BC56040841
:100B960000000000000000009B160020040000007A
:100BA600CC2A04080C00000029870308DC01002079
:100BB600000000005C5804080C00000031810308A6
:100BC600D001002000000000D02A04080C0000001C
:100BD60015810308C401002000000000D82A04087B
:100BE6000800000000000000B8010020040000001A
:100BF600E02A04080C00000061800308AC01002014
:100C060000000000E82A04080900000000000000B7
:100C1600A001002004000000F02A040803000000E0
:100C26008D12020894010020000000000429040827
:100C360001000000000000000000000000000000AD
:100C4600000000000D000000000000000000000091
:100C560000000000F42A0408000000000000000064
:100C66000000000000000000042B04080C00000037
:100C760000000000F4010020000000000C2B040816
:100C86000A00000000000000A82C00200000000060
:100C9600182B04080A00000000000000B02C0020F9
:100CA60000000000202B04080A00000000000000DD
:100CB600B82C002000000000282B040808000000C3
:100CC60000000000E801002000000000302B0408AE
:100CD60004000000C113020800000000000000002C
:100CE60004290408010000000000000000000000C4
:100CF60000000000000000000D00000000000000E1
:100D060000000000000000003C2B0408000000006A
:100D1600000000000000000000000000502B040846
:100D26000C000000000000000C0200200000000083
:100D3600602B040804000000D51002080000000023
:100D460000000000682B04080C00000000000000F2
:100D560000020020000000007C2B040804000000B4
:100D6600B510020800000000000000000429040875
:100D7600010000000000000000000000000000006C
:100D8600000000000D000000000000000000000050
:100D960000000000842B0408000000000000000092
:100DA6000000000000000000982B04080700000067
:100DB600000000004802002000000000A42B0408E8
:100DC60008000000000000003C02002000000000B7
:100DD600B02B0408080000000000000030020020CC
:100DE60000000000BC2B0408080000000000000002
:100DF6002402002000000000C82B040808000000A0
:100E06000000000018020020000000000429040869
:100E160001000000000000000000000000000000CB
:100E2600000000000D0000000000000000000000AF
:100E360000000000D42B04080000000000000000A1
:100E4600C300002000000000E02B04080B00000097
:100E560000000000C002002000000000E82B04088B
:100E66000B00000000000000B4020020000000009B
:100E7600F42B04080B00000000000000A80200206C
:100E860000000000002C04080B0000000000000019
:100E96009C020020000000000C2C04080B0000003F
:100EA600000000009002002000000000182C04083A
:100EB6000B0000000000000084020020000000007B
:100EC600202C04080B00000000000000780200201F
:100ED600000000002C2C04080700000000000000A1
:100EE6007002002000000000342C040807000000F7
:100EF600000000006802002000000000402C0408EA
:100F06000B000000000000005C0200200000000052
:100F16004C2C0408080000000000000050020020CD
:100F26000000000004290408010000000000000081
:100F36000000000000000000000000000D0000009E
:100F4600000000000000000000000000582C04080B
:100F5600000000000000000000000000000000008B
:100F66006C2C04080800000000000000F0020020BD
:100F760000000000782C04080800000000000000B3
:100F8600E402002000000000842C04080800000091
:100F960000000000D802002000000000902C040889
:100FA6000800000000000000CC0200200000000045
:100FB60004290408010000000000000000000000F1
:100FC60000000000000000000D000000000000000E
:100FD6000000000000000000982C0408000000003B
:100FE60000000000C000002000000000A82C04083B
:100FF6000B00000000000000380300200000000085
:10100600B42C04080B000000000000002C03002094
:1010160000000000C02C04080700000000000000CB
:101026002403002000000000CC2C04080700000068
:10103600000000001C03002000000000D82C04085B
:10104600070000000000000014030020000000005C
:10105600E42C04080800000000000000080300203B
:1010660000000000EC2C040808000000000000004E
:10107600FC02002000000000042904080100000012
:10108600000000000000000000000000000000005A
:101096000D0000000000000000000000000000003D
:1010A600F42C04080000000000000000C00000202E
:1010B60000000000002D04080700000000000000EA
:1010C6008403002000000000082D0408070000002B
:1010D600000000007C03002000000000102D040822
:1010E600070000000000000074030020000000005C
:1010F600182D040807000000000000006C03002003
:1011060000000000202D0408070000000000000079
:101116006403002000000000282D040807000000DA
:10112600000000005C03002000000000302D0408D1
:10113600070000000000000054030020000000002B
:10114600382D040807000000000000004C030020B2
:1011560000000000402D0408070000000000000009
:1011660044030020000000000429040801000000D8
:101176000000000000000000000000000000000069
:101186000D0000000000000000000000000000004C
:1011960000000000FD0C02088C0300200C2B002030
:1011A6001B00000038F503080B2B00200A32010053
:1011B6000A2B002001FA0100062B002000C80100BE
:1011C600042B0020E803D0070100000053504152D1
:1011D6004B5932009D80030800000000680400207F
:1011E600A1130208350F020844050020130D02085A
:1011F60000000000F8050020990D0208690D02089C
:1012060084060020210E0208650E0208240700202D
:10121600182C002001030100450D0208210D0208CB
:101226003C080020C90D0208F5100208C808002075
:10123600950E02084D110208900900200E2C002080
:1012460001030100482D0408000000000000000012
:101256000000000000000000542D040808000000F3
:1012660000000000B00A0020000000005C2D040809
:101276000700000000000000A80A0020000000008F
:101286006C2D04080700000000000000A00A0020E2
:1012960000000000782D0408070000000000000090
:1012A600980A002000000000842D04080C000000AD
:1012B600000000008C0A002000000000902D0408A9
:1012C600030000008D120208800A002000000000C2
:1012D60004290408010000000000000000000000CE
:1012E60000000000000000000D00000000000000EB
:1012F6000000000000000000982D04080000000017
:10130600000000000000000000000000A82D0408F6
:101316000A00000000000000C022040800000000CF
:10132600B02D04080A00000000000000CC210408CB
:1013360000000000B82D04080A00000000000000AC
:10134600302C002000000000C02D04080A00000018
:1013560000000000BC0A0020000000000429040868
:101366000100000000000000000000000000000076
:10137600000000000D00000000000000000000005A
:1013860000000000C82D0408000000000000000056
:101396000000000000000000DC2D0408030000002F
:1013A6008D120208D00A002000000000E82D040873
:1013B600030000008D120208E01600200000000065
:1013C600F02D0408030000008D120208C40A002054
:1013D60000000000042904080100000000000000CD
:1013E6000000000000000000000000000D000000EA
:1013F600000000000000000000000000F82D0408B6
:1014060000000000000000000000000000000000D6
:10141600042E040807000000991102082C0B002076
:101426000000000074300408030000008D1202085A
:10143600200B002000000000102E0408030000000E
:101446008D120208140B002000000000182E04085C
:10145600030000008D120208080B002000000000A7
:10146600202E0408070000007D110208000B002052
:101476000000000078580408030000008D120208DE
:10148600F40A0020000000002C2E040803000000CF
:101496008D120208E80A002000000000382E040819
:1014A600030000008D120208DC0A00200000000084
:1014B60004290408010000000000000000000000EC
:1014C60000000000000000000D0000000000000009
:1014D6000000000000000000C50C02088D0C020888
:1014E600340B0020010F020800000000E80B00206A
:1014F6000000000000000000740C0020D90E020855
:10150600B5110208EC0C0020442E0408000000006F
:10151600000000000000000000000000502E04083B
:10152600030000008D120208EC0D002000000000F0
:10153600582E0408030000008D120208E00D00205A
:1015460000000000642E0408030000008D1202084B
:10155600D40D002000000000702E040803000000D7
:101566008D120208C80D002000000000782E040825
:1015760002000000711402080000000000000000D4
:10158600802E040802000000711402080100000009
:10159600000000008C2E04080200000071140208EE
:1015A6000200000000000000000000000D00000026
:1015B6000000000000000000000000000001010122
:1015C60001000000FFFFFFFF00000000010203040E
:1015D60001020304060708090000803F000000001E
:1015E60000000000000000000000803F0000000036
:1015F60000000000000000000000000000000000E5
:1016060000000000000000000000000000000000D4
:101616000000803F00000000000000000000000005
:1016260001000000D01004080508040000000000B6
:10163600701E04081C1B04085C1E04080000000041
:10164600FC10040805080A0000000000701E0408CB
:101656001C1B0408F4F403080000000000600240AC
:101666001060024000000000000B00000000200097
:1016760000000000000000000060024028600240F8
:1016860000000000060C0000000020000000000022
:1016960000000000006002404060024000000000C0
:1016A600100D0000000020000000000000000000F7
:1016B600006002405860024000000000160E000064
:1016C6000000200000000000000000000060024052
:1016D6007060024000000000200F000000002000A3
:1016E6000000000000000000006002408860024028
:1016F600000000002610000000002000000000008E
:101706000000000000600240A060024000000000EF
:101716003011000000002000000000000000000062
:1017260000600240B860024000000000362F000052
:1017360000002000000000000000000000640240DD
:101746001064024000000000003800000000400065
:10175600000000000000000000640240286402400F
:1017660000000000063900000000400000000000F4
:1017760000000000006402404064024000000000D7
:10178600103A0000000040000000000000000000C9
:10179600006402405864024000000000163B00004E
:1017A600000040000000000000000000006402404D
:1017B6007064024000000000203C00000000400071
:1017C600000000000000000000640240886402403F
:1017D6000000000026440000000040000000000059
:1017E6000000000000640240A06402400000000007
:1017F600304500000000400000000000000000002E
:1018060000640240B8640240000000003646000052
:101816000000400000000000000000000000000181
:10182600000000000000000000000000F91E030890
:10183600B11E0308552A030800000000FD1B03081B
:10184600FD1D0308851E03085D1D0308000000003A
:1018560000000000F11B0308711B03086D1B030841
:10186600691B03085D1B0308591B0308651B030856
:10187600611B0308E51B0308D91B0308B11B0308FA
:10188600C51B03089D1B0308891B0308751B03085A
:1018960001000000040309041201000202020040D4
:1018A60083044057000201020301000009024300BD
:1018B600020100C0320904000001020201000524F1
:1018C600001001052401000104240202052406007B
:1018D60001070582030800FF09040100020A00004F
:1018E60000070501024000000705810240000000D4
:1018F600FF000000B5AC0208A1AD020871A70208FE
:10190600D5A3020821AF0208E5A3020801A4020834
:10191600351C0308251C0308000000000000000019
:101926000000803F044C0408000000000000000096
:1019360031D40208A0860100040000000000000067
:101946000000000000000000000000000000000091
:101956000000000000000000743004089C29040800
:1019660000000000D93101087D00000006000000DB
:101976000000000000000000000000000000000061
:10198600000000000000000000000000C05604082F
:10199600000000000000000035A60108E803000072
:1019A600030000000000000000000000000000002E
:1019B6000000000000000000000000000000000021
:1019C600C856040800000000000000006DB60208BA
:1019D60010270000030000000000000000000000C7
:1019E60000000000000000000000000000000000F1
:1019F60000000000D45604080000000011F201089F
:101A060039820108204E0000050000000000000099
:101A160000000000000000000000000000000000C0
:101A26000000000000000000904D040800000000C7
:101A3600000000001110010810270000010000003E
:101A46000000000000000000000000000000000090
:101A5600000000000000000000000000D856040846
:101A660000000000000000006DF20008E80300001E
:101A7600050000000000000000000000000000005B
:101A86000000000000000000000000000000000050
:101A9600E4560408000000000000000055D60208C5
:101AA600204E0000030000000000000000000000BF
:101AB6000000000000000000000000000000000020
:101AC60000000000F45604080000000000000000BA
:101AD6005FD40208204E0000030000000000000052
:101AE60000000000000000000000000000000000F0
:101AF6000000000000000000045704080000000079
:101B0600000000003DF40008400D03000300000043
:101B160000000000000000000000000000000000BF
:101B2600000000000000000000000000C84C04088F
:101B3600000000000000000019BA0308102700008A
:101B4600010000000000000000000000000000008E
:101B5600000000000000000000000000000000007F
:101B6600704B040800000000000000000555030843
:101B76001027000003000000000000000000000025
:101B8600000000000000000000000000000000004F
:101B960000000000145704080000000000000000C8
:101BA60075C80308A08601000100000000000000BF
:101BB600000000000000000000000000000000001F
:101BC6000000000000000000604B04080000000058
:101BD6000000000095C7030850C300000100000084
:101BE60000000000000000000000000000000000EF
:101BF600000000000000000000000000482A040861
:101C06000000000000000000FDC20308A8610000FB
:101C160001000000000000000000000000000000BD
:101C260000000000000000000000000000000000AE
:101C36001C570408000000000000000031B1030832
:101C4600A086010001000000000000000000000066
:101C5600000000000000000000000000000000007E
:101C660000000000984D040800000000000000007D
:101C760085C50008A00F000001000000000000005C
:101C8600000000000000000000000000000000004E
:101C96000000000000000000082A04080000000000
:101CA60000000000496F0308102700000100000033
:101CB600000000000000000000000000000000001E
:101CC600000000000000000000000000444B040873
:101CD6000000000000000000051602081A4100007E
:101CE60001000000000000000000000000000000ED
:101CF60000000000000000000000000000000000DE
:101D060028570408000000000000000079BE030800
:101D1600400D03000000000000000000000000006D
:101D260000000000000000000000000000000000AD
:101D3600000000003057040800000000000000000A
:101D460035BE0308400D030000000000000000003F
:101D5600000000000000000000000000000000007D
:101D660000000000000000003857040800000000D2
:101D7600000000005DAE0308A0860100030000001D
:101D8600000000000000000000000000000000004D
:101D960000000000000000000000000000FFFF003F
:101DA60000000000AA5505010000012D202D2D2060
:101DB6002D2D2D2D202D2D2D2D0000000000000095
:101DC60000000000000000000000AA550B01000002
:101DD600AA5507010000AA550902000000000000EC
:101DE60001000000C012AA5503009F000101010076
:101DF6004D8103080000000054180020B058040864
:101E060000000000000000000000000000000000CC
:101E1600BC5604080000000000000000941C0020CE
:101E2600040000005C5804080C0000008D10020835
:101E36007C1C002000000000D02A04080C000000D2
:101E460065100208701C002000000000D82A040853
:101E56000800000000000000641C002004000000D0
:101E6600E02A04080C000000690C0208581C002037
:101E760000000000F02A0408030000008D1202088A
:101E86004C1C002000000000C0580408030000009D
:101E96008D120208401C00200000000004290408DE
:101EA600010000000000000000000000000000002B
:101EB600000000000D00000000000000000000000F
:101EC60000000000B05804080000000000000000F8
:101ED6000000000000000000BC56040800000000DE
:101EE60000000000941C00200400000004580408B0
:101EF600030000004D870308341C00200800000082
:101F0600E02A04080C000000690C0208581C002096
:101F160000000000F02A0408030000008D120208E9
:101F26004C1C002000000000C058040803000000FC
:101F36008D120208401C002000000000042904083D
:101F4600010000000000000000000000000000008A
:101F5600000000000D00000000000000000000006E
:101F660000000000C858040800000000000000003F
:101F76000000000000000000BC560408000000003D
:101F860000000000941C0020040000000C58040807
:101F9600030000008D120208881C002000000000CB
:101FA60004290408010000000000000000000000F1
:101FB60000000000000000000D000000000000000E
:101FC60000000000000000003E91002088136F17FB
:101FD600010000004091002088136F1700000000E8
:101FE6006057040800000000000000000000000028
:101FF6000000000070570408080000000000000000
:10200600C4180020040000007C57040808000000E3
:1020160000000000B818002000000000F02A0408A4
:10202600040000008D870308000000000000000087
:102036000429040801000000000000000000000060
:1020460000000000000000000D000000000000007D
:1020560000000000000000003C91002088136F176C
:1020660001000000C890002088136F1700000000D0
:10207600AD81030800000000D018002094910020D4
:1020860001000000301E0408CA9000200100000074
:102096003C1E0408C090002002000000441E0408F4
:1020A600427A00200000000000000000407A002074
:1020B60000000000000000003E7A00200000000042
:1020C600000000003C7A0020000000000000000034
:1020D6003A7A00200000000000000000387A002054
:1020E6000000000000000000D416002000000000E0
:1020F600000000003B91002002000000501E040872
:10210600BC570408000000000000000000000000AA
:1021160000000000705704080800000000000000DE
:1021260054190020040000007C5704080800000031
:10213600000000004819002000000000F02A0408F2
:102146000400000081810308000000000000000078
:10215600042904080100000000000000000000003F
:1021660000000000000000000D000000000000005C
:102176000000000000000000CC570408000000002A
:10218600000000000000000000000000DC5704080A
:102196000C0000000D100208841900200400000045
:1021A600E85704080C000000B50F02087819002053
:1021B60004000000F45704080C000000D90F0208C0
:1021C6006C190020000000000058040803000000FD
:1021D6006D87030860190020080000000C580408E9
:1021E600030000008D120208881C00200000000079
:1021F600042904080100000000000000000000009F
:1022060000000000000000000D00000000000000BB
:102216000000000000000000FC2804080000000088
:102226000000000000000000000000001458040830
:1022360004000000A9870308000000000000000059
:10224600042904080100000000000000000000004E
:1022560000000000000000000D000000000000006B
:1022660000000000000000006458040800000000A0
:102276000000000000000000000000007C4E040882
:102286000C00000000000000E4190020040000001B
:10229600745804080800000000000000D819002047
:1022A6000400000080580408080000000000000038
:1022B600CC1900200400000088580408080000001B
:1022C60000000000C0190020040000009058040817
:1022D6000800000000000000B419002004000000FF
:1022E600985804080800000000000000A819002003
:1022F60004000000A05804080800000000000000C8
:102306009C19002004000000A858040808000000DA
:1023160000000000901900200400000004290408B1
:1023260001000000000000000000000000000000A6
:10233600000000000D00000000000000000000008A
:10234600000000009981030800000000F019002039
:102356000000000000000000681A002000000000D5
:1023660000000000081B0020C690002004000000AA
:102376005C1E0408C4900020E0150C170000000045
:10238600C3900020080000001C1B0408C290002017
:1023960005000000701E0408000000000000000098
:1023A600581B00202D202D2D202D2D2D2D202D2D9F
:1023B6002D000000000000000000000000000000EA
:1023C60000000000685E0C00BC1C0020000000003D
:1023D60000000000000000000000000000000000F7
:1023E60000000000000000000000000000000000E7
:1023F60000000000000000000000000000000000D7
:1024060000000000000000000000000000000000C6
:1024160000000000000000000000000000000000B6
:102426000000000000000000000000004300000063
:102436000000000000000000000000000000000096
:102446000000000000000000000000004300000043
:102456000000000000000000000000000000000076
:102466000000000000000000000000004300000023
:102476000000000000000000000000000000000056
:102486000000000000000000000000004300000003
:102496000000000000000000000000000000000036
:1024A60000000000000000000000000043000000E3
:1024B6000000000000000000000000000000000016
:1024C60000000000000000000000000043000000C3
:1024D60000000000000000000000000000000000F6
:1024E60000000000000000000000000043000000A3
:1024F60000000000000000000000000000000000D6
:10250600000000000000000000000000D3DA03080D
:10251600AFDA030800000000035C0408E42804089E
:10252600132704081327040813270408132704088D
:10253600132704081327040813270408132704087D
:1025460013270408FFFFFFFFFFFFFFFFFFFFFFFF4B
:10255600FFFF00000100415343494900000000000D
:102566000000000000000000000000000000000065
:1025760000000000000041534349490000000000EC
:102586000000000000000000000000000000000045
:0C25960000000000000000000100000038
:10800000002870B51EDB0928044620DD012303EBA0
:1080100083035B00B0FBF3F2092AF8D87BB10E4E64
:10802000B4FBF3F00928CCBF57223022A6FB03E5AE
:10803000024403FB1044EB0801F8012BF0D10023AC
:108040000B7070BD2D230B7040420131DBE73030E7
:1080500001F8010BF3E700BFCDCCCCCC884230B4A3
:108060004FF001042ED301FB04F4B0FBF4F58D4274
:10807000F9D284B1AAB901E0B0FBF4F5092DCCBF67
:10808000572230222A4404FB150003F8012BB4FBCD
:10809000F1F4002CF0D100221A7030BC7047B0FB14
:1080A000F4F5092DCCBF372230222A4404FB1500F9
:1080B00003F8012BB4FBF1F4002CF0D100221A706C
:1080C00030BC70470546002AEBD1D7E72DE9F047D1
:1080D00014461D46064600234FF47A722046294670
:1080E00035F08CF9DFF840814B4A4C4F88FB00316A
:1080F0000144C31782FB002EC3EB611188FB0128EA
:1081000087FB00278644464AC3EBEE2EC1EB011CD9
:1081100082FB0E29A0EB8C0C0744424A86F806C06D
:10812000C3EB27474FEAEE7C08EB010ACCEBA90C26
:1081300082FB07824FEAE1780CEB4C0CC8EB6A1823
:10814000AEEBCC0EC8EB0818DFF8E0C086F804E010
:10815000A1EB880171718CFB0010F917C1EBE212E1
:1081600040F2B55101FB1272C3EBE050B2F5896FDA
:108170004FEA80073CDA40F2DA239A4242DCB2F559
:10818000B77FB4BF4FF0000C4FF0010C4FEA4C0921
:10819000DFF89C8009EB0C0308EBC3031FFA8CFE8D
:1081A000D88A09EB0C0108EBC10116310B2301E061
:1081B00031F8020D824218DA013BF9D1CC44012397
:1081C00038F83C00B37007F2B2770132121ABE449D
:1081D000F270A6F800E0204629464FF47A72002398
:1081E00035F00CF93281BDE8F0870133DBB2E9E705
:1081F0004FF0030EF44640F29650DFF834804FF013
:108200000609CEE74FF0020EDFF82480F44640F274
:1082100029404FF00409C4E7C5B3A29107452EC217
:10822000ABAAAA2A73B06D1689888888792D0311A4
:10823000F8EB030803685A1C02601970704700BF0E
:108240002DE9F047089C2578002B804689460CBF15
:108250004FF0200A4FF0300A661C35B3002A29DDA2
:10826000334601E0024698B113F8011B501E002965
:10827000F8D1971E60B13D46013D51464046C84782
:108280006B1C002BF8DC257827EAE770013055B12C
:10829000041B29464046C847301916F8015B002DDB
:1082A000F7D1BDE8F087BDE8F087002A04DC284656
:1082B000BDE8F0870020EBE7571EDCE783684268E3
:1082C000D0ED037A00EB83010133934281ED040A80
:1082D000836004BF0023836000EB830393ED047A83
:1082E000036870EE277A9A42C0ED037A77EEC77A78
:1082F000C0ED037A0CDA013307EE103AF8EEC76AE4
:10830000B7EE007A87EEA60A036030EE070A7047E0
:1083100007EE102AB8EEC77A87EE870A704700BFCB
:1083200090ED057A90ED004AD0ED066AD0ED014A55
:10833000D0ED047A90ED035AD0ED025AA4EE007A03
:10834000B0EE406AB0EE470AB0EE667AA6EE247A46
:1083500067EEC07AA0EE457AE6EE257A80ED057AE2
:10836000C0ED067A704700BFD0ED057A90ED013A76
:10837000D0ED003AD0ED064A90ED024A90ED077A32
:1083800090ED035A90ED086AD0ED045AC0ED067ADC
:10839000F0EE406A27EE830AC0ED056AA3EEA60A56
:1083A00080ED087AA4EE240AA5EE470AA5EEC60AD7
:1083B00080ED070A704700BFD0ED007A90ED017A9A
:1083C00030EE670AE7EE007AB0EE670AC0ED007A99
:1083D000704700BF704700BF0A44914214D030B4C8
:1083E0000139551E41F2210211F8014F082380EA9C
:1083F000042004044CBF82EA40004000013B80B2EC
:10840000F7D18D42F0D130BC70474378007840EA14
:10841000032010FB01F04FF4807190FBF1F000F3AA
:108420000F0000B270472DE9F04F654B654EB3F871
:108430000AC03468B3F8048087B04FEA0C2A05906C
:108440001889B4EB0A0A4FF000024FF0000565EB03
:10845000020BA0FB0A4500FB0B55E00940EA456012
:108460004FEA084407198E46D8884FEAE51141EBD8
:108470000208A0FB0A45CDE90278B3F8028000FBB0
:108480000B55200A40EA05604FEAC83410EB040897
:108490004FEA252141EB02099A89A2FB0A0102FB5E
:1084A0000B11C20D42EA412212F5FA604FEAE15384
:1084B00043F10001B0F5FA6FCDE9000171F100015F
:1084C000B4465EDA0524A2FB040104FB031100FBA1
:1084D00003F402FB0144DDE90267A0FB0201214431
:1084E0004D104FEA3004361B4FEA900444EA817481
:1084F00067EB05078D10B8EB040869EB0509DDE9AA
:10850000004531484FF0FF31844275EB0101CDE960
:10851000026723DA40F6AC5012184FF000014B41CD
:1085200002FB03F1A2FB022303EB4103D900D000BD
:10853000101A41EA527163EB0101341847EB01054F
:10854000CDE902450B24A2FB040104FB03114910F1
:108550004FEA3000B8EB000869EB01090AFB0BF3A6
:10856000DDE90001AAFB0AAB0BEB430B4FEADA7221
:1085700042EA4B02801A4FEAEB7361EB0301CDE94B
:108580000001DCF80410A1FB082301FB0933540DA2
:108590005D1544EAC324DDE90223A21A65EB030357
:1085A0001D46D30B059A43EA454302B11360BEF161
:1085B000000F02D0009BCEF8003007B0BDE8F08F6E
:1085C000943D0020901E002024FAFFFF10B5064CB9
:1085D000237A0BB9002010BD08F070FAE368C01AC6
:1085E000D0F5FA50F6D410BD901E00204FF4805301
:1085F00083827047012380F845307047704700BF81
:10860000BFF34F8F0549064BCA6802F4E06213437B
:10861000CB60BFF34F8F00BFFDE700BF00ED00E070
:108620000400FA0570B4037B04681F2B08D9203BB3
:108630002021626801FA03F31A421CD170BC704712
:108640002021226801FA03F31A42F7D04269144943
:108650005C2000FB021251685689CD6808682968C1
:1086600021F001012960828992B222EA0602828108
:10867000A36070BC7047426909495C2000FB02128C
:1086800051685689CD680868296821F00101296080
:10869000828992B222EA06028281E36070BC70474E
:1086A000F47A00202B4B1978002951D02A4B30B492
:1086B0001C68988800226262A5899A80284380B24B
:1086C0000129A08143D09C6898896262A5892843CA
:1086D00080B20229A0819A8139D01C69988A62628D
:1086E000A589284380B20329A0819A822FD09C6952
:1086F000988B6262A589284380B20429A0819A835D
:1087000025D01C6A988C6262A589284380B205290D
:10871000A0819A841BD09C6A988D6262A5892843A7
:1087200080B20629A0819A8511D01C6B988E626256
:10873000A589284380B20729A0819A8607D0986B23
:10874000998F42628489214389B281819A8730BCA2
:10875000704700BFD47D0020D87D0020F0B5C40054
:1087600022189200AE498B585B689D8AADB2EEB27A
:10877000F7070A445CD4B70732D5BFF35F8F167E84
:10878000F6B2012E00F0C780A64D1A8BBFF35F8FA3
:10879000221801EB8202167E022E00F0D5802218EC
:1087A00001EB8202167E032E00F088809A8895F9EC
:1087B000106092B242F480629A80221801EB820229
:1087C000127E013296425BD1AA7C00266E74002A8A
:1087D00040F09580204401EB800000234375F0BDFC
:1087E00077074ED416F0400600F0C9808D4D1E8AE2
:1087F00095F910E0176AF6B207F80E605FFA8EFE80
:108800000EF1010C4FFA8CFC177E85F810C00CF1AC
:1088100003029742664600F01C81221801EB820297
:10882000127E9445C9D10EF1020676B22E74C4E7C9
:108830001E887C4D26F400663604360C1E801E8889
:10884000B6B246F480661E80967E00272F74002EF6
:1088500048D06E7C002E42D0221801EB8202012605
:10886000127E6E74022A00F0B980221801EB820297
:10887000927D42F001021A82204401EB8000037EC7
:10888000F0BD684D967E0127AF74002E73D06E7CCC
:10889000002E7BD1221801EB8202527E002A00F0CA
:1088A000A3801A882E7C92B2013642F4007276B20E
:1088B0001A802E741A88D205FCD47EE7927E002A94
:1088C0003FF474AF6A7C002A3FF470AF9A8895F940
:1088D000106022F480621204120C9A806DE7D27D3F
:1088E000FF2AB9D0221801EB8202967D06F0FE061F
:1088F0001E82D37DFF2BBFD0FF232B74BCE79A8849
:1089000022F4407212042044120C01EB80009A8081
:1089100000234375F0BD927E424D002A3FF435AFEF
:108920006A7C002A3FF431AF1A8822F48062120474
:10893000120C1A80BFF35F8F1A8B1A88AE7492B232
:1089400042F400721A8031E7927E002A3FF427AF8A
:108950006A7C002A3FF423AF1A8895F9106022F44C
:1089600080621204120C1A809A8822F48062120427
:10897000120C9A8021E76A7C002A8BD091E715F0CF
:10898000800F284D3AD195F9106016E7167ED2F87F
:1089900020E01F88022E95F9106045D927F48067E2
:1089A0003F043F0C1F801F8AFFB20EF806701F881D
:1089B000D2F820E0BFB247F400771F80F2B21F8ADE
:1089C000561C76B2FFB20EF806709F88961CBAB29B
:1089D00076B242F480622E749A806BE71A8892B263
:1089E00042F400621A8040E71A8895F9106092B24A
:1089F00042F4807201271A806F745BE795F910705A
:108A0000B7F1FF3F2CD0D669F65D1E8292F818E0D0
:108A100001377AB2964516462A747FF4CEAEA3E7A4
:108A20005C510020901E0020BFB247F400771F80E9
:108A30001F8AFFB20EF80670F6B21F8AD2F820E045
:108A4000721C52B20336FFB276B20EF802702E7468
:108A500030E79A8822F480621204120C9A80DCE6D5
:108A6000D77D1F822E74957E1DB9127E002A7FF459
:108A700003AF9A8822F480621204120C9A80FBE6FB
:108A800007B5032301AA002112F06EFF9DF80530FF
:108A90009DF804001B0243EA00439DF806001843BA
:108AA00003B05DF804FB08B5FFF7EAFF014B58601F
:108AB00008BD00BF901E002008B5FFF7E1FF014B85
:108AC000186008BD901E002038B504460D46FFF71B
:108AD0007DFD246808B108F03DF8054B00221A72AC
:108AE00049215B7A2A46204612F09EFE012038BDBD
:108AF000901E0020014B186812F0E0B87821002089
:108B00000122482112F0F8BF0122582112F0F4BFCF
:108B10002DE9F04F87B0836803900191934613B11C
:108B20001A689B885383012008F014F8039B586847
:108B300040F2E93302E0002B00F049820289013B58
:108B400012F0020F9BB2F6D0BDF80430838140F2E0
:108B5000E93302E0002B00F03A820289013B12F077
:108B6000010F9BB2F6D0838940F2E93302E0002B7B
:108B700000F032820289013B12F0020F9BB2F6D064
:108B80001FFA8BF3838140F2E93302E0002B00F0FF
:108B900023820289013B12F0010F9BB2F6D0838938
:108BA000039B9B6813B11A689B881383012007F00D
:108BB000D1FF642007F0CEFF019B814DDFF81082CA
:108BC000DFF810927F4C804E43F080030293152310
:108BD0000593039B9B6813B11A689B88538307F026
:108BE0006DFF4FF0100C82464FF47A7E0120D9F8C9
:108BF0000430C3F30803002B40F06D81EFF31183C1
:108C0000002B40F068812B68A16800BF2A6893425E
:108C1000F9D1D8F800700EFB07F2521AB2FBF7F246
:108C20000EFB03239A45E2D0039B586840F2E933D8
:108C300002E0002B00F0BA810289013B12F0020F22
:108C40009BB2F6D0BDF80830838140F2E93302E0F0
:108C5000002B00F0AB810289013B12F0010F9BB2A7
:108C6000F6D08389838940F2E93302E0002B00F0DB
:108C70009A810289013B12F0020F9BB2F6D0FF23CA
:108C8000838140F2E93302E0002B00F08C810289FD
:108C9000013B12F0010F9BB2F6D08389DBB2049343
:108CA000039B9B6813B11A689B88138307F006FF28
:108CB0004FF0100C82464FF47A7E0120D9F8043030
:108CC000C3F30803002B40F0EC80EFF31183002B7B
:108CD00040F0E7802B68A16800BF2A689342F9D171
:108CE000D8F800700EFB07F2521AB2FBF7F20EFB37
:108CF00003239A45E2D0049A934500F06481334BF4
:108D0000324ADB880133D380039B9B6813B11A6816
:108D10009B88538307F0D2FE4FF0100C82464FF42D
:108D20007A7E0120D9F80430C3F30803002B40F009
:108D30002081EFF31183002B40F01B812B68A16889
:108D400000BF2A689342F9D1D8F800700EFB07F2F1
:108D5000521AB2FBF7F20EFB03239A45E2D0039BB3
:108D6000586840F2E93302E0002B00F024810289C8
:108D7000013B12F0020F9BB2F6D0BDF804308381A4
:108D800040F2E93302E0002B00F015810289013B3B
:108D900012F0010F9BB2F6D0838940F2E93302E072
:108DA000002B00F00D810289013B12F0020F9BB2F3
:108DB000F6D01FFA8BF3838140F2E9330FE000BF56
:108DC0001454002010E000E010540020F08F002028
:108DD0001854002000ED00E0002B00F0F180028923
:108DE000013B12F0010F9BB2F6D08389039B9B6875
:108DF00013B11A689B88138307F060FE4FF0100CC4
:108E000082464FF47A7E0120D9F80430C3F3080378
:108E1000002B40F09480EFF31183002B40F08F8003
:108E20002B68A16800BF2A689342F9D1D8F8007076
:108E30000EFB07F2521AB2FBF7F20EFB03239A4520
:108E4000E2D007F03BFE4FF0100C82464FF47A7EE2
:108E50000120D9F80430C3F30803002B55D1EFF3F8
:108E60001183002B51D12B68A16800BF2A6893425F
:108E7000F9D1D8F800700EFB07F2521AB2FBF7F2E4
:108E80000EFB0323A3EB0A03632BE2D9059B013BF3
:108E900013F0FF0305937FF49CAE184607B0BDE8BE
:108EA000F08FEFF311818CF31288A7682368DA033F
:108EB00044BF3060A7682B683268C9B281F311885B
:108EC000D8F800101A440EFB01F3DB1BB3FBF1F3DF
:108ED0000EFB02330DE7EFF311818CF31288A768C4
:108EE0002368DB0344BF3060A7682B683268C9B2CF
:108EF00081F31188D8F800101A440EFB01F3DB1B34
:108F0000B3FBF1F30EFB02338CE6EFF311818CF32C
:108F10001288A7682368DB0344BF3060A7682B680A
:108F20003268C9B281F31188D8F800101A440EFBD8
:108F300001F3DB1BB3FBF1F30EFB0233A2E7EFF30C
:108F400011818CF31288A7682368DA0344BF30606C
:108F5000A7682B683268C9B281F31188D8F800106D
:108F60001A440EFB01F3DB1BB3FBF1F30EFB0233E0
:108F700065E7EFF311818CF31288A7682368DB03A0
:108F800044BF3060A7682B683268C9B281F311888A
:108F9000D8F800101A440EFB01F3DB1BB3FBF1F30E
:108FA0000EFB0233D9E612F024FC79E612F021FC24
:108FB000039B586856E612F01CFC039B5868ECE6CD
:108FC00012F017FC12E7012007B0BDE8F08F12F095
:108FD00010FC039B5868C7E512F00BFCE0E500BFEE
:108FE000F0B5876983B0064617B13B68BA885A83E3
:108FF0007069DFF8A4E08389C3244FF47A734FF0DB
:10900000060C6D464FF6FF710EF1010E03E0013BB9
:109010009BB28B4220D002899207F8D5A3B28381FC
:109020004FF47A7302E0A3B28B4215D00289D207C3
:1090300003F1FF34F7D5828992B20DB12A70013560
:10904000BCF1000F0BD00CF1FF3CFF24BEF1000F70
:10905000E1D09EF80040D7E712F0CBFBB76917B11B
:109060003B68BA881A839DF805009DF801509DF869
:1090700002109DF803409DF804209DF8063041EA57
:10908000052143EA002342EA042201203187728746
:10909000B38703B0F0BD00BF58EC0308F8B5057BFB
:1090A000466903681F2D29D9A5F120045F68202196
:1090B000A1400F422A4613D01022A240D960DA60A4
:1090C0005A68E240D10703D5012202FA04F4DC60B9
:1090D0000446304607F06CFF227B23681F2A20D904
:1090E000A2F1200008215A688140114200D0D960C5
:1090F0000422596882400A4221D1F8BD20211C680F
:10910000A9400C422A460CD01022AA4099609A60CD
:109110001A68EA40D207DBD5012202FA05F59D6004
:10912000D6E7082118689140014200D099600421D7
:10913000186801FA02F2024203D09A60F8BDDA60C0
:10914000F8BDF8BDF8B5174D2B78A52B28D16B7855
:10915000BE2B25D1022229464FF6FF70FFF73CF9BE
:10916000114FAC1C22884AB1A618BE4218D2052A5B
:1091700016D92146FFF730F93446F3E7214602229B
:10918000FFF72AF90222A118FFF726F90634074B48
:10919000641B1C8041F60F53C31A58425841F8BD56
:1091A0000020F8BD0040000800800008DC3D0020E1
:1091B0002DE9F04FDFF84C914D4F8BB00326A7EB14
:1091C00009071822002104A835F0A6FC494BCDF868
:1091D000109005971A69002A04DA474A5A6002F18A
:1091E00088325A6001228DF82420F322DA60434B42
:1091F000434C1B88ADF800300222694604A812F0E7
:1092000011FE022269464FF6FF70FFF7E5F8DFF81E
:10921000F8A080464FF0000B544539D30AAC002526
:1092200024F8245D0222214604A812F0FBFD02224C
:1092300021464046FFF7D0F840BAC043ADF80800D9
:10924000022202A904A812F0EDFD079878B106AB3E
:10925000C0F104022946184435F05EFC089818B99C
:10926000069904A812F040FD0023089007939DF88A
:109270002430089A23B11F490B6943F000430B6166
:10928000013E2DD0002A9CD1FFF75CFF50B32CE0AB
:1092900065888DF80DB0C5F30B05AB1DADF8083032
:1092A0002388C3F30B02ADF80A201B0B062202A988
:1092B00004A88DF80C3012F0B5FD062202A9404634
:1092C000FFF78AF8616880462A4604A812F0AAFDD2
:1092D000616840462A46FFF77FF8143480469BE7D2
:1092E000002AD1D0052006F00FFB0BB0BDE8F08FAF
:1092F00000800008003C0240230167455FEC030842
:109300009001000800400008180600080378202B90
:10931000024600F10100F9D0092BF7D02D2B2CD0FB
:109320002B2B03BF5378B7EE000A0246B7EE000AB4
:10933000A3F13001C8B209289FED467A10D8F2EEA9
:10934000046A07EE901AF8EEE77A12F8013FE7EEAA
:10935000267AA3F13001C8B20928B0EE677AF0D9B5
:109360002E2B4CD003F0DF03452B0BD0F7EE007A09
:1093700067EE276A20EE260A70475378BFEE000A90
:109380000246D5E710B451782D2959D02B290ABFB0
:109390009178501C901C0024A1F13003092B53D864
:1093A000002303EB830301EB430310F8011FA1F13A
:1093B0003002092AA3F13003F3D9B3F59A7F28BF0D
:1093C0004FF49A73072B42D9DFED236A1A46F7EE62
:1093D000007A083A072A67EEA67AFAD803F007035C
:1093E0002BB1F2EE046A013B67EEA67AFBD124B3FF
:1093F000C7EE276A5DF8044B20EE260A70475378C3
:10940000A3F13001C8B2092802F10102AAD8F2EE94
:10941000046AF0EE665A07EE901AF8EEE77A12F850
:10942000013F87EEA66AA3F13001C8B2092866EEB3
:10943000A56A37EE067AEED994E767EE276AD9E790
:10944000901C91780124A7E7F7EE007ACFE7F7EEBA
:10945000007AC5E70000000020BCBE4CB5EEC00A93
:10946000DFED317AF1EE10FACCBF30EE270A30EEA4
:10947000670ADFED2E7A20EE270A30B5FDEEC07ABE
:1094800087B017EE904A054684EAE470002303A9EA
:10949000A0EBE4700193009302932AF049FB002CA7
:1094A000ACBF20232D2303A88DF8003033F0FCFA45
:1094B000012803A924D002282DD0032805BF30237A
:1094C000684668468DF8013035F02EFB684633F06B
:1094D000EBFA0338C4B222466946284635F05BFBF6
:1094E00000232B55284633F0DFFA2E22431C2A5442
:1094F0000DEB0401E81835F034FB284607B030BD09
:10950000302368468DF801308DF802308DF8033035
:1095100035F00AFBDAE7302368468DF801308DF824
:10952000023035F001FBD1E76F12033A00007A44B4
:109530002DE9F041064615460846B6FBF2F43CB963
:1095400005FB1464124B1B5D00F8013BBDE8F08184
:10955000B4FBF2F767B90E4B05FB174705FB146424
:10956000DA5D00F8012B1B5D00F8013BBDE8F081DE
:10957000B7FBF2F8B8F1000F02D04046FFF7D8FF72
:1095800005FB1878024B13F8082000F8012BE3E7DD
:1095900058210408104B2DE93048D3E9004554EA1E
:1095A00005020BD1034601220020187158719871F1
:1095B0009A70DA7018801881BDE83088074B1A68F5
:1095C00014EB020B45F1000C5A466346FEF77EFD94
:1095D0000120BDE8308800BFE021002014540020A5
:1095E000F0B402888578154FC37804794179A2F2E6
:1095F000B27202F0030606EB4606013D05EB860556
:10960000013B37F815608579008940F2B55792081B
:1096100007FB0232931903EB430304EBC303C3EBD1
:10962000031301EB8303C3EB031305EB8303002157
:109630004FF47A72C2FB0301F0BC7047F8EB0308E9
:10964000FAB170B48E18044603E0101A14D1B14276
:1096500014D014F8012BA2F14103192B11F8013B8E
:10966000A3F1410598BF2032192D03F12000ECD958
:10967000D01A01D1002BEAD170BC7047002070BC19
:1096800070471046704700BF4FF0FF32FFF7D8BF5A
:10969000A0F16103192B98BF20387047A0F1410356
:1096A000192B98BF20307047202805D0093804288E
:1096B0008CBF0020012070470120704761381928B5
:1096C0008CBF002001207047413819288CBF002032
:1096D00001207047303809288CBF002001207047D6
:1096E000A0F13003092B07D920F0200041381928B8
:1096F0008CBF0020012070470120704730B4026801
:109700001146531C036011F8024B0160D31C5178C1
:1097100003609378151D05601B0443EA0123D0788C
:10972000234343EA006030BC704700BF0368591C04
:109730001A46016012F8021B0260587841EA0020C4
:10974000704700BF03685A1C02601878704700BF5A
:1097500038B504460068154635F0B9F922682A4440
:10976000226038BD036810B40A0E5C1C04601A70D5
:1097700003680A0C5C1C04601A7003680A0A5C1C0B
:1097800004601A7003685A1C026019705DF8044B7B
:10979000704700BF036810B40A0A5C1C04601A70AA
:1097A00003685A1C026019705DF8044B704700BFD3
:1097B00003685A1C026010B4197003680A0A5C1C22
:1097C00004601A7003680A0C5C1C04601A70036859
:1097D000090E5A1C026019705DF8044B704700BFF7
:1097E00003685A1C026019700368090A5A1C026057
:1097F000197070472DE9F047002488B080460F4665
:109800001E46A14605AD531C0393117839B3252993
:1098100033D1931CCDF810900393507830284ED05C
:109820004FF0000AA0F13003DBB2092B42D96C28BB
:1098300019D0642800F0938024D825281CD063D93F
:10984000582876D063281BD131784046B847039A10
:10985000531C03931178043601340029D7D12046D4
:1098600008B0BDE8F087039B5A1C03921B78642B59
:109870007CD02AD8252B54D1252140460134B84725
:10988000039AC0E7732833D044D975284FD106F125
:10989000040E30682B4600220A217646FEF7DEFBD6
:1098A000049A0095534639464046FEF7C9FC039A90
:1098B0000444A8E704AA03A92AF016F9B7E7D31CC1
:1098C000039390784FF0010AACE7732B10D05BD96B
:1098D000752B3AD0782B96D1A3F15802B2FA82F2C6
:1098E000306852092B4610210436FEF7B7FBD7E744
:1098F0003368049A0093394600234046FEF7A0FCE3
:1099000004360444039A7EE70028B9D1204608B003
:10991000BDE8F0876E28B3D1039A336804361C6023
:1099200071E72AD9582BD7D0632B8DD06BE77828D5
:10993000A6D1A0F15802B2FA82F2306852092B4641
:109940001021FEF78BFB0436AAE706F1040E3068FF
:109950002B4600220A217646FEF780FBA0E7331D46
:10996000306829461E46FEF74BFB99E7331D3068E9
:1099700029461E46FEF744FB92E7002B7FF443AFD7
:10998000204608B0BDE8F0876E2BC6D03BE700BF8D
:109990000EB400B584B005AB019053F8042B064912
:1099A000039301A8FFF726FF019B00221A7004B061
:1099B0005DF804EB03B07047358200082DE9F047ED
:1099C000484BB3F914708CB00646002F56D13D4673
:1099D0003C460A8840F2B1739A4203D98B78581EEC
:1099E0000B282FD9002301201946ADF824308DF81B
:1099F00028308DF829308DF82A30ADF82C309C466F
:109A00009A4699461A46984686468DF826008DF85D
:109A100027000346002CACBF2B242D24049107956E
:109A20000697CDF80CC0CDF808A0CDF80490CDF87D
:109A300000E0304605942C49FFF7AAFF40460CB0E1
:109A4000BDE8F08791F803E00EF1FF301E28C9D879
:109A500091F80490B9F1170FC4D891F805A0BAF1A4
:109A60003B0FBFD891F806C0BCF13B0FBAD80989AB
:109A7000B1F57A7FB6D24FF00108CBE71B4C84FBDF
:109A80000734E319FC17C4EB6314C4EB0415A7EB0C
:109A900085052DB2002D0846B8BF6D42FFF7A0FD29
:109AA0004FF47A7200238046894633F0A7FC3C23AA
:109AB00007FB03074FF47A7200234046494633F010
:109AC0009DFC24B24FF47A7192B20023C1FB0723AC
:109AD00009A884EAE477FEF7F9FAA7EBE47709A985
:109AE00077E700BF901E00208021040889888888BD
:109AF0000FB430B583B006AB0A490B4853F8042BBA
:109B0000096800680193FFF775FE084C0546206858
:109B100011F0C5F80028FAD0284603B0BDE830405F
:109B200004B07047205100202451002078210020EB
:109B3000DFED2B7AB4EEE70AF1EE10FA4ADDDFED45
:109B4000296A9FED297A01E0B0EE670AB4EEC70AF0
:109B5000F1EE10FA70EE667AF6DC9FED247AF4EE00
:109B6000C77AF1EE10FA38D5DFED1E6A9FED207A44
:109B700001E0F0EE407AF4EEC77AF1EE10FA37EE3B
:109B8000A60AF6D4DFED1B7AB4EEE70AF1EE10FA7E
:109B900014DDDFED137A37EEC00A60EE006A9FED48
:109BA000166A9FED167ADFED167AA6EE867A20EE1B
:109BB000266AE6EE877AA6EE270A7047DFED117A6D
:109BC000B4EEE70AF1EE10FA44BFDFED087A37EEA3
:109BD000C00AE2E7F0EE407ABFE7B0EE670AD1E7ED
:109BE000DB0F4940DB0FC940E4CB1641DB0F49C016
:109BF000E4CB16C1DB0FC93F92E741B99730083C6F
:109C000015A82ABEDB0FC9BF80EAE073A3EBE0739F
:109C10008B4205DB002801DD401A704702D17047F6
:109C2000002070470844704709B909E0194690FBC5
:109C3000F1F301FB13030846002BF7D108467047E8
:109C40000146FBE7F0EEC07AB0EEE07AB4EEE77AD8
:109C5000F1EE10FAB4BFB0EE676AB0EE476AB5EE47
:109C6000406AF1EE10FA46D0B4EEE77AF1EE10FA5F
:109C70008CBFF0EE675AF0EE475AC5EE866A9FED4C
:109C80001F3A9FED1F6A9FED1F4A9FED1F5ADFEDA0
:109C90001F3ADFED1F4ADFED1F5AA6EEC36AE6EE5C
:109CA000A34AA6EE864AB7EE006AA6EE845AA6EE4E
:109CB000A46AE6EE855AC5EE866AB4EEE77AF1EE5E
:109CC00010FA48BFDFED147AF5EEC00A48BF77EE10
:109CD000E66AF1EE10FA48BFDFED107AB5EEC00A81
:109CE00048BF77EEE66AF1EE10FA48BFF1EE666A19
:109CF000B0EE660A7047DFED076ADEE739094E3DD0
:109D0000E3B59E3E88FA163E45FE7F3F99FB243F11
:109D100069A2163EA7DFA834DB0FC93FDB0F49401D
:109D2000DFED317A30EE277AFDEEC76A16EE903A13
:109D30002033402B02D99FED2D0A7047B4EEE70A7D
:109D4000F1EE10FA4DDD9FED2A6ADFED2A6A01E09F
:109D5000B0EE677AB4EEE67AF1EE10FA77EE467A74
:109D6000F6DC9FED257AF4EEC77AF1EE10FA35D5E0
:109D7000DFED1F6A9FED217A01E0F0EE407AF4EE0C
:109D8000C77AF1EE10FA37EEA60AF6D4DFED167AAE
:109D9000B4EEE70AF1EE10FA1BDCDFED197AB4EE4F
:109DA000E70AF1EE10FA44BFDFED137A37EEC00A8E
:109DB00060EE006A9FED136A9FED137ADFED137A70
:109DC000A6EE867A20EE266AE6EE877AA6EE270AC7
:109DD0007047DFED0F7A37EEC00AE9E7B0EE670AA9
:109DE000D4E7F0EE477ABCE7DB0FC93F0000000084
:109DF000DB0FC940E4CB1641DB0F49C0E4CB16C1F1
:109E0000DB0FC9BF92E741B99730083C15A82ABEBD
:109E1000DB0F4940FDEEC07A17EE903A2033402B1D
:109E200051D8DFED2D7AB4EEE70AF1EE10FA50DDED
:109E3000DFED2A6A9FED2A7A01E0B0EE670AB4EE00
:109E4000C70AF1EE10FA70EE667AF6DC9FED257A1D
:109E5000F4EEC77AF1EE10FA38D5DFED206A9FED07
:109E6000227A01E0F0EE407AF4EEC77AF1EE10FAD1
:109E700037EEA60AF6D4DFED1D7AB4EEE70AF1EE6E
:109E800010FA1BDCDFED1A7AB4EEE70AF1EE10FAF5
:109E900044BFDFED147A37EEC00A60EE006A9FED32
:109EA000156A9FED157ADFED157AA6EE867A20EE1B
:109EB000266AE6EE877AA6EE270A7047DFED067A75
:109EC00037EEC00AE9E79FED0E0A7047B0EE670A69
:109ED000D1E7F0EE407AB9E7DB0F4940DB0FC9402C
:109EE000E4CB1641DB0F49C0E4CB16C1DB0FC93F01
:109EF000DB0FC9BF92E741B99730083C15A82ABECD
:109F00000000000007EE901AF8EE677A9FED837A62
:109F100027EE800A20EE070AFDEEC07A17EE903A8F
:109F20002033402B00F28C80DFED7D7AB4EEE70A1F
:109F3000F1EE10FA40F3E880B0EE407A9FED796AD6
:109F4000DFED796A01E0B0EE677AB4EEE67AF1EE21
:109F500010FA77EE467AF6DC9FED747AF4EEC77A63
:109F6000F1EE10FA40F1CD809FED6E6ADFED706A80
:109F700001E0F0EE477AF4EEE67AF1EE10FA37EE11
:109F8000867AF6D4DFED6B7AB4EEE77AF1EE10FA6A
:109F900051DCDFED697AB4EEE77AF1EE10FA44BFF6
:109FA000DFED627A37EEC77A27EE076ADFED635A94
:109FB000DFED637ADFED636A9FED635AE6EE257AA3
:109FC00067EE065AE6EE276AF7EE007AA5EEA67A65
:109FD000F0EE675AE7EE055AE7EE457A87EEA55AA6
:109FE000DFED547A30EE277AFDEEC76A16EE903A2E
:109FF0002033402B29D99FED557AF6EE006AB7EE53
:10A00000006AF7EE004AC4EEA57A0023836143613B
:10A010000362C36180ED045A67EEA66A27EE866A82
:10A0200027EE877AC0ED006AC0ED026A80ED016A12
:10A0300080ED037A7047DFED3A7A37EEC77AB3E7FF
:10A04000B7EE005AF0EE455ACAE7B4EEE70AF1EE71
:10A0500010FA5FDD9FED336ADFED336A01E0B0EEA9
:10A06000677AB4EEE67AF1EE10FA77EE467AF6DC2D
:10A070009FED2E7AF4EEC77AF1EE10FA47D59FEDF8
:10A08000296ADFED2B6A01E0F0EE477AF4EEE67A1A
:10A09000F1EE10FA37EE867AF6D4DFED267AB4EEDA
:10A0A000E77AF1EE10FA27DCDFED237AB4EEE77AF7
:10A0B000F1EE10FA44BFDFED1D7A37EEC77A27EED6
:10A0C000076ADFED1E4ADFED1E6ADFED1E7AE6EE5F
:10A0D000246A67EE064AE6EE267AB7EE006AA4EE38
:10A0E000A77AF6EE006A36EE476AF8EE007A27EEB7
:10A0F000277A66EE266A84E7DFED097A37EEC77ABB
:10A10000DDE7B0EE677A3DE7F0EE407A24E7B0EEA7
:10A11000677AC2E7F0EE477AAAE700BF27D4D236C3
:10A12000DB0F4940DB0FC940E4CB1641DB0F49C0D0
:10A13000E4CB16C1DB0FC93FDB0FC9BF92E741B9C2
:10A140009730083C15A82ABEF304353F0000008074
:10A1500070B406688E4217D90139751E002311F8B4
:10A16000014F0822634013F0800F4FEA430318BFEA
:10A1700083F0D503013ADBB2F5D18D42EFD1721CE9
:10A180000260337070BC70470023F8E710B44C09CC
:10A19000012250F8243001F01F0102FA01F10B43B3
:10A1A00040F824305DF8044B704700BF4B0901F0C4
:10A1B0001F0150F82320012303FA01F1114214BFBB
:10A1C00018460020704700BF074A084B10781B78DC
:10A1D000074A834296BFC31AC3F180030020126866
:10A1E00018441044704700BFFD2C0020802D002033
:10A1F0001C310020064A074B10781B7883428ABF27
:10A20000C3F18003C01AC018C0F17F00704700BFBF
:10A21000FD2C0020802D0020F0B55FEA930E33D096
:10A2200000F1100601F1100502F11004774616ED59
:10A23000046A55ED044A56ED026A15ED025A16ED10
:10A24000037A55ED035A56ED017A26EE246A66EE3E
:10A25000856A04ED046A15ED016A44ED026A27EE91
:10A26000257A67EE867A013F04ED037A44ED017AA0
:10A2700006F1100605F1100504F11004D7D14FEADC
:10A280000E1420442144224413F003030BD000EBAE
:10A290008303F0EC017AB1EC017A67EE877A8342AE
:10A2A000E2EC017AF5D1F0BD08B511F017FB0A20F8
:10A2B00006F050FC012008BDF8B50F4D46686A72E3
:10A2C0001446027A0F4642F0800225213046FFF7FD
:10A2D000EBFF3A4626213046FFF7E6FF04F00F0277
:10A2E00042F0800227213046FFF7DEFF06F0E6FB52
:10A2F000E86001202872F8BD901E002070B5047837
:10A30000032C0E46154603D0BDE8704011F0F4BB97
:10A310004468027A25212046FFF7C6FF32462621EF
:10A320002046FFF7C1FF2A4663212046FFF7BCFF06
:10A33000812227212046FFF7B7FF012070BD2DE9BC
:10A34000F0410478032C884617461E4621D1446804
:10A35000027A252142F080022046FFF7A5FF4246FF
:10A3600026212046FFF7A0FF06F00F0242F08002F0
:10A3700027212046FFF798FF042006F045FC72B61F
:10A38000492133463A46204611F04EFA62B6BDE8FE
:10A39000F081BDE8F04111F0E7BA37B500F10C04E7
:10A3A000054600220A212046FFF7A8FF0F220A21B6
:10A3B0002046FFF7A3FF01AA032310212046FFF741
:10A3C000BEFF9DF8043080336B839DF805308033E9
:10A3D000AB839DF806308033EB8300220A212046B0
:10A3E000FFF78CFF0DF10302012302212046FFF746
:10A3F000A6FF01230DF1030209212046FFF79FFF6D
:10A4000011220A212046FFF779FF012003B030BD59
:10A410002DE9FF47037B0546884600F10C061BB17A
:10A42000022B06D9032B3DD00024204604B0BDE802
:10A43000F08701230DF1070202213046FFF77FFF6D
:10A440000028F1D09DF80730D907EDD5072302AADF
:10A4500003213046FFF773FF0446002CE4D09DF83B
:10A460000E7011220A213046FFF748FF3B07DBD46C
:10A47000B5F91A1002A8FDF7C8FF4042A8F800007D
:10A48000B5F91C100DF10A00FDF7BFFF4042A8F816
:10A490000200B5F91E1003A8FDF7B7FF4042A8F867
:10A4A0000400C2E7224F4FF0010A0024B946BB7DE9
:10A4B000012B1BD00FD3022BCFD1FEF787F881469B
:10A4C0000028B1D102A905F11000FEF7FDFA87F8C6
:10A4D00016900446C1E73B7A23B901220221304697
:10A4E000FFF7EAFE012389F816309DE7FEF76EF8C4
:10A4F000002899D102A905F11000FEF7E5FA9DF8B0
:10A500000830044608B1DA0707D4002389F816306A
:10A51000BAF1000F88D09A46C9E73B7A23B90722DF
:10A5200003213046FFF7C8FE022389F816307BE787
:10A53000901E002008B540F2E93300E0A3B1028983
:10A54000013B12F0020F9BB2F8D089B2818140F238
:10A55000E93300E043B10289013B12F0010F9BB2E5
:10A56000F8D08089C0B208BD11F043F9C0B208BD6F
:10A5700038B504460D4600BF806810F0E1FF29465B
:10A580006068FFF7D7FFA06810F0DFFF00BF38BD9D
:10A59000F8B584894FF6FF764FF47A7433B319B364
:10A5A0000F78013101E0B44218D00589013CAD07B4
:10A5B000A4B2F8D5BCB284814FF47A7402E0BCB284
:10A5C000B4420BD00589ED0704F1FF37F7D5858933
:10A5D000ADB20AB115700132013BDFE711F009F9A4
:10A5E000003018BF0120F8BDFF27DEE70120F8BDCD
:10A5F00030B5134C237883B01BB90120237003B00E
:10A6000030BD1049052200230D688DF804208DF817
:10A61000053000BFA86810F093FF6A4601A9022325
:10A620006868FFF7B5FFA86810F08FFF00BF9DF8BE
:10A63000013003F0010383F00100237003B030BD4B
:10A64000895400204454002070B5064C0646256805
:10A6500003E023685B1BB34203D8FFF7C9FF002860
:10A66000F7D070BD145400202DE9F04F89B0B2F13D
:10A67000000A02900491039340F3C5800B46002228
:10A6800001EB8A0153F8040B8B420244FAD1039B7D
:10A690000592002B00F0AF80059B002B7CD05E4B19
:10A6A000059A1B68DFF8889100920099DAB2511878
:10A6B000B1F5807F8CBFC2F58072009A0192574A33
:10A6C00092689A4240F28280554A1178002206929E
:10A6D0008DF81C2002228DF81820002960D01A0E57
:10A6E0008DF819200DF11A021C0C190A93701470C0
:10A6F00051700620FFF7A8FF0621D9F80000FFF7E8
:10A7000037FF484A0123137000BFD9F8003098681A
:10A7100010F016FF424BD9F800201B785068002B30
:10A7200006A90CBF042305230022FFF731FF0024F4
:10A73000049D029E019FA34629684FEA84080022D7
:10A740000B46013471B1B9422DD2D9F800003168FD
:10A750004068FFF71DFF2A68336813443360BF1A4F
:10A76000C5F800B0A24505F1040506F10406E3D1E1
:10A77000D9F80030986810F0E8FE00BF264B019928
:10A7800000981B68421A0092234A0B441360039AF4
:10A790004AB3009A002A88D1059809B0BDE8F08F25
:10A7A0000DF11902A0E7029CD9F8003054F8081006
:10A7B000586800223B46FFF7EBFE54F808202B6850
:10A7C0003A44DF1B44F808202F60D1E70598009C2D
:10A7D0001549164A001B0590059800230B7013704D
:10A7E00009B0BDE8F08F059B009A9B1A0593059868
:10A7F00009B0BDE8F08FFFF7FBFE00287FF44CAFF7
:10A80000039B0593C8E7039C1CB9FFF7F1FE059471
:10A81000C2E700230593BFE71C3100200C11002084
:10A820008854002089540020FD2C0020802D002019
:10A83000445400202DE9F047DFF8F4903A4E99F89F
:10A8400000303478394FA3420D4607EB030E99BF11
:10A850000021E31AC3F18003214692465A1886B0BC
:10A860002A443F2A04978046CDF80CE001910093DA
:10A87000059002952BD96946032203A80023FFF710
:10A88000F3FE9DE80600A1B399F800301844C0B269
:10A890000306337848BF80F08000834289F80000C7
:10A8A0003CD0029D2A440A447F2A0DD9BAF1000FF8
:10A8B0001CD00123694603A80322FFF7D5FE00231D
:10A8C000337089F8003011E0DDF814803478C4F179
:10A8D0008009A94528BFA94638194C44E4B24A4624
:10A8E000414634F0F4F8802C34700BD006B0BDE84B
:10A8F000F087002AC8D1029D327089F80020002D0F
:10A90000F4D0CFE7A5EB090508EB09012A46074873
:10A9100034F0DDF8357006B0BDE8F0870023029D05
:10A92000337089F80030BDE7FD2C0020002D002099
:10A93000802D002070B5104D104E2B7831788B4251
:10A9400084B016D00E4A03921A4402928CBF0C4671
:10A95000CA1A04A98CBFC3F180020024012341F864
:10A96000102D02A802220194FFF77EFE002333700F
:10A970002B7004B070BD00BF802D0020FD2C002086
:10A98000002D002070B5194C194D23782978994273
:10A9900084B027D0174A03921A44029234BF0E465D
:10A9A000CA1A04A934BFC3F180020026002341F86B
:10A9B000102D02A802220196FFF756FE23781844B4
:10A9C000C0B203062B7848BF80F08000834220701D
:10A9D00002D0002004B070BD002301202B70237032
:10A9E00004B070BD012004B070BD00BF802D0020F8
:10A9F000FD2C0020002D002010B50C4C45F2082045
:10AA0000FFF722FE20680621FFF7B2FD084B206801
:10AA10000122C7211A70FFF7ABFD06480649074A15
:10AA2000002303700B70136010BD00BF445400205E
:10AA300089540020FD2C0020802D00201C31002096
:10AA4000F0B51F4C83B0277800234FF0030E00931E
:10AA50000E4615468DF804308DF800E06FB3030EF6
:10AA60008DF801300DF10203010C020A9870197083
:10AA700006205A70FFF7E8FDE8B100BF114F3B68B0
:10AA8000986810F05DFD23783A68002B14BF052309
:10AA90000423694650680022FFF77AFD3B6832467E
:10AAA000002158682B46FFF773FD3B68986810F04B
:10AAB0004CFD00BF284603B0F0BD0DF10103D3E704
:10AAC0008854002044540020F0B5124B9D6885B096
:10AAD0000DB905B0F0BDED0A14D0002704AE7C1905
:10AAE0006410E00210226946FFF7AAFF0F2809DD73
:10AAF0006B4653F8042B01320AD1B342F9D12546F3
:10AB0000AF42ECDBFFF716FF034BED021D60E0E701
:10AB1000671CF5E70C1100201C310020084B70B5B4
:10AB20009B68154682189A4288BF1D1A04460E4635
:10AB3000FFF700FF2A4631462046BDE870407FE718
:10AB40000C110020144B984224D003F580639842E6
:10AB500020D0038823F040031B041B0C03800388D0
:10AB600023F038031B041B0C59B141F480710029F8
:10AB700091FAA1F2B2FA82F108BF4FF0FF31013928
:10AB8000C900194389B2018003889BB243F0400396
:10AB9000038070474908DCE7003800400C4B9842BE
:10ABA00013D0A3F5806398420FD003F580439842F9
:10ABB0000BD003F58063984207D003F58063984279
:10ABC00003D0044B186840087047024B1868704760
:10ABD00000040140B45B0020F0B5774B774A87B0A2
:10ABE0001968914200AF00F0DB800023744A3B609B
:10ABF0007B60136843F48033136003E03B68B3F574
:10AC0000A04F09D0136803F400337B603B68013325
:10AC10003B607B68002BF1D0694B1B6813F4003359
:10AC200018BF01237B607B68012B7BD0654D644B93
:10AC3000654AEA606549586F654A0860AA605E6BBC
:10AC4000644C654A654826F080065E635E6F46F098
:10AC500080765E67196B0C431C63596B5963996B63
:10AC60009963196C41F05B5141F47B1141F41F6110
:10AC700041F00F011964596C07F118040A4348F2B6
:10AC8000FF715A6444F8101D002621460123FB730E
:10AC90003E737E73BE7320F0E5FB21464FF6FF73D3
:10ACA0004F48BB6020F0DEFB4FF6FF7321464D4856
:10ACB000BB6020F0D7FB21464B4820F0D3FB214658
:10ACC0004A4820F0CFFB2146494820F0CBFB2146E3
:10ACD000484820F0C7FB2146474820F0C3FB2146E7
:10ACE000464820F0BFFB204620F08CF9444B454CF1
:10ACF0001B68BA6844484549A4FB03439B09A0FB71
:10AD00000202013B920CB3F1807F0A6007D2404AF5
:10AD1000F0200721536085F82300966011601C37EE
:10AD2000BD46F0BD264B3B4D1A6C3B4842F080526D
:10AD30001A642C684268816844F440442C609C6822
:10AD40009C609C6844F400449C609C6844F4A0545B
:10AD50009C600068120642EA801242F480024908B0
:10AD600042F00802013942EA01425A601A6842F090
:10AD700080721A601A689201FCD52849104A40F284
:10AD800005700860996821F003019960996841F0A5
:10AD900002019960936803F00C03082BFAD145E790
:10ADA00000221A6062B61E4B1B6883F308881D4B95
:10ADB0001B689847FEE700BFFCFF0120EFBEADDE39
:10ADC0000038024000ED00E00005FA05407E00205A
:10ADD00000000008FF916700335F07000000024099
:10ADE0000004024000080240000C02400010024033
:10ADF0000014024000180240001C024000200240E3
:10AE0000B45B0020D34D621083DE1B431854002036
:10AE100010E000E00070004000000020003C024014
:10AE20000000FF1F0400FF1F08B5054B1B6803B19E
:10AE30009847044B044A1A6072B6FDF7E1FB00BF65
:10AE4000B4390020FCFF0120EFBEADDE2DE9F04F4C
:10AE500090F8553087B00446002B40F067830DF121
:10AE600010082F4BDB7D002B00F02083636904F179
:10AE700010062C4A934200F01783A2F574429342C5
:10AE800000F00B83284A934200F0058327498B4248
:10AE900014BF082100211A8822F040021204120C6B
:10AEA0001A801A8892B222F0380211431980198848
:10AEB00089B241F0400119804246304606234321C1
:10AEC00010F052FD48B39DF812609DF813309DF8C4
:10AED00010509DF811109DF814009DF8152043EABC
:10AEE00006231BB241EA052142EA0022638721873B
:10AEF000A2875BB2013304D194F93830013300F0FA
:10AF0000FD846369074A934200F0BD82A2F5744252
:10AF100093420DD007B0BDE8F08FB4F93A30E8E7BE
:10AF2000901E00200030014000380040003C0040EE
:10AF3000AD4A538D9BB2002BECD0022302EB0312DF
:10AF4000002353810A23A94DA94FAA4CAA4E03936B
:10AF50003220DFF8BC9223F029FF4FF4FA7A4FF049
:10AF6000100C4FF47A70D9F80430C3F30803002BA7
:10AF700040F0E081EFF31183002B40F0DB81296882
:10AF8000A26800BF2B689942F9D1D7F800E000FB16
:10AF90000EF39B1AB3FBFEF300FB01314FF0010EE1
:10AFA0000191D9F80430C3F30803002B40F06E81FF
:10AFB000EFF31183002B40F069812B68A16800BF7B
:10AFC0002A689342F9D1D7F800B000FB0BF2521A6D
:10AFD000B2FBFBF200FB0323019A9B1AB3F57A7FC5
:10AFE000DFD3BAF1010ABED1844B1978844BC1F387
:10AFF0004001586810F0AEFA804B1978804BC94375
:10B00000186801F0010110F0A5FA072302937C4BA8
:10B010005A6832B11368928859690A4214BF5A8338
:10B020001A83774B1A6832B11368928859690A42B9
:10B0300014BF5A831A83734B1B88002B40F0D181B5
:10B04000714A724B1178186810F084FADFF8C091D9
:10B050004FF0FA0A4FF0100C4FF47A70D9F8043020
:10B06000C3F30803002B40F09F81EFF31183002B03
:10B0700040F09A812968A26800BF2B689942F9D1F3
:10B08000D7F800E000FB0EF39B1AB3FBFEF300FBC6
:10B0900001314FF0010E0191D9F80430C3F30803D8
:10B0A000002B40F02B81EFF31183002B40F0268121
:10B0B0002B68A16800BF2A689342F9D1D7F800B085
:10B0C00000FB0BF2521AB2FBFBF200FB0323019AC6
:10B0D0009B1AB3F57A7FDFD3BAF1010ABED1484B90
:10B0E0005A6832B11368928859690A4214BF5A8368
:10B0F0001A83434B1A6832B11368928859690A421D
:10B1000014BF5A831A833F4B1B88002B40F0788171
:10B110003D4A3E4B1178186881F0010110F01AFA8F
:10B12000DFF8EC904FF0FA0A4FF0100C4FF47A7001
:10B13000D9F80430C3F30803002B40F01881EFF373
:10B140001183002B40F013812968A26800BF2B688F
:10B150009942F9D1D7F800E000FB0EF39B1AB3FB3C
:10B16000FEF300FB01314FF0010E0191D9F80430DC
:10B17000C3F30803002B40F0A580EFF31183002BED
:10B1800040F0A0802B68A16800BF2A689342F9D1E3
:10B19000D7F800B000FB0BF2521AB2FBFBF200FB37
:10B1A0000323019A9B1AB3F57A7FDFD3BAF1010A20
:10B1B000BED1029B013B13F0FF0302937FF427AF44
:10B1C0004FF47A7ADFF8489050464FF0100CD9F8D7
:10B1D0000430C3F30803002B40F03881EFF31183F0
:10B1E000002B40F0338115E0585400201454002007
:10B1F0001854002010E000E010540020DC53002020
:10B20000E0530020EC530020EE530020F0530020C8
:10B2100000ED00E02968A26800BF2B689942F9D1CF
:10B22000D7F800E000FB0EF39B1AB3FBFEF300FB24
:10B2300001314FF0010E0191D9F80430C3F3080336
:10B24000002B40F0E780EFF31183002B40F0E28009
:10B250002B68A16800BF2A689342F9D1D7F800B0E3
:10B2600000FB0BF2521AB2FBFBF200FB0323019A24
:10B270009B1AB3F57A7FDFD3BAF1010AA7D1039BFA
:10B28000013B03937FF464AEFFF7CEFDEFF311882B
:10B290008CF31288A1682368DB0344BFC6F800E082
:10B2A000A1682B6832685FFA88F888F31188D7F8AC
:10B2B00000801A4400FB08F35B1AB3FBF8F300FBB1
:10B2C000023389E6EFF311888CF31288A1682368B2
:10B2D000DB0344BFC6F800E0A1682B6832685FFA60
:10B2E00088F888F31188D7F800801A4400FB08F327
:10B2F0005B1AB3FBF8F300FB023352E7EFF311885C
:10B300008CF31288A1682368DB0344BFC6F800E011
:10B31000A1682B6832685FFA88F888F31188D7F83B
:10B3200000801A4400FB08F35B1AB3FBF8F300FB40
:10B330000233CCE6EFF311828CF31288D4F808E0E4
:10B340002368D90303D501233360D4F808E02B68C0
:10B350003168D2B282F311883A68194400FB02F3D3
:10B36000A3EB0E03B3FBF2F300FB013116E6EFF3A0
:10B3700011828CF31288D4F808E02368D90303D52E
:10B3800001233360D4F808E02B683168D2B282F32D
:10B3900011883A68194400FB02F3A3EB0E03B3FBD8
:10B3A000F2F300FB0131DEE6EFF311828CF3128839
:10B3B000D4F808E02368D90303D501233360D4F817
:10B3C00008E02B683168D2B282F311883A681944D8
:10B3D00000FB02F3A3EB0E03B3FBF2F300FB01311E
:10B3E00057E6B84B5A69002A3FF430AEB64A19689E
:10B3F0001088B64A92FBF0F201200A60587425E6E4
:10B40000B04B5A69002A3FF48BAE196800220A60DB
:10B410005A7485E6EFF311888CF31288A1682368CB
:10B42000DB0344BFC6F800E0A1682B6832685FFA0E
:10B4300088F888F31188D7F800801A4400FB08F3D5
:10B440005B1AB3FBF8F300FB023310E7EFF3118252
:10B450008CF31288D4F808E02368D90303D50123BC
:10B460003360D4F808E02B683168D2B282F31188D7
:10B470003A68194400FB02F3A3EB0E03B3FBF2F3AB
:10B4800000FB0131D5E6924A53899BB2002B3FF471
:10B4900041AD002352E50021FDE402218C4A02EB7C
:10B4A000011200215181EDE40021F7E76369894A27
:10B4B000934200F0FE8088498B420CBF3021382136
:10B4C0001A8822F040021204120C1A801A8892B2D2
:10B4D00022F03802114319801A8892B242F04002D9
:10B4E0001A80A36904F1100613B11A689B8853836C
:10B4F000012005F02FFB606940F2E93304E0013BD5
:10B500009BB2002B00F0D78002899107F7D56B23FF
:10B51000838140F2E93304E0013B9BB2002B00F051
:10B52000CA800289D207F7D58389C7E01D09013D8A
:10B53000022D03F00F0300F2FF81684A32F8150074
:10B5400040FA03F2D60740F1F781012606FA03F329
:10B55000013B184031F0A2FF614BDFF89CA113F8CA
:10B56000059081441AEBC90500F0E6815AF83900CC
:10B57000AF8802693A407FF472AC00F13F4303F5B3
:10B580007E035849EA719B0ACB5C03F01F025B09FA
:10B590002021032B06FA02F2A97100F0C881042BC6
:10B5A00000F0C081022B03D14F494B6C1A434A640F
:10B5B0000DF1100841460026049705961FF052FF32
:10B5C000AA884A4BE360B2FA82F2C2F11F02501C11
:10B5D00004F10C0100F0A381D3B203F0FC0707F1E2
:10B5E000804707F59C3703F00300D7F808C05AF8E6
:10B5F00039304FEA800E0F2000FA0EF02CEA0000DE
:10B60000DFF8F8C003F13F434CF8221003F57E0346
:10B61000B860C3F38720BB683549DFF8E4C000FA9F
:10B620000EF04FF00109184309FA02F3B8604B61BC
:10B630000F68DFF8D0E0D84307400F604F6807403D
:10B640004F600F681F430F608F6807408F60CF689F
:10B650003840284FC860DCF800103A44194392F88B
:10B660006C20CCF800101EF80210F02918DDBB1871
:10B67000F02193F87C308DF81030404603238DF88C
:10B6800011308DF812608DF813900EF802101FF033
:10B6900071FCAB88B3FA83F3C3F11F0309FA03F318
:10B6A000002B3FF4DEAB12490A6813430B60FFF72F
:10B6B000D8BB302104E710F09CF8606940F2E93310
:10B6C00025E000BFF45300200C54002020A1070007
:10B6D0005854002000380040003C00405C11040831
:10B6E000581104086C12040800380240F58500085F
:10B6F000003C0140F8EB03085C5200204425002088
:10B70000083C014084250020013B9BB27BB10289AB
:10B710009707F9D58023838140F2E93302E0013BAA
:10B720009BB223B10289D507F9D5838901E010F0D6
:10B7300060F8A36913B11A689B881383012005F090
:10B7400009FA7F4D7F4FDFF820E2DFF82092029464
:10B75000322301934FF0100A4FF47A7C7A4B5B68E6
:10B76000C3F3080393B9EFF311837BB92868DEF8BC
:10B77000081000BF2B689842F8D13A680CFB02F31E
:10B780005B1AB3FBF2F30CFB00301DE0EFF3118208
:10B790008AF31288DEF80810DEF80030D80304D5EA
:10B7A0000123C9F80030DEF808102B68D9F8000032
:10B7B000D2B282F311883A6818440CFB02F35B1A88
:10B7C000B3FBF2F30CFB003001245F4B5B68C3F367
:10B7D0000803002B6BD1EFF31183002B67D12B688B
:10B7E000DEF8081000BF2A689342F8D1D7F800B0FD
:10B7F0000CFB0BF2521AB2FBFBF20CFB03231B1ADD
:10B80000B3F57A7FE1D3019B013B0193A6D1029C62
:10B8100001226B213046FDF77BF994F84F30042B61
:10B8200034BF18221A221B213046FDF771F994F813
:10B830004E30042B5CD0032B94BF0722019A1A21AF
:10B840003046FDF765F994F8502019213046FDF790
:10B850005FF910221C213046FDF75AF912223721D8
:10B860003046FDF755F9012238213046FDF750F9F1
:10B870006369364A934239D035498B4214BF082157
:10B8800000211A8822F040021204120C1A801A8831
:10B8900092B222F03802114319801A8892B242F013
:10B8A00040021A802B4A0121D175FFF7E2BAEFF36B
:10B8B00011818AF31288DEF808B0DEF80030DB036D
:10B8C00044BFC9F80040DEF808B02B68D9F8002062
:10B8D000C9B281F31188396813440CFB01F2A2EB61
:10B8E0000B02B2FBF1F20CFB032388E70021C8E74F
:10B8F00001221A213046FDF70BF9A4E76369164AC5
:10B90000934208D0A2F5744293427FF41BAB02230A
:10B91000124AFFF713BB0023104AFFF70FBB0123A6
:10B920009340BDE60E490B6B1A430A6340E60C498F
:10B930000B6C1A430A643BE60A4BE360FFF78FBACD
:10B94000145400201854002000ED00E0003800409E
:10B95000003C0040901E0020003001405854002060
:10B9600000380240F585000810E000E01054002087
:10B9700008B5034B1B6803B1984772B6FCF740FE4D
:10B98000B43900202DE9F04F7A4C54F8204083B0B0
:10B99000002C00F0EA80D4F86090B9F1000F00F0BC
:10B9A000E680D9F81050D9F80470734EA16004F104
:10B9B00066012660616104F266264FF40071A6619B
:10B9C000E1602161A765A0464DB3DFF8B4C14FF037
:10B9D000000E61464E68B54201F11C0106D00EF121
:10B9E000010EBEF1100FF5D14FF0000ECEEBCE0ED2
:10B9F0000CEB8E01DFF884C10E69DCF830E04FF00B
:10BA00000C0A4EEA060E461CCCF830E081F818A06D
:10BA10004E76D9F80810E16304376765656305461B
:10BA2000D9F80C001F46164600283CD0DFF850C15C
:10BA3000002163465A68904203F11C0303D0013190
:10BA40001029F7D10021C1EBC1010CEB81014B4B57
:10BA50000A69186BDFF82CE1104318630B20087695
:10BA6000681C4876186B024399F81F001A63830913
:10BA700091F80DC08DF80530002201234C61C1F80A
:10BA800008E001A88DF806208DF807308DF804C075
:10BA90001FF070FAA36DD9F80810D9F80C20A26332
:10BAA00004332164236594F865000FF0ABFA8246F5
:10BAB00094F864000FF0A6FA834699F81C00002859
:10BAC00050D1380739D4B2070ED5BAF1000F0BD0D8
:10BAD0000B226B1C8AF806208AF80730504699F82A
:10BAE0001D2022210FF0A8FBF30716D4E36B83B9C6
:10BAF00099F81E208DF8042099F820208DF8063042
:10BB000001A8930901228DF805308DF807201FF058
:10BB100031FA404603B0BDE8F08FBBF1000FE5D02D
:10BB200001350C238BF807508BF80630584699F8EE
:10BB30001D2022210FF080FBD8E70135EDB2BAF1CC
:10BB4000000F04D00B238AF807508AF8063017F04C
:10BB5000100F50460CBF1221022199F81D200FF042
:10BB60006BFBC3E722F062FFABE7A046D1E7C84614
:10BB7000CFE700BF2C5100207CEC030800380240C6
:10BB80004C0F00209D900008084B10B507281B683B
:10BB9000C8BF143818440C46007D0FF033FA20B1AA
:10BBA0002146BDE810400FF0D5BC10BD4C5100201F
:10BBB00038B50D4B07281B68CCBFA0F11404044610
:10BBC00023440546187D0FF01DFA58B12822013490
:10BBD000C471827101210FF0FBFB28460021BDE8F2
:10BBE0003840D1E738BD00BF4C5100200348D0F8A1
:10BBF000AC3113B100F5D270184770474C0F0020DC
:10BC00000348D0F8903113B100F5C470184770475D
:10BC10004C0F00200348D0F8743113B100F5B67012
:10BC2000184770474C0F00200348D0F8583113B123
:10BC300000F5A870184770474C0F00200348D0F853
:10BC40003C3113B100F59A70184770474C0F002033
:10BC50000348D0F8203113B100F58C7018477047B5
:10BC60004C0F00200348D0F804310BB1FC301847CA
:10BC7000704700BF4C0F00200348D0F8E8300BB1EC
:10BC8000E0301847704700BF4C0F00200348D0F841
:10BC9000CC300BB1C4301847704700BF4C0F0020A8
:10BCA0000348D0F8B0300BB1A8301847704700BF38
:10BCB0004C0F00200348D0F894300BB18C3018475B
:10BCC000704700BF4C0F00200248836F0BB17030EB
:10BCD000184770474C0F00200248C36D0BB1543019
:10BCE000184770474C0F00200248036C0BB13830E6
:10BCF000184770474C0F00200248436A0BB11C30B4
:10BD0000184770474C0F00200248836803B118475A
:10BD1000704700BF4C0F0020F8B5654C0601A7190D
:10BD20000546387A22F082FE3B7A03F01F015B0958
:10BD30000122032B02FA01F26DD0042B66D0022BF4
:10BD40005CD0A319013518790FF05CF9EDB2074604
:10BD500010B11223C5718371A31958790FF052F9EC
:10BD600010B11323C5718371A31998790FF04AF9A3
:10BD700010B11423C5718371A5190A21EA793846D7
:10BD80000FF05AFA68790FF03DF9EA790A210FF0BD
:10BD900053FAA8790FF036F9EA790A210FF04CFA34
:10BDA000A359444A934247D0434A934250D0434A0E
:10BDB000934259D0424A934262D0424A93426BD056
:10BDC000414A93422CD03444227BE2B90120022222
:10BDD000198801F4415141F445710A4302431A8024
:10BDE0009A8B22F400621204120C07219A831982A2
:10BDF0001A8892B242F040021A80F8BD334B596A59
:10BE00000A435A629DE700200246E1E72F4B196979
:10BE10000A431A6195E72D4B196A0A431A6290E7A3
:10BE200002F564424FF40010536A43F40013536266
:10BE30001FF0D8F8A359C6E702F584324FF48050BA
:10BE4000536A43F4805353621FF0CCF8A359BAE706
:10BE500002F500324FF48040136A43F480431362CA
:10BE60001FF0C8F8A359AEE702F5FE324FF40040C8
:10BE7000136A43F4004313621FF0BCF8A359A2E70E
:10BE800002F582324FF40050536A43F40053536278
:10BE90001FF0A8F8A35996E702F568424FF4801006
:10BEA000536A43F4801353621FF09CF8A3598AE746
:10BEB000585400200030014000380040003C004051
:10BEC000003401400050014000540140003802405D
:10BED000431C00F014812DE9F04F4FEAC00808EB35
:10BEE00000039B00DFF8F4A25AF803B087B00AEB16
:10BEF0000304BBF1000F00F0FF8014330AEB0301D1
:10BF00000022DBF804704AF803204A608A60CA60A5
:10BF10000346A56801900133D4F80C90DBB2002DE4
:10BF200000F0EE801522EB71AA71B9F1000F00F05C
:10BF30000081162289F8062089F807309BF80E0048
:10BF400022F074FDBB8823F440731B041B0CBB80E0
:10BF500028460FF0FAFA48460FF0F7FA1121284662
:10BF60000EF09AFF112148460EF096FF0826642431
:10BF700004E00A203CB104F0EDFD013C28460FF03E
:10BF80000BFB0028F5D028460FF0DAFA0A2004F05F
:10BF9000E1FD28460FF0D9FA0A2004F0DBFD013E4E
:10BFA000ECD148460FF0CCFA0A2004F0D3FD284625
:10BFB0000FF0C6FA0A2004F0CDFD28460FF0C5FAAE
:10BFC0000A2004F0C7FD48460FF0BFFA019B08EBBA
:10BFD00003040AEB84042846637C002B0CBF122167
:10BFE000322104220FF028F9637C002B0CBF1221B0
:10BFF0003221484604220FF01FF9704B9F4200F097
:10C00000B7806F4B9F4200F0BD806E4B9F4200F0A7
:10C01000A580BB8801996C4A6C4C23F440731B04C7
:10C020001B0CBB803B8888440AEB880A9BB243F018
:10C0300001039AF810103B80BD8802A8002918BFA0
:10C0400014461EF0DFFF049A6148B2FBF4F325F0BA
:10C050003F05A0FB02122D04900C2D0C0543BD8062
:10C060005C4C39884FF4967202FB00F284FB02406C
:10C070009BB2D217002BC2EBA01221F0010108BF26
:10C0800001230904013243F40043090C92B23980C0
:10C090003A84BB833B889BB243F001033B803B88DF
:10C0A00023F4816323F002031B041B0C43F480631D
:10C0B0004FF480423B803A813B8823F080031B048D
:10C0C0001B0C3B809BF810308DF8083000240123B6
:10C0D00002A88DF80B308DF809408DF80A401EF04B
:10C0E00049FF9BF80F308DF8083002A88DF8094001
:10C0F0008DF80A401EF064FF07B0BDE8F08F70476E
:10C10000B9F1000F48D0162289F8073089F80620C7
:10C110009BF80E0022F08AFCBB8823F440731B04BA
:10C120001B0C2846BB800FF010FA48460FF00DFAA2
:10C1300018E79BF80E0022F079FCBB8823F44073CB
:10C140001B041B0CBB8028460FF0FFF948460FF07C
:10C15000FCF9112128460EF09FFE07E71E4A136ADC
:10C1600043F4000313624FF400001EF043FF50E756
:10C17000194A136A43F4001313624FF400101EF0BF
:10C1800039FF46E7144A136A43F4800313624FF4FD
:10C1900080001EF02FFF3CE79BF80E0022F046FCCB
:10C1A000BB8823F440731B041B0C4846BB800FF074
:10C1B000CCF948460FF0C9F9D8E600BF005400405A
:10C1C00000580040005C0040009F2400804F120097
:10C1D00083DE1B43D34D6210003802405C510020C7
:10C1E000F0B5C60033189B00254DEA585468A28A62
:10C1F00083B092B20192019A2B4412F4706F1CBF6B
:10C2000001221A75019B13F4E06F07460CD1A38A33
:10C210003E4423F4706305EB86051B041B0C0022CF
:10C22000A3826A7503B0F0BD238BA38823F48063D7
:10C230001B041B0CA380019B9B05E8D42388980555
:10C24000E5D42388D9050ED52388DA05FCD42388C4
:10C250009BB243F40073238023889B05FCD43846AB
:10C26000FFF736FED3E723889BB243F400732380A5
:10C27000A38823F440731B041B0CA380C7E700BFF3
:10C280005C510020F0B5037A012B83B0054664D0E1
:10C29000022B68D1036913B11A689B885383E8683D
:10C2A00040F2E93302E0002B00F0AA800289013B52
:10C2B00012F0020F9BB2F6D0BB23838140F2E93328
:10C2C00002E0002B00F09C800289013B12F0010F7C
:10C2D0009BB2F6D0838983894FF0060E4FF47A73B0
:10C2E0006E464FF6FF71FF2703E0013B9BB28B4286
:10C2F0003CD002899407F8D587814FF47A7302E025
:10C30000A3B28B4232D00289D20703F1FF34F7D5B2
:10C31000828992B20EB132700136BEF1010EE8D1BF
:10C320002B6913B11A689B8813839DF804009DF84C
:10C3300000609DF801109DF802409DF803209DF8D3
:10C34000053041EA062143EA002342EA04220120A3
:10C35000E9822A836B8303B0F0BD90F90C00461C80
:10C3600001D0032805DD002003B0F0BD0FF041FA35
:10C37000D6E7C700294E3A1806EB82025168002919
:10C38000F1D06C7B6400E4B294754FF0000E06248B
:10C390004FF03B0C82F817C082F819E093761476C0
:10C3A000537582F814E08B88C2F820D09C05C2F83F
:10C3B0001CD014D40B88DA050CD44FF4805401E05F
:10C3C000013C21D00B889B05FAD40B889BB243F427
:10C3D00080730B808B889BB243F440738B8007443F
:10C3E00006EB87024FF4805401E0013C0CD0537DF2
:10C3F000002BFAD106EB87073B7D002B95D0B2E7E7
:10C400000FF0F7F9E86866E7054A138801339BB235
:10C410001380FFF75DFD2046A6E700BF5C510020BA
:10C42000DA3D0020F0B583B0441C8DF8073001D010
:10C43000032802DD002003B0F0BDC700244E3B18E6
:10C4400006EB83035D68002DF4D04900C9B29975ED
:10C4500001240021DA755C7699761C765C75197575
:10C46000A9880DF107028905DA611A6214D42B88B4
:10C47000DA050CD44FF4805401E0013C1ED02B8827
:10C480009B05FAD42B889BB243F480732B80AB8836
:10C490009BB243F44073AB80074406EB87024FF432
:10C4A000805401E0013C09D0537D002BFAD106EB0A
:10C4B00087073C7D84F0010003B0F0BD054A138876
:10C4C00001339BB21380FFF703FD2046B3E700BFA3
:10C4D0005C510020DA3D00200220FCF73FB900BF8C
:10C4E00002207DE60120FCF739B900BF012077E684
:10C4F0000020FCF733B900BF002071E61549164B48
:10C5000016480A6810B48C681549B2FBF4F203FBB4
:10C5100002F30360D1F88820124B134C42F47002EE
:10C52000C1F888201A68002042F001021A60986061
:10C530001A6822F0847222F480321A605C601A68F1
:10C540004FF0006422F480221A60D8608C605DF89D
:10C55000044B70470000002040420F00B45B0020F5
:10C5600000ED00E00038024010300024044B4FF48E
:10C57000F0700A21022283E80700FFF7BFBF00BF67
:10C58000000000202DE9F04F2DED028B95B00646FE
:10C590002AF04AFA9E4B1D7825B115B0BDEC028BEE
:10C5A000BDE8F08F9B4B1B685805F6D5DFF8B092BD
:10C5B000D9F80020002A00F02781974CD4F82831C0
:10C5C00003F5F43348339E42C0F01E81934F94F834
:10C5D0002C113B68C4F82861013184F82C119907AB
:10C5E00001F1798713F0140F41F0178713F0080F4A
:10C5F00094F82C3140F0C28113F0070801F0BA859D
:10C60000282B874B029302F0B1805E209047854B28
:10C610001B78002B6BD0804C834AD4F83431F31A4A
:10C62000934201F24384DFF83CA29AF80080B8F10B
:10C63000000F33D1DFF80092D9F800000EF03BFB79
:10C64000C0B201280ED90228784F42F04F813B78C2
:10C65000002B42F02A82D4F83C31F31AB3F57A6FFA
:10C6600082F0D58272480768002F40D09AF80030D7
:10C67000BBB9704BD9F800001B689B781E3B012B9F
:10C680004FF0020142F2688204302AF09FF8012242
:10C6900000238AF8002084F8483126E064480768BF
:10C6A0002FB3D4F8443140F6B732F31A93421ED96F
:10C6B00094F84031002B02F00F81013BDBB284F88B
:10C6C0004031002B01F0978717F8011B94F848219F
:10C6D000076094F8493158480A440133006884F8E7
:10C6E000482184F849310EF0E9FAC4F84461534A0C
:10C6F000029B12781B68012A03F101030C9301F0DD
:10C70000FF824F4B1B787BB1DFF85C91D9F800308A
:10C7100053B1414C029BD4F85C21D3F800B0ABEB91
:10C720000202632A01F21A82DFF8408198F800A021
:10C73000BAF1020F01F03A873C4F97F87430032B9F
:10C7400001F0DC843F4B1B7873B13F4D2B685BB12C
:10C75000314C04F0B3F9D4F86831039044F61F6209
:10C76000C31A934200F26081384B1B78002B7FD1B3
:10C77000374B1B7843B1284CD4F8B83203F500434B
:10C78000E8339E4281F03283324B1B78002B3FF41A
:10C7900004AF214E304C314D06F2C12720680EF017
:10C7A0008AFA00283FF4F9AE20680EF07EFA2B7862
:10C7B00080465A1E33B120682A700EF07CFA002899
:10C7C000F2D1EAE603223946781E32F08BF996F868
:10C7D000C03296F8C12286F8C38283F47F4383F087
:10C7E000FF039B1A1FFA88F89BB2B8EB132FD5D121
:10C7F00096F8C222DBB29A42D0D1781E2BF0A0FA72
:10C800002B7818442870C9E7054B0293FFE600BF58
:10C8100081920020B8630020B41E0020408E0020CA
:10C8200014540020528F00203F0D03001C000020F4
:10C83000B88E0020B48E0020B08E0020538F0020D0
:10C84000608F0020688F00206C8F0020908F002068
:10C85000918F0020728F0020788F00207C8F002025
:10C86000C08E0020BC8E0020288E0020FC9100206D
:10C87000604C2278002A41F03A82DFF8A49199F8BE
:10C880000040002C40F0AB805B4D2878002842F03F
:10C890008C805A4C5A4DD4F8B0222978594B93FBCE
:10C8A000F1F313449E42FFF463AF94F8B432564A56
:10C8B000C4F8B062D75CFB0702F17482B80702F1DA
:10C8C000E981790702F12A823A074CD54F4BDFF80C
:10C8D00054810D930DF15009A3F13D0249F8202D2B
:10C8E0000021A3F1400203F8401C022311215170E2
:10C8F00093704846D8F80010FCF734FF4846D8F843
:10C900000410FCF72FFFB8F80E30414903EBC303C6
:10C910009B00053381FB0321DB17C3EBA10189B227
:10C920004846FCF737FFB8F8103003EB8303590093
:10C9300089B24846FCF72EFF364B1B789B0743BF56
:10C94000B8F8081001F57A7189B24FF47A71484647
:10C95000FCF720FF0C9B98F81420591C0C914846BA
:10C960001A702AF021F894F8B4322978013393FB35
:10C97000F1F201FB123384F8B432F9E613F0030A42
:10C980007FF43AAE5E209047D9F8003014209847E3
:10C99000214B1F4AB3F9043082FB03124FEAE378BC
:10C9A000C8EBA2080FFA88F85FFA88F029F062FF56
:10C9B000C8F3072029F05EFFD9F800305E209847C1
:10C9C000D9F800301C209847504629F053FF5046B4
:10C9D00029F050FF94F82C31D9F800200CE60F4DC7
:10C9E0002F6E002F41F09D86044B89F80070C3F82C
:10C9F000B062BDE6448F0020B8890020B41E00203C
:10CA0000C0890020A0860100BC890020048F00207E
:10CA1000676666669E8E00204C8E0020C8890020C6
:10CA2000B9890020787E002094F86E31002B41F007
:10CA3000EA85DF4B1B6803F00802002A48F6034131
:10CA40004AF60B404BF60F4249F6074704BF024631
:10CA50000F4613F0040F4FF0190118BF17469B063D
:10CA600084F86E1103D547F4804747F0200720F083
:10CA7000F5FEC7F30909002842F0D282CD4B9B791D
:10CA8000002B42F09F82984664204FF0FF3A4FF00F
:10CA9000000C0C970D97ADF83CC0CDF842C0CDF816
:10CAA00046C0CDF84AC0CDF83890ADF83E80ADF81C
:10CAB00040A08DF84E000CAF0FCFDFF808E384F8EC
:10CAC00005C0AEE80F0097E80F00AEE807002EF8AB
:10CAD000023B71464FF0010C1B0CFE271F20C822A1
:10CAE00001F81E39A770A27184F807C0E07094F8AD
:10CAF0007E01207180F0F10383EA0313DAB2130997
:10CB000083F0E70343EA022383EAC2031BB283EA0A
:10CB10000312D2B2C3F3072383EA121343EA0223B8
:10CB200083EAC2031BB283F0C80282EA0212D2B2C5
:10CB3000C3F3072383EA121343EA022383EAC203FF
:10CB40001BB283EA0C0787EA0717FFB2C3F3072279
:10CB500082EA171242EA072200EB0C0382EAC707B7
:10CB60000EEB0C0084F87E31278011F8013B7B40EE
:10CB700083EA0313DBB21A0982EA172242EA03228C
:10CB800082EAC3031BB29FB281422780EDD183F0BA
:10CB90007C0383EA0313DBB24FEA131E8EEA172EDF
:10CBA0008EEA032E8EEAC30E0FFA8EFE1FFA8EF95E
:10CBB000DFF814C2A4F800905FFA8EFE4FEA19293C
:10CBC00084F8289084F827E00CF5D37804F1220A41
:10CBD000DCF80000DCF80410DCF80820DCF80C308D
:10CBE00047460FC70CF1100CD445B846F0D1DCF81D
:10CBF00000003860704F9CF8043088F8043007F16A
:10CC0000270884F8CDE184F8CE9117F8011F286831
:10CC10000EF054F8B845F8D194F86F21002A41F08D
:10CC20005E856649029B08781B680A2184F86F11AB
:10CC3000002801F09A86DFF894E10128BEF8001080
:10CC4000059142F2EE820228BEF8028002F00082D4
:10CC5000BEF804100491032802F0DD820428BEF817
:10CC600006A002F0D3820528BEF8087002F0C78241
:10CC70000628BEF80AC002F0BF820728BEF80C10D2
:10CC800001D0BEF80E2094F87EB10C938BF03003E7
:10CC900083EA0313DBB24FEA131E494884F804B059
:10CCA0008EF07A0E4EEA032E00888EEAC303DFF878
:10CCB00020E1C0EB00208EFB009E8644C0171BB213
:10CCC000C0EB6E200690C3F3072E83EA0310059B8A
:10CCD000C0B24FF0000963F30F098EEA10130593F9
:10CCE0004FF0000E049B68F31F4967F30F0E4FF0DF
:10CCF0000008002763F30F0861F30F07059BCDF8C9
:10CD000034906CF31F4E62F31F474FF0000C9DF8F8
:10CD10001820CDF83CE06AF31F48CDF83880109712
:10CD20008DF844C08DF8452043EA00230DF130080A
:10CD300083EAC007B8E80F003FB287F0C80989EA64
:10CD40000919DFF880E084F805C05FFA89F9C7F3B4
:10CD50000727AEE80F0087EA191747EA092398E882
:10CD6000030083EAC9031BB283F023074EF8040BC8
:10CD700087EA0717FFB2C3F3072282EA1712704649
:10CD800042EA072282EAC70720F814190BF1010BC7
:10CD90004FF0230CFE211622C82384F87EB1278091
:10CDA00084F807C00EF1020EA170E270A37111E0C9
:10CDB000408E0020308E00205B200020E492002076
:10CDC000D82E0020BC1E0020B61E0020EC790020CA
:10CDD0000308208010F8013B7B4083EA0313DBB299
:10CDE0001A0982EA172242EA032282EAC3031BB22B
:10CDF0009FB270452780EDD183F0F40383EA0313DB
:10CE0000DBB24FEA131E8EEA172E8EEA032E8EEA4D
:10CE1000C30E0FFA8EFE1FFA8EFCD64FA4F800C088
:10CE20004FEA1C295FFA8EFE84F81EE084F81F90FA
:10CE30007968BA683868FB6807F5D37CACE80F00FE
:10CE400038697969BA6904F2C518ACE8070004F2D8
:10CE5000A71784F8C59184F8C4E117F8011F286862
:10CE60000DF02CFFB845F8D194F87231002B41F049
:10CE70004684C14F3B681922980684F8722140F11C
:10CE80000E83BE4BDFF800831B78990741F186873C
:10CE900098F81430042B8CBF4FF003094FF00209AF
:10CEA00003F00CFEB8F81030B8F808200C9003EB33
:10CEB00083035B00ADF84A304FF47A70D8F8003045
:10CEC0008DF84C900E93B8F80E1098F814E0D8F83E
:10CED00004308DF84DE000FB02F24FF0000A4FF0F5
:10CEE000FF300DF13009CDF834A010920F93ADF85A
:10CEF00048101190CC46BCE80F00DFF890E2AEE895
:10CF00000F009CE80F00AEE807007246182122F8D7
:10CF10001C39E17194F87E1184F805A081F0780342
:10CF200083EA0313D8B2030983F0F60343EA00232C
:10CF300083EAC0031BB283EA0310C0B2C3F3072322
:10CF400083EA101343EA002383EAC0031BB283F091
:10CF5000C80080EA001C5FFA8CFCC3F3072080EA5B
:10CF60001C1040EA0C2080EACC0000B280F01803CC
:10CF700083EA0313DBB2C0F3072080EA131040EA10
:10CF8000032080EAC30301F1010CFE204FF01E0ACA
:10CF90004FF0C80BA0700EF1020E217184F87EC113
:10CFA000238084F803A084F806B0184612F8011B09
:10CFB000414081EA0111C9B20B0983EA102343EA17
:10CFC000012383EAC10109B288B272452080EDD104
:10CFD00081F0180181EA0111C9B20A0982EA10231D
:10CFE00083EA012383EAC1031BB29AB2614922801A
:10CFF000DBB2120A04910692059384F8272084F884
:10D0000026308E4601F5D37B04F1220ADEF80000BB
:10D01000DEF80410DEF80820DEF80C30DC46ACE860
:10D020000F000EF1100ED645E346EFD1DEF80000FA
:10D03000CCF800009DF81430DFF854A184F8CC310E
:10D040009DF8183084F8CD31D3461BF8011F2868AD
:10D050000DF034FE4A4B5B45F7D103F02FFDD8F8B5
:10D0600000103B68B8F808200591D8F80410069124
:10D0700013F0140F4FF47A7101FB02F141F0748543
:10D080000F4694F87EB10C908BF06A003D4BDFF8B0
:10D0900004E1B3F90420109780EA0010C0B203093C
:10D0A00083F0D50343EA002383EAC0031BB283EA7B
:10D0B0000310C0B2C3F3072383EA101343EA00232B
:10D0C00083EAC0031BB28EFB020E05980D90D217A7
:10D0D0004FF00008C2EBAE0206980E9083F0C80C29
:10D0E0000F91ADF84A20ADF84480ADF84680ADF818
:10D0F00048808CEA0C1CCE465FFA8CFCC3F30727F1
:10D10000BEE80F0087EA1C1747EA0C2787EACC071E
:10D11000DFF878C084F804B03FB2ACE80F0087F0C5
:10D1200021039EE8070083EA0313DBB2C7F3072756
:10D1300087EA13170BF1010E47EA03278CE8070073
:10D1400087EAC30384F87EE14FF0210B4FF0FE0E17
:10D150001C27C8220CF10C0C84F8058084F807B059
:10D1600084F802E0ACF11C01E7701846A27123803C
:10D1700012E000BFB61E0020408E00209E8E0020D0
:10D18000812000204C8E0020787E0020BC1E0020D4
:10D190005B2000206766666611F8012B424082EA38
:10D1A0000212D2B2130983EA102343EA022383EA6C
:10D1B000C20212B290B261452080EDD182F06802C5
:10D1C00082EA0212D2B24FEA121B8BEA102383EAE0
:10D1D000022B8BEAC20B0FFA8BFB1FFA8BF3DB4F90
:10D1E00023805FFA8BFB1B0A059384F8253084F8B3
:10D1F00024B007F5D37C04F1220838687968BA684E
:10D20000FB68E646AEE80F0010374745F446F4D118
:10D210003B88AEF800309DF81430CD4F84F8CAB189
:10D22000D04684F8CB3118F8011F28680DF046FD70
:10D230004745F8D194F87EC1C64A84F804C08CF002
:10D24000EB0383EA0313D9B20B0983F0C50343EA66
:10D25000012383EAC1031BB283EA0310C0B2C3F304
:10D26000072181EA101141EA002181EAC00109B2D7
:10D270000CCA81F0C80787EA0717FFB24FF0000E0B
:10D28000C1F307210D93CDF838E081EA17130C9212
:10D2900099E8070043EA072383EAC7030FFA83F8F4
:10D2A000AD4B84F805E088F0310783E8070087EA92
:10D2B0000717FFB2C8F3072383EA171343EA0723CC
:10D2C00083EAC703277A607AA27AE17A94F80CE0BD
:10D2D00094F811801BB25F4087EA0717FFB2C3F3CF
:10D2E000072383EA171343EA072383EAC7031BB222
:10D2F000584080EA0010C0B2C3F3072383EA10133A
:10D3000043EA002383EAC0031BB25A4082EA0210B8
:10D31000C0B2C3F3072282EA101242EA002282EA74
:10D32000C00212B2514081EA0111C9B2C2F307230F
:10D3300083EA111343EA012383EAC1031BB28EEA95
:10D34000030E8EEA0E1E5FFA8EFEC3F3072383EAF6
:10D350001E1343EA0E23677BA07BE17B227C83EADA
:10D36000CE031BB25F4087EA0717FFB2C3F3072360
:10D3700083EA171343EA072383EAC7031BB2584023
:10D3800080EA0010C0B2C3F3072383EA101343EA14
:10D39000002383EAC0031BB2594081EA0111C9B2DC
:10D3A000C3F3072383EA111343EA012383EAC1038A
:10D3B0001BB25A4082EA0212D2B2C3F3072383EAB5
:10D3C000121343EA022383EAC2031BB288EA03086A
:10D3D00088EA08185FFA88F8C3F3072383EA18136A
:10D3E00043EA082383EAC803A17CE27CDFF8748166
:10D3F0001BB2594081EA0111C9B2C3F3072383EA82
:10D40000111343EA012383EAC1031BB25A4082EAA3
:10D410000212D2B2C3F3072383EA121343EA0223B0
:10D4200083EAC2031BB283F0270787EA0712D2B24E
:10D43000C3F3072787EA121747EA022787EAC207DA
:10D440003FB20CF10103BAB25FFA87F94FF0310C29
:10D45000FE200C2184F87E31C8234FEA122E228050
:10D4600084F807C0A070E170A37184F81490049F41
:10D4700084F815E07968BA68FB683868B7F810C0B6
:10D48000A8E80F0028F803CB84F8BBE184F8BA9130
:10D490001AF8011F28680DF011FCD045F8D194F856
:10D4A0007671002F41F026812C4B94F87E81B3F9E0
:10D4B0000010B3F90220B3F904309FED296A6771B7
:10D4C00007EE103A029B1B680C9388F06A0383EA0C
:10D4D000031306EE901AD9B20B0983F0D50343EA81
:10D4E000012383EAC1031BB283EA03115242C9B28A
:10D4F00007EE902AC3F3072383EA111343EA0123BB
:10D50000F8EEE77AF8EEE66AB8EEC77A83EAC10386
:10D510001BB267EE867A66EE866A27EE067A0020F0
:10D5200083F0C80ECDED0E7ACDED0D6A8DED0F7A3C
:10D530001090119012908EEA0E1C0DF130095FFAD6
:10D540008CFCC3F3072EB9E80F000DE0B61E0020D7
:10D550007F2000202C8A0020BC1E00204C8E002042
:10D5600088C3E43A5C2000208EEA1C1E4EEA0C2E92
:10D570008EEACC0EDFF888C40FFA8EFEACE80F00FE
:10D580008EF01E0799E8070087EA071A5FFA8AFA01
:10D59000CEF3072787EA1A1747EA0A278CE807001D
:10D5A00087EACA071C214FF0050A4FF01E094FF009
:10D5B000FE0EC82208F10103E17084F876A184F818
:10D5C000079084F802E0ACF11001A2710CF10C0C90
:10D5D00084F80480278084F87E3111F8013B7B4079
:10D5E00083EA0313DBB21A0982EA172242EA032212
:10D5F00082EAC3031BB29FB261452780EDD183F05D
:10D60000270383EA0313DBB21A0982EA172282EAAC
:10D61000032282EAC3031BB21FFA83FCDFF8E48310
:10D62000A4F800C05FFA83FE4FEA1C2C84F825C0E2
:10D6300084F824E008F5D37904F1220AD8F8000030
:10D64000D8F80410D8F80820D8F80C304F460FC787
:10D6500008F11008D045B946F0D1E04FB8F80030D5
:10D66000A9F8003007F1240884F8CAE184F8CBC196
:10D6700017F8011F28680DF021FBB845F8D194F880
:10D6800077A1BAF1000F41F02F80D54B1B6805221E
:10D6900084F877219A0641F17281D24ADFEDD27A7D
:10D6A000D18907EE101AB8EEC77A13F0140F27EEDF
:10D6B000277A01F0F984CD4BDFEDCB6AD3ED007A08
:10D6C000F8EEE77A67EEA67A94F87EC1C84BC94AAD
:10D6D000B3F90410B2F90620C74FC8488DED0D7A92
:10D6E0008CF0220383EA03135FFA83FE4FEA1E13D2
:10D6F00083F0590343EA0E23B2F5FA6F83EACE03AF
:10D700001BB2A8BF4FF4FA6283EA0318B2F57A7F1E
:10D710005FFA88F8C3F3072EB8BF4FF47A72A2F508
:10D720007A728EEA181E642303FB02F34EEA082E77
:10D7300087FB03278EEAC80EDA17C2EBA71280FB1D
:10D7400001300FFA8EF7CB174FF0000BC3EBA0039D
:10D7500087F0C8080DF13009CDED0E7AADF8422002
:10D76000ADF84030CDF830B0CDF83CB0CE4688EAC8
:10D770000818BEE80F005FFA88F8C7F3072787EAA2
:10D78000181747EA082787EAC8089D4FDEF800E027
:10D7900084F804C00FC70FFA88F888F04A0383EAB8
:10D7A0000310C0B2C8F3072383EA10133A460CF102
:10D7B000010143EA002383EAC00342F810E9002094
:10D7C0004FF04A084FF0FE0C4FF0140E84F87E1113
:10D7D000C82160712380043784F8078084F802C070
:10D7E00084F803E0A171184612F8011B414081EA58
:10D7F0000111C9B20B0983EA102343EA012383EA2A
:10D80000C10109B288B2BA422080EDD181F0140181
:10D8100081EA0111C9B24FEA111E8EEA102E8EEA7A
:10D82000012E8EEAC10E774B0FFA8EFE1FFA8EFC88
:10D830001F464FEA1C2B5FFA8EFE84F81DB084F859
:10D840001CE0596838689A68DB68A4F800C007F5DE
:10D85000D37CACE80F0038697969B7F81880049771
:10D86000ACE8030004F2A717ACF8008084F8C3B159
:10D87000B84684F8C2E104F2C31B18F8011F2868F7
:10D880000DF01CFAC345F8D15F4B604A1B78127843
:10D89000013B12F00100DBB214BFC0214021172B65
:10D8A00003D85B4A134493F814A05A4B1A88930781
:10D8B0001ABF002341F01001012312F4027F18BFA8
:10D8C000022312F0100F18BF062312F0200F18BF0A
:10D8D0001023002841F091814FF0030894F87EC195
:10D8E0000C938CF0460383EA0313DAB2130983F036
:10D8F000920343EA022383EAC2031BB283EA0310C2
:10D90000C0B2C3F3072282EA101242EA002282EA7E
:10D91000C00212B282F0C80E8EEA0E1E00235FFA19
:10D920008EFE0320C2F307228DF834A08DF83780D5
:10D9300082EA1E128DF835308DF836108DF83800D9
:10D9400042EA0E2899E8070088EACE0E0FFA8EF810
:10D95000DFF8ACA0E37188EA0819AAE803005FFACF
:10D9600089F9C8F3072888EA191848EA092181EAE1
:10D97000C90994F808808AF800200FFA89F988EA22
:10D98000090282EA02185FFA88F8C9F3072282EADC
:10D99000181242EA0822607AA17A94F80B90637117
:10D9A00082EAC80212B2504080EA0010C0B2C2F34C
:10D9B000072282EA101242EA002282EAC00212B270
:10D9C000514081EA0111C9B2C2F3072282EA111261
:10D9D00042EA012282EAC1021EE000BF5B20002071
:10D9E000408E0020787E00200AD7233C448E002001
:10D9F0004C8E0020EC790020D34D6210676666667D
:10DA0000BC1E0020B61E002020310020484100200E
:10DA1000A4EC03089C8E002012B289EA020989EA6C
:10DA200009195FFA89F9C2F3072282EA191242EA58
:10DA3000092294F80C80607BA17B84F804C082EA00
:10DA4000C90212B288EA020888EA08185FFA88F860
:10DA5000C2F3072282EA181242EA082282EAC802C6
:10DA600012B2504080EA0010C0B2C2F3072282EA2C
:10DA7000101242EA002282EAC00212B2514081EA48
:10DA80000111C9B2C2F3072282EA111242EA01224D
:10DA900082EAC102E17B94F8109013B281EA03029A
:10DAA00082EA0212D2B2C3F3072383EA121343EAD3
:10DAB000022383EAC2031BB289EA030282EA02124A
:10DAC000D2B2C3F3072383EA121343EA022383EAA1
:10DAD000C2031BB283F0320282EA0212D2B2C3F353
:10DAE000072383EA121343EA022383EAC2031BB229
:10DAF0009AB24FF0FE085FFA83FE0920C8210CF1AC
:10DB0000010C84F802804FEA1228E070A17184F8B9
:10DB10007EC1228084F8128084F811E0049B18688A
:10DB200059689A68B3F80CB00AF5CC7CACE80700E9
:10DB30000AF5D47A8CF80290ACF800B084F8B88179
:10DB400084F8B7E117F8011F28680DF0B7F8BA4557
:10DB5000F8D1039BC4F86831FEF706BEDFF83C83BA
:10DB6000BF4FDFF83CA3412028F0B0FAB8F90220FB
:10DB700087FB0230D217C2EBA00080B228F08AFAED
:10DB8000B8F9002087FB0230D217C2EBA00080B2A8
:10DB900028F080FAB8F9042087FB0230D217C2EBD4
:10DBA000A00080B228F076FA9AF80010D9F80000A8
:10DBB0000DF084F894F8608118F0010700F02885D2
:10DBC000A84F3A68910640F18180A74ADFF8D482D5
:10DBD0001278920740F1C48798F81420042A8CBF69
:10DBE000032302230393472028F070FAD8F800009B
:10DBF00028F01CFAD8F8040028F018FAB8F80E201B
:10DC00009A49D9F80000A1FB0232C2F3471211462B
:10DC100004920DF053F89AF800003968049A11F054
:10DC2000140F82EA00028AF8002040F0BA86B8F8A1
:10DC30000820642000FB02F028F0F8F998F814702E
:10DC4000039BD9F8000043EA8707FFB239460DF07D
:10DC500035F89AF80020D9F80000574039468AF87C
:10DC600000700DF02BF894F86081B8F1000F2DD101
:10DC70007F4F4F2028F02AFA386828F0D7F97868C3
:10DC800028F0D4F9404628F0D1F90121D9F8000054
:10DC90000DF014F8744A9AF800701278D9F8000060
:10DCA00002F00108414687F001078AF800700DF084
:10DCB00005F89AF80020D9F8000088EA0202114617
:10DCC0008AF800200CF0FAFF94F86081694AC4F8E1
:10DCD0005CB108F10103DBB2A2FB0312D20802EB34
:10DCE0008202A3EB420384F86031FEF71DBD624B54
:10DCF000624918680CF0B0FF00232370FEF7BDBD29
:10DD00005F4F386800283EF4FCAC4FF0000ADFF8A3
:10DD100098815C4CAB4655460CF0CDFFF8B1F5B997
:10DD20004FF00109AA4638680CF0BFFF83B27E2B82
:10DD300000F0518498F80120002A49D194F84C1140
:10DD4000B1B11B2B84F84C2100F01E840D2B45D063
:10DD5000386888F801900CF0AEFF0028E3D1AA469D
:10DD600050460CAA48495D4628F0CAF9FEF7C9BCDE
:10DD70007D2B00F0F08594F8502122B180F0200333
:10DD8000DBB284F8501194F84B21062A10D8B4F86D
:10DD90004E1138681944A4F84E11A118013281F8C7
:10DDA000543184F84B210CF086FF0028BBD1D6E714
:10DDB000B4F84E2188F8019013449BB21A0A52FA23
:10DDC00083F3FF2BA4F84E31386802D12F4DA3E71F
:10DDD00038680CF070FF0028A5D1C0E73868A4F8B7
:10DDE0004E210CF068FF00289DD1B8E794F8BC32B2
:10DDF000C4F8B862012B40F2738594F8BD2224491F
:10DE0000981801EB8001013202F00102CF6A84F818
:10DE1000BD22BFB11F4D0D950DF15009123DA52337
:10DE200049F8205D802284F8103115233146484698
:10DE300084F8112184F81231B847002840F0D184C9
:10DE400094F8BC32144A013382FB0312A2EBE37252
:10DE500002EB42029B1A84F8BC32FEF795BC00BF6D
:10DE600067666666408E00209E8E00201F85EB51FF
:10DE70002C8A0020CDCCCCCCB4890020048F00208B
:10DE8000AC8E0020B41E0020FE1F002008200020C1
:10DE9000A4EC0308D91F0020565555554C8E002080
:10DEA0002C8E0020787E00201C0000209E4A9F4B74
:10DEB00092F80BE0029AD4F8381110681B889C4A3B
:10DEC000401A4FF47A71DFB201FB0EF11B0A97770B
:10DED000177588424FF00007D37753759770177105
:10DEE00080F0EA84934BDFF870C21B689249934F2D
:10DEF0000868DFF8689289683F688CFB038EDB173F
:10DF0000C3EB6E1303F5FA739BB293761B0AD376B9
:10DF100089FB00A389FB01A9C017C917C0EBA300A7
:10DF2000C1EBA90107F5EA43DFF834E2107730339B
:10DF3000001282F8201009121B12DFF828829EF8C6
:10DF400000E0507782F821108CFB0790F917C1EBA5
:10DF5000601182F823307A4B98F814A083F81AA045
:10DF6000783130371EF0020F82F8241082F82270C8
:10DF700000F09F84D8F800E0724AD8F80400DFF877
:10DF8000E8B182FB0E714FEAEE77C7EBA151039126
:10DF900082FB0092C117C1EBA25203990BFB01E176
:10DFA00001EB410149000F460BFB020B0497B946F8
:10DFB0000BEB4B0B644F4FEA4B01059187FB099B21
:10DFC00087FB01194FEAA949CDF81C90B8F80E90CB
:10DFD0000399B8F8088002EB820209EBC90902EB49
:10DFE0008202089201EB81074FEA890205990392A8
:10DFF00007EB8707049A0697CF17C10F099104987A
:10E0000052494FEAAB4BD2174FEADE7E83F809E064
:10E01000ABEB020E01FB1E020798069908F5FA7891
:10E02000BAF1050F1FFA88FAA0EB0708059F4748C9
:10E0300083F815A04FFA8EF909EB8109414600FBE0
:10E0400018789DF8240098730898414FDFF81CE178
:10E0500049B201EB80018CFB020B4FEAE2720492A1
:10E06000039ABEF800E08CFB08C087FB02C74FEAAA
:10E07000E27C049AC2EB6B120392364A1FFA89F9CA
:10E080001288ADF8102083F80A90039A83F813E001
:10E0900089B24FEAE8784FEA112BC8EB6010CCEB5D
:10E0A000A7174FEA1A284FEA192C4FEA222A9DF89F
:10E0B0000C2083F810B04FEA202983F80BC0D973E5
:10E0C000C7F3072C4FEA1E2134BF4FF0320B4FF03D
:10E0D000330B1A739DF8102083F80DA0587483F841
:10E0E000129083F81680DF7183F808C0197583F8E1
:10E0F0001BB01A77C4F83461FEF795BADFF8709058
:10E10000D9F800000CF0CBFD00283EF41BABD9F889
:10E11000000001210CF0C0FD0222002387F87420CA
:10E1200088F80030FEF70EBBE8900020E090002059
:10E130005C890020448E00206C8C0020488E0020DA
:10E14000888900206BCA5F6B83DE1B4340420F004F
:10E15000D34D62107C8A00201F85EB51676666668E
:10E160009E8E0020787E0020806967FFA88E0020A8
:10E17000202A00205E209047D9F8003002209847DE
:10E18000FF2029F063FD0378FF2B00F0998490F9BC
:10E1900001304FEAE3785FFA88F8D8B228F06AFBDA
:10E1A000404628F067FBD9F800305E209847D9F840
:10E1B000003003209847FF2029F048FD0378FF2B0B
:10E1C00000F07984B0F90830D8B2C3F3072828F0FA
:10E1D00051FB404628F04EFBDA4B1B78042B7DD0D8
:10E1E000DFF88CB3B4F82E119BF80020DFF884A37D
:10E1F00091FBF2F302FB13139BB2BAF80010A4F8E0
:10E200002E314FEA03181FFA88F8642303FB012319
:10E210005200B3FBF2F348EA0328C3F303225E2063
:10E22000D9F800301FFA88F848EA02089847D9F868
:10E230000030062098475FFA88F028F01BFB4FEA71
:10E24000182028F017FBC049B4F82E214B7ABAF8F1
:10E2500000A00132012BA4F82E2100F00C874A7B8C
:10E260000AEB8A031FFA83FA002A40F0C084D9F827
:10E2700000305E209847D9F800303A209847B34BD9
:10E28000A3FB0A384FEA58181FFA88FB5FFA8BF095
:10E2900028F0F0FA4FEA1B2028F0ECFAD9F8003009
:10E2A0005E209847D9F800303B209847642303FB51
:10E2B00018A39BB2A648053380FB0320DB17C3EBF2
:10E2C000A000C0B228F0D6FA002028F0D3FADFF878
:10E2D000A88298F80630002B40F051843B689F06D6
:10E2E00040F11282DFF894A29AF80030980700F10A
:10E2F000EA83DFF88C820027BB46D9F800305E2025
:10E300009847D9F8003001209847584628F0B2FACB
:10E31000384628F0AFFAD9F800305E209847D9F88F
:10E32000003009209847002028F0A4FA002028F0A7
:10E33000A1FAB8F8123098F814B0B3F5967F0AD95C
:10E3400094F82C2102F00F02072A04D842F20F7B26
:10E350009B4528BF9B46D9F800307B4F5E209847ED
:10E36000D9F80030052098473B7A002B00F06685ED
:10E37000ABF1200307EE903A9FED767AF8EEE77A5C
:10E38000F6EE006A67EE877ABEEE007AF5EEC07AA6
:10E39000F1EE10FA58BFB0EE667A77EE877AFDEEAE
:10E3A000E77ACDED027ABDF908B05FFA8BF028F07C
:10E3B00061FACBF3072028F05DFA9AF800200023D9
:10E3C00092070A930B9300F1658394F83031012B87
:10E3D00000F06083B7F90030DFED5F6A07EE103AB6
:10E3E000B7F9023007EE903AB8EEC77AF8EEE77A5E
:10E3F00027EE267A67EEA67ABDEEC77AFDEEE77ABB
:10E400000CA88DED0C7ACDED0D7A28F055FA94F824
:10E410002C31D9F80020FEF7F3B85E209047D9F8E8
:10E420000030302098474D4BD3F800805FFA88F0D9
:10E4300028F020FAC8F3072028F01CFA94F82C31B1
:10E4400013F003087EF4C8AA454AD4F82811454BB6
:10E450009142186840F28F8380EAE073A3EBE07387
:10E460003A4A1BB282FB03124FEAE37ACAEB621A02
:10E470004FF0640808FB1A380FFA88F80FFA8AFA86
:10E480005FFA88FB5FFA8AF2C8F30728CAF3072A03
:10E49000D9F8003002925E209847D9F80030102059
:10E4A0009847029A104628F0E5F9504628F0E2F91C
:10E4B000D9F800305E209847D9F8003021209847DD
:10E4C000584628F0D7F9404628F0D4F93B68D9F8E7
:10E4D0000020FEF78BB8DFF8AC809FED238A4FF069
:10E4E000240A5E2090475046D9F8003098471F4BC9
:10E4F000F8EC016A9B8A07EE103AF8EEE66AB8EE8D
:10E50000C77A0AF1010AC6EE877A5FFA8AFA67EEDD
:10E51000887AFDEEE77ACDED027ABDF908B05FFAB0
:10E520008BF028F0A7F9CBF3072028F0A3F9BAF174
:10E53000270F02D0D9F80020D3E73B68D9F8002094
:10E54000FEF750B8D83D0020E89000201F85EB5121
:10E5500067666666E4380E3F0050C347488E002069
:10E560003F4B4C00448E002000007A44548E002023
:10E57000F6900020E0900020308E00209E8E00203B
:10E58000787E0020848E002038680CF094FB0028F0
:10E590007FF4DEAB386884F84A9188F801900CF07B
:10E5A0008AFB00287FF4BFABFFF7D9BB02F086FAE5
:10E5B000D14B1B68A0EB030B40F6B8339B4500F230
:10E5C000BF81CE4B1A793A2A00F04284002388F8A2
:10E5D0000030FEF7B7B8386884F84AA184F84BA138
:10E5E00084F84C9188F801A00CF065FB00287FF4BA
:10E5F0009AABFFF7B4BB94F8481194F84931C0487E
:10E600004A1CFEF76AB8013B84F86E31FEF704BB82
:10E61000BC4A1288D30513D4D00600F1E6829106D5
:10E6200000F11D85530600F13C85100700F154856B
:10E63000D10700F1588512F0020F0CBF04270C27F8
:10E64000B149B24A0B78D27803F001030AB143F022
:10E6500002035320039327F039FDAD4A128802EBE1
:10E66000820202EB8202900080B227F013FD0020AC
:10E6700027F010FDA74AA8491288D9F80000C2EB7C
:10E68000C212520081FB023111444FEAE278C8EB1A
:10E6900061285FFA88F841460CF010FB9AF80020D8
:10E6A000039BD9F800001F4388EA020800218AF87A
:10E6B00000800CF003FB3946D9F800000CF0FEFA9C
:10E6C0009AF80020D9F800007A40D2B211468AF8B0
:10E6D00000200CF0F3FA94F86081FFF7C6BA013A13
:10E6E00084F86F21FEF7C0BB0AF1FF3A84F877A1E6
:10E6F000FFF72FBA013F84F87671FEF7C0BF013BE8
:10E7000084F87231FEF7CBBE1B077FF580AE834BDA
:10E7100093E803000CAB83E80300184628F0CCF81C
:10E7200075E60024DFF8108227464FF0500A02E019
:10E73000DBB283F3118815F804B0601C59462844F5
:10E7400027F07CFB002840F025810BF101031C44DD
:10E75000EFF311838AF312882A6E9442E8DB0022D9
:10E76000DBB22A6683F31188FEF73EB94FF0000A48
:10E770005E201F6884F82CA19047D9F80030DFF89C
:10E78000BC8117209847504628F074F8644BA3FBCF
:10E7900007239B0BA8FB03125209C2EB0212A3EB47
:10E7A0008203D8B228F066F8D9F800305E20984786
:10E7B000D9F80030182098475A4BA3FB07239B0930
:10E7C000A8FB03125209C2EB0212A3EB8203D8B2D8
:10E7D00028F050F8504628F04DF8D9F80020FDF701
:10E7E00014BF0C9EAE424FF000014FD941F2210000
:10E7F00015F8013B81EA03235A0013F4004F80EA25
:10E80000020192B289B208BF11464A0080EA0203AF
:10E8100011F4004F99B293B218BF0B46590013F48C
:10E82000004F80EA010289B292B208BF0A46530043
:10E8300012F4004F80EA03019BB289B208BF194667
:10E840004A0080EA020311F4004F99B293B218BF54
:10E850000B465A0013F4004F80EA020192B289B2CB
:10E8600008BF11464B0011F4004F80EA03029BB22F
:10E8700092B208BF1A46530080EA030112F4004F17
:10E880009BB289B208BF1946B542B1D14846FAF7E2
:10E89000A7FF25490C9D25486D1A152DA8BF1525E4
:10E8A0002A4630F014F9224A94F8BC321570FFF76A
:10E8B000C9BA2D22DA761DE41E4B02991B7809682D
:10E8C000C4F83811013B012B3FF60CAB1021022399
:10E8D00091701371FFF706BB27F0AEFFFDF705BF80
:10E8E0000E4A02EB8302D76AFFF793BA27F094FF30
:10E8F00001233B70FDF7B6BE04920020EC9100208E
:10E90000B08E00209C8E00204841002008930020FB
:10E91000E0900020D82E002003082080A4EC0308FB
:10E9200073B2E745D34D6210C41F00205C2700205E
:10E9300071270020D83D0020DD6903088988888878
:10E94000C44AB2F8623100210133A2F8623188F87A
:10E950000010FDF7F7BE386884F850910CF0ABF961
:10E9600000287FF4E0A9FFF7FAB90146844607467C
:10E9700082460490804605900246FEF784B99FEDDA
:10E98000B67A13F0140F08BFF0EE477A7EF493AE18
:10E99000FEF79ABE41463A2029F05CFA0743FFB2DF
:10E9A000D3E6AE4A1068FFF747B9AD49AD4B0093C7
:10E9B000A1F13F07AC4BAD4A0B9101F8404C0CA8BC
:10E9C000AB490A97FAF7E4FF0A9F7B1C0A933C7055
:10E9D0000A9B2922591C0A911A700A9BEA22591C87
:10E9E0000A911A700A9BC822591C0A910CA81A7025
:10E9F0002EF05AF800F101080CA942460A9830F0AE
:10EA000066F80A9A02EB080301330A9302F80840F9
:10EA10000A9B5A1C0A921C700A9B5A1C0A921C7070
:10EA20000A9B5A1C0A921C700A9B5A1C0A921C7060
:10EA30000A9B5A1C0A921C700A9B5A1C0A921C7050
:10EA40000A9B5A1C0A921C700A9B5A1C0A921C7040
:10EA50000A9B5A1C0A921C700A9B5A1C0A921C7030
:10EA60000A9B5A1C0A921C700A9B5A1C0A921C7020
:10EA70000A9B0122991814A80A911A7050F8283D8F
:10EA8000DB1B3B7027F090FF724B2C70C3F8B06219
:10EA9000FDF76EBE98E80C0001210AA884F8301139
:10EAA0000A920B9327F008FFB1E4C4F83C6187F8A1
:10EAB0000080FDF7D7BD4FF000084046FFF787BB49
:10EAC0004046FFF76BBBDFF8C081D9F80030694FD3
:10EAD0005E209847D9F8003011209847B8F80E20EA
:10EAE0004FF4F36B0BFB02F287FB0237D217C2EB3A
:10EAF0006737F8B227F0BEFEC7F3072027F0BAFE4B
:10EB0000D9F800305E2098471920D9F8003098478E
:10EB1000B8F80E30584A0BFB03F382FB0301DB17F6
:10EB2000C3EB611382FB0321DA17C2EB611264218C
:10EB300001FB1233D8B227F09DFE002027F09AFE89
:10EB40009AF80030B8F8087099077FF5D4AB5FFAEF
:10EB500087FB3F0AFFF7D1BB0CF09EF8FDF797BD8E
:10EB600001230393FFF73FB83C4B1F6807EB870770
:10EB70007F00FEF786BAC346C246424688E4D9F80B
:10EB80000030DFF808B1DFF808A15E209847D9F817
:10EB9000003028209847DBF800308AFB032ADB1777
:10EBA000C3EBAA0A5FFA8AF027F064FECAF30720D3
:10EBB00027F060FED9F800305E209847D9F8003081
:10EBC00004209847B8F80830002B40F04B82DBF85F
:10EBD000083083F310085FFA88F027F04BFEC8F383
:10EBE000072027F047FEFFF779BB342728E59BF87D
:10EBF00000309AFBF3FAFFF73ABB204AD278002A9A
:10EC00000CBF4FF004084FF00508FEF767BE012364
:10EC1000D9F800003B700CF048F80746D9F800001E
:10EC20000CF043F87F067DF41DAD8A2800F0438286
:10EC30008E287DF417AD9AF80030002B7DF42EADB0
:10EC40000F48104B03602D2384F840310768FDF70F
:10EC50000DBD00BFB41E002000000000448E002047
:10EC6000048F0020A2920020CC210408D4210408A3
:10EC7000E021040889B5F8141F85EB5108930020A2
:10EC8000B88E00205C890020787E00206C8C0020EB
:10EC900067666666CF4AD04B0D920DF15008A2F11F
:10ECA0003D0048F8200D1988DFF85493A2F1400385
:10ECB00000204FF00A0E02F8400C082283F801E011
:10ECC00040469A70FAF766FDD9F80030C349DA1762
:10ECD00081FB0313C2EBA30399B24046FAF75AFD36
:10ECE0001EF0CAFDD9F808900C9B4FEA1942591C36
:10ECF0000C911A700C9B4FEA1922591C0C911A7036
:10ED00000C9B5A1C0C9283F800900C9B5A1C0C9282
:10ED10001870404627F048FEFDF7D3BDAD4B0D936C
:10ED2000A3F1400900222121A3F13D0A03F8402C60
:10ED300089F8021089F80120CDF830A01DF0A8FF55
:10ED4000A74BA84A1B88A84900280ABF11464FF0C4
:10ED500003084FF004085A0500F19F81D80700F11D
:10ED6000BE8103F00203A14A002B1CBF4FF0030831
:10ED7000114642469E482FF0AAFE0AEB080314A84B
:10ED80009C4A013340F8203D9B1A00220AF80820D3
:10ED900089F8013027F008FEFDF796BD4FF0010914
:10EDA000FEF77EB8DFF86C929FED938AB9F90230D6
:10EDB000884A0D9207EE903AF8EEE77A0DF1500886
:10EDC00067EE887AA2F14003FDEEE77AA2F13D01F9
:10EDD00048F8201D02F8400C0822CDED027A5A7046
:10EDE0001E229A70BDF808104046FAF7D3FCB9F914
:10EDF000003007EE903AF8EEE77A404667EE887A00
:10EE0000FDEEE77ACDED027ABDF80810FAF7C2FC04
:10EE1000B9F9043007EE903AF8EEE77A404667EE2B
:10EE2000887AFDEEE77ACDED027ABDF80810FAF7A0
:10EE3000B1FC404627F0B8FDFDF740BD5FFA8BF00E
:10EE400027F018FD4FEA1B2027F014FDFFF7B5BA95
:10EE50009978039318462AF0F1FD00287FF4B6ABA9
:10EE60005D49664F664A09886648674CF961DFF874
:10EE7000A891116803689268F962B4F86211C7F842
:10EE80006CB0FB63FA64D9F80000F96500F0C2FACF
:10EE9000834600287DF451AC5146D9F800000BF0B0
:10EEA000FBFE039B94F86421DB780493642A4FF003
:10EEB000040387F8743040F0198194F86531072B0A
:10EEC00008BF84F865B194F86521504B079207EBB1
:10EED000021A0393DAF80410069108462DF0E4FDB7
:10EEE000DAF8083005935FFA80FA18462DF0DCFD59
:10EEF0005FFA80FB454B079A06990AEB0B00083036
:10EF0000D87122F00F00987202F00F020BEBCA00CA
:10EF10005A739873524603F10F002FF0D8FD059BEA
:10EF200019463B4B0AF1090018445A462FF0CFFD11
:10EF30003648C37903F1010ACBB1013B5FFA83FC88
:10EF40000CF1080CDFF8D4E084440023073010F8FB
:10EF5000012B5A409300D10883EA420301F01801C3
:10EF600053404EFA01F253408445DBB2EFD1284AB8
:10EF700004980AF802302EF0B1FC94F865310022B2
:10EF8000013384F8653184F86421039BDDF80CA01B
:10EF90009B785BB11AF80510D9F800000BF08EFED3
:10EFA00001359AF80230EDB2AB42F3D894F86431EF
:10EFB0000322013384F8643187F8742088F8002034
:10EFC000FFF79EB80E4B8046B3F900A06420FDF712
:10EFD0005EBD00BF048F0020E0900020676666667B
:10EFE0009C8E0020B0210408B8210408C821040820
:10EFF000C78E0020C58E002058A08B411C00002029
:10F000006C8C0020448E0020B41E0020907E0020D6
:10F01000967E00204C8E0020202A00200007090E3A
:10F02000854B864A1B88927903EB830303EB8303AA
:10F030004FEA83081FFA88F8002A40F0FA804FF060
:10F04000FF330FFA83FA1EF017FC40B2FDF71FBD25
:10F0500011469446174692460492FDF714BE2427A3
:10F06000FFF7EEBA1EF008FC27F004FC002027F0A2
:10F0700001FCFFF733B9D9F800305E209847D9F882
:10F080000030392098475FFA8AF027F0F3FB4FEA07
:10F090001A2027F0EFFBFFF71AB94FF00308684971
:10F0A00067E61027FFF7CCBA138907EE903AF8EE1F
:10F0B000677AFEF709BB634B1B6898067DF5D2AAF9
:10F0C0009AF80030002B7DF4E9AA5F485F4B03609B
:10F0D0002D2384F84031B9E52027FFF7B1BA5C4908
:10F0E0004FF0040845E60827FFF7AABA97F87530ED
:10F0F00058481A0704BF0133DBB2072B28BF01238E
:10F100004FEA031B07EB0B025FFA8BFA92F810E051
:10F11000514A039200EB0E010022087A4E498A728E
:10F1200001F10D0207EB0B014AEA0E0E012882F8ED
:10F1300000E0C96802F1010C0DD90238C0B200F13B
:10F14000020E9644624602F8011B72454FEA1121F5
:10F15000F9D101308444BB4421F0600201339BF8B3
:10F160001110DBB20A43082B8CF800200CF10102CD
:10F1700049D04FEA031B07EB0B00384990F810E029
:10F1800034487044511A007A01EB000C0AF1100A5D
:10F19000BCF1130F5FFA8AFAC4DDC9B28A1DD2B27C
:10F1A000039842F0400E80F807E002F1010ADFF810
:10F1B000B8E0CAB105315FFA81FB0BF1080B83445B
:10F1C0000EF1010C00221CF8010B5040820082EA73
:10F1D0004002C1084240224801F0180140FA01F102
:10F1E0004A40E345D2B2EED104980AF80E2087F8DF
:10F1F00075302EF073FBC8E61146FDF744BD11468D
:10F200009446FDF740BD1549511AC6E7114694468C
:10F210001746FDF738BD1146944617469246FDF74E
:10F2200032BD114694461746924604929046FDF729
:10F230002ABD0C4B1B6804E7E0900020308E0020B4
:10F24000BC210408408E0020B88E00208889002050
:10F25000C0210408A4EC0308907E00209D7E0020BD
:10F260000007090E6C8C0020967E002038B50B4CF0
:10F2700023688BB15A68821A002A054604DA0CE02A
:10F280005A68AA1A002A07DB9A68226018461A6888
:10F2900090472368002BF3D138BD38BD1C290020CE
:10F2A0000B4B002210B4027203F1F004032102E0C0
:10F2B000072A09DC9979890702D519798154013225
:10F2C0009C4203F11803F3D15DF8044B704700BF73
:10F2D0006411040837230370704700BF01233121F4
:10F2E000322241704271037203700371704700BF94
:10F2F0002322032302704370704700BF436A826970
:10F30000D154436A0169826B01338B4228BF0023C9
:10F310004362002A2FD0EFF31182502383F3128827
:10F32000836B1968C9072CD470B45E686EB9456ADE
:10F33000816A8D4217D084690C44DC600ED9691A49
:10F3400059608562002180F85C10196841F0010164
:10F35000D2B2196082F3118870BC70470469611AD7
:10F3600059608662EEE7012380F85C30D2B282F306
:10F37000118870BC7047826DD36843F08003D360FE
:10F380007047D2B282F31188704700BF426B10B44D
:10F3900062B1C36CC2684469D11A013B615C5DF81B
:10F3A000044B08BF1346C364C8B27047016A43697F
:10F3B000C4685B5C0131A14228BF114601625DF85F
:10F3C000044BD8B2704700BF836B13B190F85C0058
:10F3D0007047836A406A181AB0FA80F04009704793
:10F3E000416A836A99420AD3CB1A816B026961B17F
:10F3F0004968501E0B4483420AD2C01A7047026902
:10F400001144CB1A816B0029F2D1501EC01A7047EB
:10F4100000207047436B43B1C26C5B6893422FBFBF
:10F42000981AC0689B1AC0187047C269036A9A424A
:10F430002FBFD01AC0688018C01A70472DE9F04756
:10F440008C4B1B78DB07074644D58B4B8B4D1C78C8
:10F450008B4E012C59D01CD3022C07D189498A4AE2
:10F4600009881288914201D901241C70EB7AE3B11A
:10F470002B89D3B1854B1B78BBB11EF0FDF9002859
:10F4800000F09B802B7B83422CBF01210021317037
:10F490000CE07C497E4A098810886A7B801A884281
:10F4A000E2DAEB7A0024002BE2D131782A79632A60
:10F4B00006D8022C774E00F0BA803378002B5DD14D
:10F4C000754AAB7A8C4238BF0C461470002B4CD175
:10F4D000BDE8F0876B4B694D19885B88E878CB1ADB
:10F4E00083EAE3728142A2EBE3721DD32B788B4255
:10F4F0001AD3614B1C78E01E012861D9674909784D
:10F5000002294FD0012C5E4EA5D15F4A5D49128879
:10F51000687B0988121A914239DD5D4A12888A4255
:10F52000A4D200241C70A1E7B1EB400FE1DC524BE8
:10F530001C78E11E012940F29480022ADEDC574942
:10F540004F4E0878DFF84481DFF844C1DFF838E136
:10F5500000210324022834701C7088F80010ACF8D5
:10F560000010AEF8001081D11FE0012C71D0022CE8
:10F570000BD10720BDE8F0472CF008BA7068381AA4
:10F58000474B984258DD72709AE7BDE8F087022435
:10F590001C706BE7022AD2DD4049097802294FF03E
:10F5A000040464D13949364E09783E48022ACCBF5A
:10F5B00000220122C28081804BE70221317075E771
:10F5C000022A9BDC95F800C091FBFCFC0CF1010CBD
:10F5D000BCF1080FDFF8B4A0304EA87895F801E030
:10F5E00096F800802A4CDFF8A090254EA8BF4FF077
:10F5F000080C8AF800C01FFA8CFA10FB0AF01EFBF8
:10F600000AFE80B2DFF88CA02080A9F800E0002478
:10F610004FF0640EB8F1020F34701C70CAF8044049
:10F620008AF801E07FF439AF0FFA8CF1BDE730784A
:10F63000A0B9012377603370C2F164021A4B00FB5A
:10F6400002F083FB0023C017A0EBA350643070705E
:10F6500036E70820BDE8F0472CF098B97368F81A2F
:10F660008EE7032C96D10D49097802299AD0044ED1
:10F67000FCE600BF4841002078430020308E002087
:10F680007E430020E09000207C430020F690002084
:10F690007A4300209C230020D83D0020EC8F0020DE
:10F6A0007F969800F08F00206BCA5F6B038A2DE96C
:10F6B000F0478589ADB21D4029D00F4606464FF070
:10F6C00000484FF00009B5FA85F328FA03F2D24357
:10F6D00091B21B3B15403182042B16D8DFE803F0B2
:10F6E0003129211903007B6A002B32D003F1FF3A44
:10F6F0001FFA8AFAC7F824903C6A34B1236820467E
:10F70000514698476468002CF8D1002DDBD1BDE844
:10F71000F0873868716B036889B29847002DD2D1A1
:10F72000F5E77868B16B036889B29847002DCAD1B4
:10F73000EDE7B868F16B036889B29847002DC2D134
:10F74000E5E7F868316C036889B29847002DBAD1B3
:10F75000DDE7F36A1FFA83FACEE700BF30B504464F
:10F76000806D61718389A26823F400531B041B0C14
:10F77000838185B0A379009213F0040230D04FF456
:10F78000805213F00203ADF8042056D1ADF80630D4
:10F790004FF480630022ADF8083011F00103ADF89A
:10F7A0000C2028D1ADF80A3008238D07694648BFE0
:10F7B000ADF80A301BF06EFCA279A36DD10724D4FA
:10F7C00012F0080F9A8A1BD122F008021204120CC0
:10F7D0009A829A8992B242F400529A8105B030BD61
:10F7E00013F00203ADF8042024D04FF40055134663
:10F7F000ADF80650CEE70423ADF80A300C23D4E769
:10F8000092B242F008029A82E3E70D498B420FD090
:10F81000A1F548418B4209D00A498B42D0D105203D
:10F820000121FCF7B1F9A279A36DC9E70220F7E73E
:10F830000020F5E7ADF80630ACE74FF40053A5E73C
:10F84000001001400014014008B5012102200BF016
:10F8500089FE094B1B7803F00503052B08D0002116
:10F8600001200BF07FFE002108460BF07BFEFEE737
:10F870001CF090FDF3E700BF28510020022828BFAC
:10F88000022010B4084C094B207000EB8002C0EB42
:10F89000C20207495DF8044B013003EB4203C0B2DA
:10F8A0000B602CF09BB900BF9C9200201A2B00200B
:10F8B000A08E002010B50CF0F5FA094A094B0A4950
:10F8C0000A4C0B48146000221A705A70086010F03D
:10F8D000E9F9F9F76DFCBDE8104010F0CBB900BFB5
:10F8E000A08E00209C920020A48E00201A2B0020C5
:10F8F000A892002008B510F0D5F9F9F759FCBDE839
:10F90000084010F0B7B900BF2DE98048013085B03C
:10F91000C3B203938B4D8C4F8C4C8D4E0A230293B4
:10F920003220DFF830921FF041FA4FF4FA7A4FF0AC
:10F93000100C4FF47A70D9F80430C3F30803002B8D
:10F9400040F0C180EFF31183002B40F0BC802968A8
:10F95000A26800BF2B689942F9D1D7F800E000FBFC
:10F960000EF39B1AB3FBFEF300FB01314FF0010EC7
:10F970000191D9F80430C3F30803002B40F08780CD
:10F98000EFF31183002B40F082802B68A16800BF49
:10F990002A689342F9D1D7F800B000FB0BF2521A53
:10F9A000B2FBFBF200FB0323019A9B1AB3F57A7FAB
:10F9B000DFD3BAF1010ABED1039B002B40F0BD801A
:10F9C0004FF47A7ADFF88C9150464FF0100CD9F84A
:10F9D0000430C3F30803002B40F09280EFF311834F
:10F9E000002B40F08D802968A26800BF2B689942E7
:10F9F000F9D1D7F800E000FB0EF39B1AB3FBFEF33E
:10FA000000FB01314FF0010E0191D9F80430C3F32E
:10FA1000080303BBEFF31183EBB92B68A16800BFA8
:10FA20002A689342F9D1D7F800B000FB0BF2521AC2
:10FA3000B2FBFBF200FB0323019A9B1AB3F57A7F1A
:10FA4000E3D3BAF1010AC2D1029B013B02937FF4D6
:10FA500067AFFBF7E9F9EFF311888CF31288A1681F
:10FA60002368DB0344BFC6F800E0A1682B68326856
:10FA70005FFA88F888F31188D7F800801A4400FBF1
:10FA800008F35B1AB3FBF8F300FB0233D4E7EFF3A0
:10FA900011888CF31288A1682368DB0344BFC6F881
:10FAA00000E0A1682B6832685FFA88F888F3118853
:10FAB000D7F800801A4400FB08F35B1AB3FBF8F395
:10FAC00000FB023370E7EFF311828CF31288D4F855
:10FAD00008E02368D90303D501233360D4F808E094
:10FAE0002B683168D2B282F311883A68194400FB5E
:10FAF00002F3A3EB0E03B3FBF2F300FB013135E796
:10FB0000EFF311828CF31288D4F808E02368D9034C
:10FB100003D501233360D4F808E02B683168D2B2F2
:10FB200082F311883A68194400FB02F3A3EB0E0339
:10FB3000B3FBF2F300FB013164E718461EF098FFB7
:10FB40003EE700BF145400201854002010E000E0ED
:10FB50001054002000ED00E038B5484B5A899989CF
:10FB6000914224BF00225A81198ADA89914224BF26
:10FB70000022DA81DA78CAB1072A41496AD091F8BD
:10FB80005300404D012400210A282C709C70D9712B
:10FB90005DD00C2807D0002A6CD0DFED3B7A072A15
:10FBA0000ED00A2862D0DFED397A09E0344A92F8A3
:10FBB00053000A2856D00C285BD1D979DFED347A6E
:10FBC000344C9FED350AA278002918BFF0EE407A38
:10FBD000062A04D8314901EB820191ED000A21790E
:10FBE00079B1013A032A0BD8F7EE007A87EE800A42
:10FBF0002DF0CCFF2388984228BF1846208038BDBE
:10FC000038BD9B781F4A07EE103A1178B8EEC77AD4
:10FC100067EE277A07EE101AB8EEC77A27EE277A32
:10FC2000B4EEC70AF1EE10FAEADD80EE277AFDEEB7
:10FC3000C77A17EE903A102BA8BF1023012BB8BF3C
:10FC40000123DBB28B4238BF0B46137038BDDFEDAA
:10FC5000147AA4E791F853000A2803D00C28ACD0FA
:10FC6000D9799AE7D979DFED0E7AA9E7DFED0D7A38
:10FC7000A6E7D979DFED047AA2E700BFB85B0020E0
:10FC8000CC5B0020E03000206F1203396F12833A02
:10FC90000AD7A339CC7A00206F120338E0EC0308AE
:10FCA0005304E9380F506E3A2DE9F047B04FB14E8A
:10FCB0000FF0F8FFBE421ED2DFF83C83DFF83C9322
:10FCC0004446258862197DB14A450DD2052D0BD9D0
:10FCD00033886188C3F30B03994200F0EB8014462C
:10FCE00025886219002DEFD17168304614360CF06A
:10FCF000B4F8BE42E4D3A04A1378A3F11701022955
:10FD00000FD99E4911F83300002840F00281D80035
:10FD10000144497829B19A4911F833300BB91823B5
:10FD20001370984B5A78022A00F2E480964997485B
:10FD300002EB420201EB82011A780160022A00F212
:10FD4000E28002EB8201924BC2EBC10203EB420361
:10FD5000998C5A8C8F4C9142236001D300225A8493
:10FD60008D4B9A78042A00F0F58032B91A88B2F5E2
:10FD7000F07F84BF4FF4F0721A80884DFFF7ECFEDD
:10FD80002B68874A1A40002A00F0ED80D80700F15E
:10FD9000DC80590400F1D4801A0700F1C3809B0471
:10FDA00000F1C78020F02EFB10B97E482BF01AFB23
:10FDB00040200CF099F84FF400700CF095F84FF4D7
:10FDC00080300CF091F84FF480200CF08DF84FF457
:10FDD00000100CF089F84FF000700CF085F84FF02F
:10FDE00080600CF081F81CF0C5FF002130226E48C5
:10FDF0002EF092FE206817F00DF86C4B256803F189
:10FE0000500103E00433994200F081801A78002AFF
:10FE1000F8D19C78D8788442F4D26549654B0A7051
:10FE200028461D6028F0B8FD634A64491079644A89
:10FE3000644B1160C822642111FB0021002259602B
:10FE40009A60DA601A615A619A61DA6183F8202057
:10FE500083F8212018F07EFD5B4B9FED5C5A1B88D8
:10FE60005B4A9FED5C6A55795B4C5C495C48086075
:10FE700006EE903AF8EEE66A1388C5EE265A07EECB
:10FE8000103A53881279C4ED005A07EE903AB8EE52
:10FE9000C77A544BF8EEE77A1D725A7227EE067A4B
:10FEA00067EE867ABDE8F04783ED017AC3ED007A0C
:10FEB0000FF0E0BE63799B077FF411AF716894F88F
:10FEC00004A030460BF0C9FF3388BAEB133F04D0CF
:10FED0001436BE42FFF4F4AE0DE773887068AA1FB3
:10FEE000C3F30B039A4204F10601A8BF1A462EF091
:10FEF000EEFDEDE700225A701A782448224901608D
:10FF0000022A7FF61EAF00221A70214B20E7012241
:10FF100083E7D8000C186468002C7FF4F9AE17242E
:10FF20001470F5E630480BF0DFFF2B689B047FF57B
:10FF300039AF2E480BF0D8FF40200BF0D5FF31E74A
:10FF40002B480BF0D1FF2B6826E72A480BF0CCFF9B
:10FF50002B681EE79A8AB2F57A7FBFF40EAF4FF492
:10FF60007A729A8209E743F008032B600EE700BF1C
:10FF700018060008900100082031002074120408BF
:10FF800048F603089C920020A8920020A48E00202E
:10FF90001A2B0020A08E0020CC7A002010310020E7
:10FFA00009600002BC5A0020E024002080290020C3
:10FFB000100F00201425002094420020F230002071
:10FFC0001C25002008930020D0230020C0C9FB4836
:10FFD000D421002017B7D138D4230020D4410020E9
:10FFE0003661023DB041002001600002094000027C
:10FFF000092000020860000202400008008000089A
:020000040801F1
:1000000008B50FF04FFEF9F7D3F80FF033FEFFF706
:100010004BFE0120BDE808402BF0E0BDF0B50C29F7
:1000200034D8DFE801F0893333335E33333334338C
:1000300033330700048C9689B2F802E01788734DB9
:1000400024F480542404240C0484038C8488818B3D
:1000500023F4005321F4E6411B0409041B0C46EA77
:100060000E06090C43EA063341EA0721A8429BB277
:10007000A4B289B200F09E8005F58065A84200F028
:10008000998092688480818302640384F0BD048C2B
:100090009589B2F802C0B2F800E05C4F24F4807495
:1000A0002404240C0484038C8688818B23F400733D
:1000B0001B0421F073011B0C45EA0C04090443EAFC
:1000C0000423090CB8429BB2B6B241EA0E015CD0DF
:1000D0004F4CA04259D0926886808183C2630384CA
:1000E000F0BD048C9589B2F802C0B2F800E0474E2A
:1000F00024F010042404240C0484038C8788018BCE
:1001000023F0200321F4E6411B0409041B0C45EAFB
:100110000C04090C43EA041341EA0E21B0429BB2DD
:10012000BFB289B25DD03A4CA0425AD09268878063
:10013000018382630384F0BD048C9789B2F802E0E6
:100140001688324D24F001042404240C0484038C0A
:100150008488018B23F002031B0421F073011B0C24
:1001600047EA0E0709043B43090CA8429BB2A4B21C
:1001700041EA060125D005F58065A84221D09268A4
:100180008480018342630384F0BDD589148A578A31
:1001900023F4006343EA05254FF6FF332B4095888F
:1001A00026F440563C4343EA052346EA04169BB234
:1001B000B6B290E7158A24F4804444EA8514A4B2C8
:1001C0005FE7D689158A578A23F00803334324F45E
:1001D000407496883D4323F004032C433343A4B278
:1001E000CDE7D489158A568A23F0800343EA0413A5
:1001F0004FF6BF741C40938827F44067354344EAA8
:10020000031347EA85079BB2BFB28FE700000140A6
:10021000000401402DE9F04FF022002183B08A480C
:100220008A4CDFF84C928A4D8A4E8B4FDFF844821D
:100230002EF072FC89488A49DFF83CE2DFF83CC2C4
:1002400000221359834200F0D580B3F1804F00F0B3
:10025000E580AB4200F0E480B34200F0E380BB42B3
:1002600000F0E280734500F0E180634500F0E0803B
:10027000434500F0DF80DFF808A2534500F0DC8042
:100280000AF5806A534500F0D9800AF5806A534523
:1002900000F0D680AAF5983A534500F0D3800AF5CD
:1002A000806A534500F085800AF5806A534508BF8F
:1002B0000D237FD01832B2F5847FC2D1634C694ED2
:1002C000694F6A4D04F5847802E01834A0456DD07A
:1002D000A379002BF9D023794FEA131909F1FF39DB
:1002E000B9F1020F03F00F03EFD836F8190040FA06
:1002F00003F2D207E9D54FF0010A0AFA03F3013BF2
:1003000018402DF0CBF817F80930184415EBC0024F
:10031000DBD055F83000DFF86CE1217A00F13F4383
:1003200003F57E039B0A1EF8033003F01F0E5B09E2
:10033000032B0AFA0EFA68D0042B5DD0022B07D1EA
:10034000DFF81CE1DEF844304AEA0303CEF844301B
:1003500093880093B3FA83F3C3F11F039BB2DA08C7
:1003600000EB820203F00703D2F820E09B004FF07D
:100370000F0C0CFA03FC2EEA0C0EC2F820E0D2F8A7
:1003800020E001FA03F343EA0E03136269460023F7
:10039000022218348DF804208DF805308DF80630CF
:1003A0008DF807301BF05EF8A04591D103B0BDE891
:1003B000F08F0C2309EBC3034FF0010A1B7903F004
:1003C0001F0B5B09032B0AFA0BFA09D0042B0CD084
:1003D000022B7FF46FAF4B6C4AEA03034B6469E76F
:1003E0000B6C4AEA03030B6464E70B6B4AEA0303F2
:1003F0000B635FE70023DDE7DFF864E0DEF8303011
:100400004AEA0303CEF83030A2E7DFF854E0DEF822
:1004100040304AEA0303CEF8403099E70123C9E7A8
:100420000223C7E70323C5E70423C3E70523C1E786
:100430000623BFE70723BDE70823BBE70923B9E786
:100440000A23B7E70B23B5E77831002064110408CD
:100450000004004000080040000C00400000014083
:10046000003802405C110408581104085C52002056
:1004700094180408000401400010004000140040DB
:10048000004001406C12040801490248FFF70EB910
:10049000403200200018004001490248FFF706B929
:1004A000183200200040014001490248FFF7FEB821
:1004B000F03100200004014001490248FFF7F6B87E
:1004C000F03100200004014001490248FFF7EEB876
:1004D000C8310020000C004001490248FFF7E6B88F
:1004E000A03100200004004002494FF08040FFF797
:1004F000DDB800BF78310020F0B504684B4DA30A89
:10050000AB4276D009D94A4DAB425CD00F35AB42F5
:1005100073D04A3DAB425AD0F0BDB3F5801F64D0D2
:10052000023DAB4257D14FF0480E01264779B0004B
:100530004FEA970C002964D063460227A5899F40A3
:1005400083190CEB43032F4303F1040C394DBFB265
:1005500045F8231045F82C20A781EFF31181502294
:1005600082F31288821905EBC2021369002B33D083
:1005700013620433821905EBC202576917B11F6079
:1005800053690433821905EBC202976917B11F60E2
:1005900093690433821905EBC202D76917B11F6052
:1005A000D36904330027CAB21F6082F31188304434
:1005B00005EBC000036A93B9A38923F001031B0470
:1005C0001B0CA381F0BD4FF0980E0326AEE74FF051
:1005D000E80E0526AAE7F0BD05EB0E03CAE7A389DE
:1005E0009BB243F00103A381F0BD4FF0200E002623
:1005F0009CE74FF0700E022698E74FF0C00E0426DD
:1006000094E70223BF0803FA07F7A389094D9BB2B9
:1006100023EA070387190CEB470CA3810CF10403B1
:1006200045F82C1045F8232097E700BF0300100081
:10063000410010007831002010B50368824801396C
:10064000834282B089B200F0CA80A0F58060834204
:1006500000F0C58000F58040834200F0B78000F5CF
:100660008060834200F0B28000F58060834200F039
:10067000AD80764C188824686408B4FBF2F4013C21
:10068000A4B282B2B3F1804F0AD07148834207D03E
:1006900000F58060834203D000F58060834202D180
:1006A00022F0700292B26B48834200F0A18000F504
:1006B0008060834200F0A68022F4407200F56C4016
:1006C00092B283421A80D9621C854FD05E4A93420F
:1006D0004CD001229A821A8892B242F001021A800A
:1006E000B3F1804F00F09880594A934200F0968011
:1006F00002F58062934200F0938002F5806293429B
:1007000000F0908002F58062934200F08D8002F547
:100710008062934200F08A8002F57042934200F0BA
:10072000878002F57052934200F0848002F5806267
:10073000934200F0818002F5806293427ED0A2F560
:10074000983293427CD002F5806293427AD002F5CF
:100750008062934208BF0D2215D002A84FF00123FA
:1007600040F8043D1AF006FC02B010BD0122002141
:1007700019869A821A88384892B242F0010283425E
:100780001A80ADD10A46354B03EBC20301A85C7950
:100790008DF80440012300228DF805308DF80730D4
:1007A0008DF806201AF0E6FB1B2C08D02E2CDBD18E
:1007B0002B4B019301A81AF0DDFB02B010BD294BB1
:1007C000019301A81AF0D6FB02B010BD1F4C188887
:1007D0002468B4FBF2F4013CA4B282B252E71B4C91
:1007E00018882468B4FBF2F4013CA4B282B257E743
:1007F00001201A80D9621C8598821A8892B202431D
:100800001A8071E701201A80D9621C8598821A88A3
:1008100092B202431A8063E70122B4E70222B2E7F0
:100820000322B0E70422AEE70522ACE70622AAE7DE
:100830000722A8E70822A6E70922A4E70A22A2E7DE
:100840000B22A0E70C229EE700040140B45B0020CD
:10085000000400400010004000000140941804080B
:100860002C010001190100012DE9F04F013085B084
:10087000C3B203930B4602918B4C8C4E002B00F0BD
:100880009A8032208A4D8B4FDFF82C921EF08EFA20
:100890004FF4FA7A4FF0100C4FF47A70D9F8043014
:1008A000C3F30803002B40F0DE80EFF31183002B2D
:1008B00040F0D9802968A26800BF2B689942F9D11D
:1008C000D7F800E000FB0EF39B1AB3FBFEF300FB2E
:1008D00001314FF0010E0191D9F80430C3F3080340
:1008E000002B40F08780EFF31183002B40F08280D3
:1008F0002B68A16800BF2A689342F9D1D7F800B0ED
:1009000000FB0BF2521AB2FBFBF200FB0323019A2D
:100910009B1AB3F57A7FDFD3BAF1010ABED1039BEC
:10092000002B40F0BD804FF47A7ADFF88C9150466E
:100930004FF0100CD9F80430C3F30803002B75D125
:10094000EFF31183002B71D12968A26800BF2B68D7
:100950009942F9D1D7F800E000FB0EF39B1AB3FBE4
:10096000FEF300FB01314FF0010E0191D9F8043084
:10097000C3F3080313BBEFF31183FBB92B68A16822
:1009800000BF2A689342F9D1D7F800B000FB0BF200
:10099000521AB2FBFBF200FB0323019A9B1AB3F538
:1009A0007A7FE3D3BAF1010AC4D1029B013B0293DF
:1009B000002B7FF466AF05B0BDE8F08FEFF3118830
:1009C0008CF31288A1682368DB0344BFC6F800E0FB
:1009D000A1682B6832685FFA88F888F31188D7F825
:1009E00000801A4400FB08F35B1AB3FBF8F300FB2A
:1009F0000233D2E7EFF311888CF31288A1682368E1
:100A0000DB0344BFC6F800E0A1682B6832685FFAD8
:100A100088F888F31188D7F800801A4400FB08F39F
:100A20005B1AB3FBF8F300FB023370E7EFF31182BC
:100A30008CF31288D4F808E02368D90303D5012386
:100A40003360D4F808E02B683168D2B282F31188A1
:100A50003A68194400FB02F3A3EB0E03B3FBF2F375
:100A600000FB01317FE7EFF311828CF31288D4F899
:100A700008E02368D90303D501233360D4F808E0E4
:100A80002B683168D2B282F311883A68194400FBAE
:100A900002F3A3EB0E03B3FBF2F300FB013118E703
:100AA00018461DF0E5FF3EE710E000E0105400207E
:100AB000145400201854002000ED00E0204B5B6827
:100AC000C3F3080330B4BBB9EFF31183A3B91D4BD3
:100AD0001D4C1868A16800BF1A689042F9D11B4BE1
:100AE0001C684FF47A7202FB04F3591AB1FBF4F15B
:100AF00030BC02FB00107047EFF31182102383F328
:100B0000128811498C680B6813F4803F104B02D097
:100B1000012018608C680B49D2B20D68186882F306
:100B200011880A4B19684FF47A72284402FB01F3CA
:100B30001B1B30BCB3FBF1F302FB0030704700BF5E
:100B400000ED00E01454002010E000E018540020F4
:100B5000105400202DE9F84F8046FFF7AFFF254ED7
:100B60002549DFF8A0E0254A254D844610274FF49B
:100B70007A740120DEF80430C3F30803D3B9EFF32D
:100B80001183BBB90B68D2F808A000BFD1F8009060
:100B90004B45F7D1D6F800B004FB0BF9A9EB0A09D5
:100BA000B9FBFBF904FB0393A3EB0C034345E1D32F
:100BB000BDE8F88FEFF3118A87F31288D2F808B0F6
:100BC0001368DB0344BF2860D2F808B00B68D5F87F
:100BD00000905FFA8AFA8AF31188D6F800A0994447
:100BE00004FB0AF3A3EB0B03B3FBFAF304FB093397
:100BF000DAE700BF185400201454002010E000E091
:100C00001054002000ED00E02DE9F04FDFF830C176
:100C1000474A4849484E494D8046102718F1FF3849
:100C2000C0F08480DCF80430C3F30803002B5CD1EF
:100C3000EFF31183002B58D10B68946800BF08684C
:100C40008342F9D1D6F800904FF47A7000FB09FE88
:100C5000AEEB040EBEFBF9FE00FB03EEDCF8043045
:100C6000C3F308034FF47A740120FBB9EFF3118347
:100C7000E3B90B68D2F808A000BFD1F800904B454B
:100C8000F7D1D6F800B004FB0BF9A9EB0A09B9FBC0
:100C9000FBF904FB0393A3EB0E03B3F57A7FBDD2FC
:100CA000DCF80430C3F30803002BDFD0EFF3118A24
:100CB00087F31288D2F808B01368DB0344BF2860BA
:100CC000D2F808B00B68D5F800905FFA8AFA8AF378
:100CD0001188D6F800A0994404FB0AF3A3EB0B0398
:100CE000B3FBFAF304FB0933D5E7EFF3118487F381
:100CF0001288D2F808901368D80303D501232B601B
:100D0000D2F808900B682868E4B284F31188D6F80A
:100D100000A04FF47A7400EB030E04FB0AF3A3EB7C
:100D20000903B3FBFAF304FB0E3E97E7BDE8F08F2F
:100D300010E000E01454002018540020105400204B
:100D400000ED00E030B4EFF31183102282F312883B
:100D50000649074C0A680748013200250A602560E9
:100D6000DBB2026883F3118830BC70471454002052
:100D70001054002010E000E00F4B1B88014643B9DF
:100D80000E4B0F4A1B7810680BB981F001010AF075
:100D9000E1BB0C4B5A691AB118B91A681060587443
:100DA0007047094A18681188084A92FBF1F201213C
:100DB00002605974704700BFEC530020EE530020CE
:100DC000F0530020F45300200C54002020A1070011
:100DD00038B5264B5C69636B73B1A36DA26BD2B15E
:100DE000998A1A88C90592B201D5D20700D438BDB4
:100DF0004FF6F7721A8038BDA36D99891A88890653
:100E000092B2EBD59206E9D5E26AD2B19888216B0D
:100E100080B29047E1E799891A880D0692B2DFD532
:100E20001006DDD5A26A616A8A4219D0A1692569D6
:100E3000885C98800132B2FBF5F105FB1122A262B9
:100E4000CEE79B88E2696169DBB28B54E269E068B6
:100E5000A36D0132B2FBF0F100FB1122E261BDE7AC
:100E6000DA6822F08002DA60BAE700BF2C51002075
:100E700038B5264B9C68636B73B1A36DA26BD2B17E
:100E8000998A1A88C90592B201D5D20700D438BD13
:100E90004FF6F7721A8038BDA36D99891A888906B2
:100EA00092B2EBD59206E9D5E26AD2B19888216B6D
:100EB00080B29047E1E799891A880D0692B2DFD592
:100EC0001006DDD5A26A616A8A4219D0A169256936
:100ED000885C98800132B2FBF5F105FB1122A26219
:100EE000CEE79B88E2696169DBB28B54E269E06816
:100EF000A36D0132B2FBF0F100FB1122E261BDE70C
:100F0000DA6822F08002DA60BAE700BF2C510020D4
:100F100038B5264B1C68636B73B1A36DA26BD2B15D
:100F2000998A1A88C90592B201D5D20700D438BD72
:100F30004FF6F7721A8038BDA36D99891A88890611
:100F400092B2EBD59206E9D5E26AD2B19888216BCC
:100F500080B29047E1E799891A880D0692B2DFD5F1
:100F60001006DDD5A26A616A8A4219D0A169256995
:100F7000885C98800132B2FBF5F105FB1122A26278
:100F8000CEE79B88E2696169DBB28B54E269E06875
:100F9000A36D0132B2FBF0F100FB1122E261BDE76B
:100FA000DA6822F08002DA60BAE700BF2C51002034
:100FB00070B4EFF31186502383F31288836B1A68A1
:100FC000D20720D45D686DB9446A826A944217D012
:100FD00081691144D9600ED9A21A5A608462002234
:100FE00080F85C201A6842F00102F1B21A6081F3C5
:100FF000118870BC704701698A1A5A608562EEE7F1
:10100000012380F85C30F3B283F3118870BC704721
:101010002DE9F04FBC4B1E788BB0002E40F0818044
:10102000BA4BBB4C1D78BB4FDFF80CB305F0010584
:10103000A4F10A0954F80A0CB8B14FF0CC0808FB27
:10104000069809F038FE80B154F80A0C09F02DFE1C
:1010500014F8023C024683B924283BD075B354F8F7
:101060000A0C09F028FE0028EED10136032E04F107
:10107000CC04DFD10BB0BDE8F08F012B2ED0022BBA
:1010800033D0032B40D0042B00F06981052B00F0F6
:101090005781062BE3D114F801ECBEF1000F00F0EC
:1010A000D881BEF1010F00F01B8201360023032E10
:1010B00004F8023C04F1CC04BCD1DBE7232A54F849
:1010C0000A0C00F08281944B93F822309342B8D1FD
:1010D000F9F7AAFE012304F8023CC0E74D2800F00E
:1010E0006781002304F8023CB9E700233C2804F898
:1010F000023C00F057813E28B1D10122032304F8BD
:10110000012C04F8023CAAE7C028EAD800210423F5
:1011100004F8050C04F8040C04F8061C04F8023C5E
:101120009DE77E4B18680028A4D00AF040FDDFF848
:101130000CA27B4DDFF8F891DAF8000009F0BBFD56
:10114000002897D0DAF8000009F0AFFD09281BD07D
:101150003F2819D02B68002B67D1042800F0BA81F2
:101160000C2800F0CA807F28E6D0A0F12002D2B27D
:101170005E2AE1D80BB92028DED05A1C09F80300FA
:101180002A6014F0CDFCD7E72C68002C5AD1654FAB
:10119000A34607F51C78BBF1000F08BFBB4610370C
:1011A0004745F8D1BBF1000F00F04E81103FDBF84E
:1011B00000003A68065D135D9E42204402EB040184
:1011C00040F04081661E4E4422460BB9FD2A5CD990
:1011D00006F8013F01322A6010F8013F11F801EFD3
:1011E0009E45F2D00AB15F4512D04F4814F0A0FCE2
:1011F0005F4508D35BF8100B14F09AFC092014F03B
:101200008FFCBB45F6D9494814F092FC2A680024AB
:10121000944291D2661E4E4416F8010F14F080FCE1
:101220002B6801349C42F7D386E70C2865D00A2846
:1012300034D00D2832D07F2800F0BE80FF2B3FF63F
:101240007BAF92E7374E002706F51C78BB4602E0DD
:10125000103646450DD0224631684846F8F7F0F979
:101260000028F5D1B346002FF2D137461036464557
:10127000F1D13B465F469B46002B98D1002F3FF4AF
:101280005BAF294814F054FCB4E7511C202009F846
:101290000200296009F801300A46A4E714F0C9FCED
:1012A000232123482DF04FFC002800F01181A0EBF2
:1012B0000900286090B1431E19F80310202940F05E
:1012C0002C8109EB030243B112F8011D202903F11F
:1012D000FF304FD10346002BF6D12B604FF48072C4
:1012E000002148462DF018FC074B1B78002B3FF4DB
:1012F000C1AE0E4814F01CFC1EE70E4814F018FC9A
:101300000A4814F015FC17E781920020484100209C
:10131000EE76002078210020BC5A0020D440002026
:101320008C260020D4FA03084C2204085422040816
:101330008C2500205C220408FCEC0308D840002027
:1013400014F8063C14F8051C99426FD814F8043CB4
:1013500083427FF4C6AE062304F8023C9BE614F8F1
:10136000043C04F8030C5A40052304F8042C04F848
:10137000023C74E62B606A4C002204F51C7809F8E4
:10138000032002E0103444454CD0216848460CF05C
:1013900057FE0028F6D0444544D2E368984700231E
:1013A0002B609BE7032204F8013C04F8022C56E66C
:1013B000022304F8023C52E6013B002259482B600C
:1013C00009F8032014F0B4FBB6E6574B5749DB7815
:1013D000574ADFF888E11060003318BF01230B7013
:1013E000544B554ACEF80030544B7A604FF0400EC3
:1013F000012187F80CE03860B8607D73504819709F
:1014000014F076FD4F4814F093FB4FF400600BF09E
:10141000DDFD4D4B93F82230232B3FF459AE14F8E9
:10142000023C36E6494814F083FBB8E714F8041C84
:1014300008EB03005140013304F8041C04F8063C97
:1014400082720CE62246CDE64148103F14F070FB54
:10145000D0E69BE80F000DF1280C0DF1080888E894
:101460000F004CF824ED14F8053C14F803AC069476
:10147000624623444FF0010C414606A8ADF822E035
:101480000793ADF820A08DF824C000F069F840B1B2
:10149000029A304B03924146A4F10A0002931CF0D9
:1014A000F9FBDDF80480002304F8023CB8F1000FDA
:1014B0003FF4DBAD54F80A0C1CF0ACFC013654F8D8
:1014C0000A0CC047032E04F1CC047FF4B3ADD1E580
:1014D0002868EFE620480CF083F90BB0BDE8F08FE8
:1014E00014F8053C14F8032C0694234407936E2A41
:1014F0004FF0000308930993ADF820207FF4D5AD99
:1015000006A8F8F71FF906A8F8F710F906A8F8F7E3
:101510000DF906A8F8F70AF9C7E503462BE700BF5F
:10152000D4FA0308842204089C920020E04300209F
:10153000D84000207C210020D1AA010881920020FF
:101540008822040854220408BC5A00206822040897
:101550004C220408E09400208C250020D440002078
:101560002DE9F04F95B0B0F908500D81EDB2442D42
:1015700000AF0C46904600F04684064643D9812DC4
:1015800000F07F8300F29880542D00F0CC8040F270
:10159000D6806E2D00F00584802D40F0D380764BF0
:1015A00093F800A00AF1020A1AF0FF0A00F09780EF
:1015B000724BDFF8F481724EDFF8F0B19A4403F118
:1015C00001090A2516E0322D01F0E882A5F13C0060
:1015D000C0B2132841F2E98200232268511C216025
:1015E00015702268CA4502F101012160137076D09E
:1015F00019F8015B0A2DE6D1BBF80030FF2BA8BF1C
:10160000FF23DBB2E9E7052D00F0EB8320D8022DA4
:1016100000F0818040F21483032D00F0B983042D83
:1016200040F09080574920462A46F8F791F800216B
:101630002046F8F7D5F822680021531C01252360C5
:1016400028462B46543711706381BD46BDE8F08FA4
:10165000242D5ED040F2AA82282D00F05B83382D25
:1016600070D10A68484B0125511C21601570226811
:10167000052150192060117022680A21501920603C
:1016800011702268002150192060117022681978A9
:10169000501920601170226859785019206011701B
:1016A00022689978531923602B46117028465437C5
:1016B0006381BD46BDE8F08FA02D18D040F2958221
:1016C000B82D00F06383FE2D3CD1304D05F10806A6
:1016D00035F8021B2046F8F783F8B542F8D101250A
:1016E0002B46284654376381BD46BDE8F08F284B12
:1016F00008461968F8F75CF8264B20461968F8F791
:1017000057F8254B196820460125F8F751F82B4664
:10171000E7E7224BF6E70422214920460125F8F7A6
:1017200017F82B46C2E70B6800215A1C226019707B
:1017300022680125531923602B461170B6E7522DFC
:101740003FF479AF214628460AF0E6FB034600281D
:10175000C5D1742D00F08782772D29D13268716848
:1017600091421EBF531C336011780E4A08BF1946C0
:1017700020462AF0F1FAB2E7CD8F00200CED0308E5
:1017800028430020A2920020072B0020F08F002089
:10179000107AFF1F147AFF1F187AFF1F10310020E4
:1017A000C0220408D9B30308676666665043002068
:1017B000F52D01F04A83762D00F02D83472D01F0A1
:1017C0008B82292D326801F05482392D01F020825C
:1017D000212D01F02E8270680B3D811AEF2D00F251
:1017E00063860FF2080E5EF825F000BF032601089D
:1017F000A9240108A9240108A9240108A924010891
:10180000A9240108A9240108A9240108A924010880
:10181000A9240108A9240108A9240108A924010870
:10182000A9240108A9240108A9240108A924010860
:10183000A9240108A9240108A9240108A924010850
:10184000A9240108A9240108A92401088526010862
:10185000A9240108E1250108A9240108B7250108E8
:10186000A9240108A9240108A92401088F25010839
:10187000A924010819250108A9240108A92401089F
:10188000A9240108A9240108A924010807250108A1
:10189000A9240108B3240108A92401085B24010834
:1018A000A9240108A9240108A9240108A9240108E0
:1018B000DF160108A92401082F240108A924010822
:1018C000A924010815240108A92401083D290108BB
:1018D000A9240108A9240108A9240108A9240108B0
:1018E00031290108A9240108A9240108A924010813
:1018F000D9290108A9240108E3280108A92401081D
:10190000A9240108A3280108A9240108A924010881
:10191000A9240108A9240108A9240108A92401086F
:10192000A924010835280108A9240108B3270108C2
:10193000A9240108F9260108A9240108E72A0108B9
:10194000A9240108BF2A0108312A0108192A01081F
:10195000A9240108A9240108A9240108A92401082F
:10196000A9240108A9240108A9240108A92401081F
:10197000A9240108A9240108A9240108A92401080F
:10198000A9240108A9240108A9240108A9240108FF
:10199000A9240108A9240108A9240108A9240108EF
:1019A000A9240108A9240108A9240108A9240108DF
:1019B000A9240108A9240108A9240108A9240108CF
:1019C000A9240108A9240108A9240108A9240108BF
:1019D000A9240108A9240108A9240108A9240108AF
:1019E000A9240108A9240108A9240108A92401089F
:1019F000A9240108A9240108A9240108A92401088F
:101A0000A9240108A9240108A9240108A92401087E
:101A1000A9240108A9240108A9240108A92401086E
:101A2000A9240108A9240108A9240108A92401085E
:101A3000A9240108A9240108A9240108A92401084E
:101A4000A9240108A9240108A9240108A92401083E
:101A5000A9240108A9240108A9240108A92401082E
:101A6000A9240108A9240108A9240108A92401081E
:101A7000A9240108A9240108A9240108A92401080E
:101A8000A9240108A9240108A9240108A9240108FE
:101A9000A9240108A9240108A92401086B2A010826
:101AA000A92401084F2A0108952A0108A924010840
:101AB000A9240108A9240108A9240108A9240108CE
:101AC000A9240108A9240108A9240108A9240108BE
:101AD000A9240108A9240108A9240108A9240108AE
:101AE000B9230108672301082F230108A92401084D
:101AF0008D22010819220108FD210108A9240108ED
:101B0000E3210108772101084F2101083D21010847
:101B1000DD200108A9240108AD200108A92401083D
:101B2000A92401088320010855200108412001084B
:101B300019200108A9240108EF1F0108C31F01088B
:101B4000AB1F0108A9240108A9240108A924010840
:101B5000A9240108A9240108A9240108A92401082D
:101B6000A9240108A9240108A9240108A92401081D
:101B7000A9240108A9240108A92401088B1F010830
:101B8000A9240108A9240108311F0108A92401087A
:101B9000A9240108A9240108CD1E0108A9240108CF
:101BA000A9240108A9240108631E0108202D7FF43F
:101BB000C9AD0B68B14D591C6A7821601A70236851
:101BC0002A78591C21601A702368AA78591C216050
:101BD0001A7029892046F7F703FE23686A79591C91
:101BE00021601A702268A97927E5822D7FF4AAADB9
:101BF0000B68A34AA34D1178A04A581C20601970A5
:101C000011892046F7F7ECFD9F4B22681B88FF2BBC
:101C100002F10101A8BFFF2321601370A96881F3BD
:101C2000100189B22046F7F7DBFD296801F30F01A7
:101C300089B22046F7F7D4FD944B22681978FCE46A
:101C4000012D7FF47FAD0B680022591C21601A70B2
:101C500023685A1C22601D7022682521531C2360B2
:101C60002B46117022E53268716891421EBF531CE9
:101C700033601178864A08BF194620462AF06CF86E
:101C80002DE5844B1E78033616F0FF063FF427AD92
:101C9000814BDFF830821E4403F1010A4FF00A093C
:101CA00020E0B9F1500F00F07687B9F1320F00F063
:101CB0009287A9F13C00C0B2132840F2908700251A
:101CC000294623685A1C2260204683F80090F7F7C3
:101CD00087FD29462046F7F783FD56453FF4FFACC4
:101CE0001AF8019BB9F10A0FDBD16C4B9D6819689A
:101CF00005EB85054FF6FF736D009D42A8BF1D469D
:101D00009942A8BF194625EAE57521EAE171ADB20D
:101D100089B2D6E70B68DFF8B091614E591C0222F8
:101D200021601A7023684FF006085A1C226083F85D
:101D3000008023680A22591C21601A70236801253B
:101D40005A1922601D70B9F800102046F7F748FDB7
:101D5000B9F802102046F7F743FD23685A192260AC
:101D600083F8008023685022591921601A70236873
:101D70000022591921601A7031882046F7F730FD8A
:101D800071882046F7F72CFD2B468FE4454BB9E4CC
:101D90000B685A1C0A601D700B685A1C0A601D7083
:101DA00049E4394B0A681B88364DFF2BA8BFFF2337
:101DB000511C21601370A96881F3100189B220467B
:101DC000F7F70EFD384B20461988F7F709FD29680B
:101DD00001F30F0189B220460125F7F701FD2B46DB
:101DE00064E40B2231492046F7F7B2FC082230495F
:101DF0002046F7F7ADFC012507222E492046F7F7CC
:101E0000A7FC2B4652E4002A3FF469AC2A4B13602E
:101E100001252B464AE43268511C31601278002AB1
:101E200001F0C080102A01F02D811E461946256858
:101E30006B1C236020462A70F7F7BAFC3146204617
:101E4000F7F7B6FC1D4B20461968F7F7B1FC2046A2
:101E50000021F7F7C5FC00212046F7F7C1FCFFF78A
:101E6000EABB174B1B78DB0700F11E830125FDF74A
:101E700041FDFDF719FF2B4618E400BF308E00200E
:101E8000F69000206C8C0020E0900020D83D0020CF
:101E900061B40308CD8F00201CED0308DC42002054
:101EA000104300208C3F0020D82E0020C8220408B8
:101EB000D4220408E0220408F9BE0108C42300204B
:101EC0004841002020430020DC3000203046F7F756
:101ED0002DFC3368B8851A46591C316012F8021B74
:101EE000326087F82E105A7887F82F20DA1C32607B
:101EF0009A7887F830201A1D3260DA7887F8312016
:101F00005A1D32601B7987F8323007F12C0000230C
:101F1000BB86F7F765FBC74AC74B1268801A4FF0BC
:101F2000010561F10001C3E906012B46FFF7BEBBC5
:101F3000531C336013780F2B00F2B682911C316072
:101F4000C3EBC303BD495078C854D01C30600B4468
:101F500091785970111D3160D1789970511D31609F
:101F60001179D970911D316051791971D11D31608C
:101F70009179597102F108013160D2799A71012584
:101F800014F042FC2B46FFF791BB3046F7F7CEFB2F
:101F9000DFF8B882A8F80E003046F7F7C7FB012536
:101FA000A8F80C002B46FFF781BB3046F7F7BEFBC5
:101FB000A34A00EB80004300012513802B46FFF766
:101FC00075BB1146531C33609E4B11F8020B187001
:101FD000316051785970D11C316091789970111D20
:101FE0003160D278DA7001252B46FFF75FBB3046AF
:101FF000F7F79CFBDFF88482A8F810003046F7F76B
:1020000095FBA8F812003046F7F790FB0125A8F8D9
:1020100014002B46FFF74ABB1346511C31608A4916
:1020200013F8020B08703360884953788B70D31C07
:102030003360834B92789A7001252B46FFF736BBAD
:10204000834B844918684E2201252CF040FD2B4615
:10205000FFF72CBB1146531C33607F4B11F8020B6A
:102060001870316051785970D11C316092789A7033
:102070003046F7F75BFB794B0125D8802B46FFF7FD
:1020800015BB3046F7F752FBDFF8D081A8F8000007
:102090003046F7F74BFBA8F802003046F7F746FB4F
:1020A0000125A8F804002B46FFF700BBDFF8D0910C
:1020B00099F80030002B3FF412ABDFF8C8810025FF
:1020C0003046F7F733FB15F05BF999F80030A8ECD0
:1020D000010A01359D42F3DBFFF701BB0D2940F0FA
:1020E000E381531C33601578072D00F2DD81DFF8A2
:1020F000989130464FF00C08F7F718FB08FB05F8ED
:1021000009EB0805A8803046F7F710FBE880304659
:10211000F7F70CFB336828811A46591C316012F816
:10212000021BA97232605B78EB723046F7F7E6FA71
:10213000012549F808002B46FFF7B8BA3046F7F7F3
:10214000F5FA474B012518802B46FFF7AFBA531C11
:1021500033601078060600F1F787424B1B78DD07E5
:102160003FF5BDAA032828BF00200125FDF786FB07
:102170002B46FFF79BBA531C3360304692F800A001
:10218000F7F7BCFA81463046F7F7B8FA054630460D
:10219000F7F7B4FA80463046F7F7C8FA3046F7F753
:1021A000C5FA3046F7F7CEFABAF1000F00F0B5875E
:1021B000BAF1100F7FF493AA1F4BC3F804909D60EF
:1021C000B8F1000F02D0284BC3F800802749284BF4
:1021D0000222081F01251A7026F088FB2B46FFF704
:1021E00065BA204B1B78D8073FF579AA0125FDF782
:1021F00061FBFDF759FD2B46FFF758BA194B1B78C9
:10220000DA073FF56CAA1B4A1378012543F0040353
:1022100013702B46FFF74ABA124B1B78D9073FF5CC
:102220005EAA154B4FF4C87201251A802B46FFF7A2
:102230003DBA00BF14540020C8210020A03E002059
:10224000FC30002058870020B85B0020EC300020D4
:10225000A08E0020F4F50308E4300020784200202E
:10226000448B002048410020C4230020D0210020BE
:10227000388A00209E8E0020B8420020CC7A0020B0
:10228000CD8F0020B4400020E03D0020092940F31C
:102290000B81DFF8E4831346511CD8F800503160FD
:1022A00013F8021B297033605378AB70D31C336072
:1022B0009378642B02F10401A8BF64236B71316031
:1022C000D378642B02F10501A8BF6423AB713160A0
:1022D0001379EB71931D33605379642B02F107017D
:1022E000A8BF64232B7231609379EB7002F108036D
:1022F0003360D3792B713046F7F718FA7268336878
:102300006881D11A00290CDD591CD8F80000316011
:10231000521A002A1978417203DD9A1C32605B78E8
:10232000437001251AF026FD2B46FFF7BFB9C34BBA
:102330001868D31C014621329D1E356013F8035CDA
:102340000D705D1E356013F8025C4D70336013F83C
:10235000015C8D7003339A4201F10301ECD114F05A
:10236000B9FEFFF7BCB9531C33601378B449002B96
:1023700000F09A860B7843F00203901C0B70B14D6D
:10238000306053782B753046F7F7B8F9286030463F
:10239000F7F7B4F968603046F7F7C8F92881304696
:1023A000F7F7C4F9A84AE8811378012543F002033E
:1023B00013702B46FFF77AB9C1F34705122D73D876
:1023C000C5B107F1500307F12A0903EB450AC846D6
:1023D000AAF1260A3046F7F7A9F928F8020FD045E6
:1023E000F8D19A4B39F8022F23F8022FC845F9D1BA
:1023F000112D09D8964A6B00023B1344002122326A
:1024000023F8021F9A42FBD1924A01231D46137002
:10241000FFF74CB9904B02F108010132326012F81B
:10242000010C03F8010F8A42F7D1FFF758B91346A0
:10243000511C3160894913F8025B8D703360557807
:102440004D7083423FF44BA9D31C3360844B927888
:102450001A7401252B46FFF729B90723B1FBF3F3C3
:10246000C3EBC305491B1FD1DBB203F1FF395FFA90
:1024700089F9002B3FF433A9DFF8E8A109F101093C
:102480000D46531C336092F90010764B4FF0000854
:1024900093F902208A4203F1080300F0888508F1CD
:1024A0000108B8F1040FF3D14FF0FF352B46FFF7C9
:1024B000FDB8531C336013780E2BF5D8911C316096
:1024C0005578032DF0D86848062101FB03F1431825
:1024D00002F1030E5D71C6F800E095784554111DB8
:1024E0003160D1785970511D316011799970911D09
:1024F00031605179D970D11D316092791A710125FD
:102500002B46FFF7D3B8531C3360584B12785A75DB
:1025100001252B46FFF7CAB8531C544D336013787E
:102520002B723046F7F702F9A8833046F7F7FEF82A
:1025300028833046F7F7FAF832686883531C336013
:102540001278EA747268D31A032B00F3B2853368E9
:10255000D11A05290EDD5A1C32601B78EB72304609
:10256000F7F7CCF83368E8605A1C32601B782B749C
:1025700033687268D21A002A7FF7B1A85A1C3260F9
:102580001B7885F8213001252B46FFF78FB8531CA7
:102590003360374915780D70C01A00287FF79FA85F
:1025A000931C33605378003318BF012301254B700F
:1025B0002B46FFF77BB83046F7F7B8F8DFF8BC805A
:1025C000C8F800003046F7F7B1F8C8F80400304604
:1025D000F7F7ACF80125C8F808002B46FFF766B8F6
:1025E000DFF89C800023C8F800303046F7F786F803
:1025F000D8F8003001250343C8F800302B46FFF718
:1026000055B81C4810294FF000020B4628BF102374
:10261000026042608260C2600274002B3FF45FA8D7
:102620003268411E13440132326012F8010C01F885
:10263000010F9A42F7D1FFF752B800BFA08E0020D9
:102640009E8E0020787E0020368A002052280020AE
:1026500054280020782800208F5A00200C310020B8
:10266000C8210020BC5A0020983F0020905A00202A
:1026700020310020C8300020A48E0020D45100203A
:1026800010310020511C316015783B62132D3FF64C
:102690000BAF911C316050787A6229F097FB0028CB
:1026A0003FF402AF7A6ABC49007801F82500D01CDB
:1026B000306001EB850590786870101D3060D0782F
:1026C000A870501D30601279EA7001F150003B6A29
:1026D00002E00431884207D00A78002AF9D18D78C7
:1026E000CA789542F5D20123AC4A83F00103012553
:1026F00013702B46FEF7DABF531C3360A84DDFF88A
:10270000C882137888F805303046D5F80090F7F77E
:102710000DF8A9F820003046D5F80090F7F706F834
:1027200072683368A9F81E00D11A072919DD3046EE
:10273000F6F7FCFFA8F80A003046F6F7F7FFA8F80E
:102740000C003046D5F80090F6F7F0FFA9F822000B
:102750003046D5F80090F6F7E9FF33687268A9F8BB
:102760002400D11A03290BDD3046F6F7DFFFA8F865
:102770000E003046F6F7DAFF33687268A8F81000EA
:10278000D21A002A05DD591C2A6831601B7882F8AC
:102790002630FDF7E1F91EF0C1FA824B1B68002BD1
:1027A00000F077842868012514F0C4F82B46FEF762
:1027B0007DBF1346511C3160DFF80C8213F8021BF9
:1027C00088F802103360784953780B70D31C33605B
:1027D000764D93782B71131D3360D378092BA8BFE6
:1027E00009233046AB70F6F7A1FF33687268288082
:1027F000D11A012905DD3046F6F798FF3368726873
:10280000E8819A4207D05A1C32601B78003318BF07
:10281000012388F80730FDF79FF9336872689A4200
:102820003EF45DAF5A1C32601B78EB7001252B46DD
:10283000FEF73CBF5E4B1B68002B3EF450AF26F00A
:102840004DF9FF283EF44BAF3046F6F76FFF3F28B7
:1028500040F29284DFF87481002588F800503368D4
:102860007268A8F80400D21A012A7EF738AF1A4617
:10287000591C316012F8021B88F8021007F1500051
:10288000326000225D7800F8242D26F0F9F897F8E0
:102890002C30AB423EF423AF284626F015F9FEF764
:1028A0001EBF444B1B78012B3EF619AF531C11463B
:1028B0003360DFF81C8111F8023B88F80230D31C2A
:1028C000C01A3160012892F801E0336040F3478478
:1028D0003046F6F72BFF0125A8F800002B46FEF73F
:1028E000E5BE531C336092F80080B8F1110F3FF63B
:1028F000DBAD931C3360304D537805F8183030460B
:10290000F6F714FF40F6CA039842A8BF184640F2F3
:10291000EE23984205EB4801B8BF18460125A0F206
:10292000EE222B46192092FBF0F24A70FEF7BEBE53
:102930000125F8F761F82B46FEF7B8BE531C33604B
:102940001E4B1278DFF88C801A700023C8F8003014
:102950003046F6F7D3FE3368D8F800201849194DF1
:1029600010435A1CC8F8000032601B780B723046C6
:10297000F6F7DCFE28603046F6F7D8FE6860304691
:10298000F6F7D4FEA8603046F6F7D0FE3046F6F7EC
:10299000CDFEFEF7A4BE00BF80290020100F00204E
:1029A000A08E002018310020E0300020CC7A0020DA
:1029B0004C410020382C0020902A0020203100209B
:1029C000905A0020D4510020B85B002050410020D4
:1029D0003A2C0020103100201346511CB14D3160BB
:1029E00013F8021B2971336053786B713046F6F788
:1029F0009DFE336828805A1C32601B78AB713046CC
:102A0000F6F794FE336868805A1C32601B78EB71CD
:102A100001252B46FEF74ABE531C33601378002B6A
:102A200000F06B834FF400400AF0D0FAFEF757BE77
:102A30009D4B1B7813F001017FF436AD531C3360BE
:102A40001078012512F09EFE2B46FEF72FBEDFF810
:102A5000808200233046C8F80030F6F74FFE01258B
:102A6000C8F800002B46FEF721BE1346511C31600A
:102A700013F8025B3360D31C507833609178002DDB
:102A800000F08A83012D7EF42AAE12F039FF2B4626
:102A9000FEF70CBE531C854833600178137800297B
:102AA00040F0378304220270814A9B001380FEF7B6
:102AB00005F8804B012518622B46FEF7F7BD13463B
:102AC000511C31607C4913F8020BC87033607B499C
:102AD00053784B71D31C3360794B9278DA700125AF
:102AE0002B46FEF7E3BD3046F6F720FE3046F6F7FC
:102AF0001DFE3046F6F71AFE3046F6F723FE336821
:102B0000704D1946581C2A68306011F8020B82F883
:102B10002C003160597882F83610D91C31609B78CE
:102B200082F837303046F6F70DFE3046F6F70AFEEB
:102B30003046F6F707FE3046D5F80080F6F7F6FD8A
:102B4000A8F83A003046D5F80080F6F7EFFD336874
:102B50007268A8F83800D11A01290ADD591C2A68C0
:102B600031601B7882F82E303046F6F7EBFD336883
:102B70007268D31A032B0BDD3046D5F80080F6F7C8
:102B8000D5FDA8F8320030462E68F6F7CFFDB086A6
:102B90002868FFF7E4BB4C4BFFF7A8B83388FF2B3E
:102BA000A8BFFF23DBB2FEF718BD25F04FF80028C1
:102BB0003EF412AD03780A2B28D8B0F9023088FB16
:102BC0000312DB17C3EBA2039BB2FF2BA8BFFF23AB
:102BD000DBB2FEF702BD98E82200FFF789B825F0C6
:102BE00035F800283FF46BA803780A2B3FF667A856
:102BF000B0F90430B0F9061003EB830383F35005FA
:102C000021EAE171ADB289B2FFF75BB80023DFE7DB
:102C1000531C336013780A2B00F0B3813046F6F76B
:102C200091FD3046F6F78EFD3046F6F78BFDFEF748
:102C300056BD1346511C3160244D13F8021B6970B8
:102C4000336053782B70D31C33609378AB7030466D
:102C5000F6F76CFD33682881591C1A46316012F86A
:102C6000021B697132605B78AB7101252B46FEF760
:102C70001DBD531C336013780A2B00F07C81502B50
:102C80007FF481AE3046F6F751FDDFF84880A8F8B2
:102C900000003046F6F74AFD0125A8F802002B4651
:102CA000FEF704BD94420020484100202A3D002048
:102CB000D82E0020C8210020EC300020CC8B002032
:102CC000FC300020A08E002014430020308E002015
:102CD0008C3F002010430020726835687B623046CC
:102CE000551BF6F70BFD052D38627B6A00F2368125
:102CF0008026B246012594E80600521A103AB242E4
:102D0000B8BF1FFA82FABC4A396A92683A61521A0D
:102D10009245396A7B622046FA6088BF1FFA82FAC0
:102D2000F6F746FD7B6A002B00F00281002D40F093
:102D3000E9802368C7F800D05D71C0B00533C7F8DB
:102D400008D0FB61BAF1000F00F0D3813B6A3A6909
:102D5000934280F0DB81386A7D62AB462A467C6014
:102D60008025FB68BC689A1AB2F5807F28BF4FF4B3
:102D700080722146F7F7D2FEF969B86104EB000CC6
:102D80000B787B6164452ED2DFF888920CF1FF3C12
:102D900004F1FF3E1EF8013F09EB830219F82340BE
:102DA0005688ECB100234FF4004204F1FF3816427C
:102DB0004FEA520202D00878284308706D0806D105
:102DC0000BF1010B4D701FFA8BFB01318025DA45A9
:102DD00003D8F44533D8984531DC01339C42E6D121
:102DE000F445D7D1F9617B6ABA6913449BB2DA45DD
:102DF0007B6206D97B6A3A6AD0181A463B699842C8
:102E0000AFD37C68802D1CBF0BF101031FFA83FB3D
:102E10000BF1020189B22046F6F7E2FC2368796AD9
:102E200001255A19226020461D70F6F7D9FC236847
:102E30005B4423602B46D7F800D0FEF737BCFB6914
:102E40007C681A463B7D1370DCE7336872689A42EF
:102E500040F0E680694BFF221A704FF0000A684D7F
:102E600011F02CFB51462022664885F800A02BF07B
:102E700053FE87F82CA097F82C30072B00F207811F
:102E8000DFF894915F4E524697F82C3003EB4303E2
:102E900009EBC3035B7CE3B197F82C3003EB4303EE
:102EA00009EBC30320215B699BB197F82C3003EB3E
:102EB000430309EBC303586946F8220008F088FA77
:102EC0002B7856F8230008F040FB2A780132D2B262
:102ED0002A7097F82C300133DBB287F82C3097F842
:102EE0002C30072BD0D92368591C21601A70B8F1F7
:102EF000000F3EF4F4AB444BC8F8003001252B46DC
:102F0000FEF7D4BB5246386A2168F7F707FE2368FC
:102F1000B04203442360BEF6E2AB002100E0236828
:102F200001305A1CB04222601970F8D1FEF7D7BBAD
:102F3000002DE7D151462046F6F752FC2368386A47
:102F40005A1C22601D7052462168F7F7E7FD23687E
:102F50000125034423602B46FEF7A8BB3046F6F755
:102F6000E5FB326871687B6A9142824640F081805D
:102F700006461D46BFE63046F6F7D8FBDFF89C80D4
:102F800085E6931C3360214B51781970D11C316058
:102F900091785970111D3160D2789A7001252B46B5
:102FA000FEF784BB1A4B93E84200FEF740BF0AEBE2
:102FB000C80B30468BF80210F6F7B8FB33682AF8D6
:102FC00038001A46591C316012F8021B8BF80310A6
:102FD00032605A788BF80420DA1C32609A788BF8C9
:102FE00006201A1D32600135DB788BF80530A945C3
:102FF0007FF447AAFEF773BB0C110020C821002004
:1030000077920020389200205D9E0308072B002055
:103010002C8A00202CED0308F8640020DC3000200E
:103020005A1C194632605F4811F8022B0270316059
:103030005B784370042A03D9FF2A7EF4FCAA0CE7CC
:1030400059490978994205D8022A7EF4F4AAFF2B3F
:103050007EF4F1AA236801255A1922601D70B8F187
:10306000000F3EF43CAB514BC8F800302B46FEF746
:103070001DBB511C316012781D46131C064618BF3B
:10308000012338E6474B59689E68FEF7D0BE52468A
:1030900029E747484749484A484B036001250B60E8
:1030A00013602B46FEF702BB0B7803F0FD03FFF71E
:1030B00064B93046F6F73AFBA8843046F6F736FB9B
:1030C00033687268E884D11A03297FF741AA1A4647
:1030D000591C316012F8021BA97732605B7885F8C1
:1030E00020303046F6F722FB336872686884FFF7B9
:1030F0002FBAD346C7F824A08AE6314A13680125BF
:1031000023F4004313602B46FEF7D0BA7D62AB4632
:103110007EE604297EF4E3AAC6E42A4B1020C3F815
:1031200000905D6009F022FF274A137843F0010305
:103130001370B8F1000F3EF4D2AA244B0125C3F856
:1031400000802B46FEF7B2BA00F07F00032828BFAC
:103150000020012512F0F0FB2B46FEF7A7BA1C4B0E
:1031600091781A88012512FB0EF22B4692FBF1F2A0
:10317000A8F80020FEF79ABAC50800F00703013549
:103180000133EDB2DFF84C802846194688F801304B
:1031900024F0B8FCFFF761BB012513F01EFE2B469F
:1031A000FEF784BAC8210020CD8F002005BF01089A
:1031B0006C340020C0340020C0380020D5830008C3
:1031C000988E00202C8A00209E8E0020C423002090
:1031D000462F0020504100202DE9F04F2DED0C8BA3
:1031E000364C97B06368069020469847002800F058
:1031F0007D82B4F8A870002284F85120002F67D196
:10320000656AB4F93860206AB4F93A20A16AB4F961
:103210003C30521B301A2A4DE0625B1A04F12C003C
:1032200094F8521063630795226315F015FB2B6821
:10323000990042F14D81D4ED0B7ADFF88CA0DFF8D4
:103240008C909AED405ADAED415A9AED426ADAF8DA
:103250000C31D9F80020F8EEE76AD4ED0C7AB8EE1C
:10326000E77AD4ED0D7AF8EEE77A013376EE856AE7
:1032700037EE257A77EE867A9342CAED406A8AED78
:10328000417ACAED427ACAF80C3101F0D2840D4B72
:10329000049393F800C0BCF1140F03F05B85DAF8D7
:1032A00014210025062A01F2A285DFE812F0E518B4
:1032B00051180B1764187F17FD17810DCC5B002088
:1032C000B8630020EC8F0020F8210020B8390020DE
:1032D000D44BD549079391F801901B68D348DFF888
:1032E000A08304904FF47A71B1FBF3F3C3EB431660
:1032F00003EB8603DE00B6B2B7420578B8F90600E4
:1033000003F00D82D4F87CE0B4F93820236E0EF17E
:10331000010107EE902A13440129E1672366F8EEC4
:10332000E77A03F00682D4ED1B5AD4ED1D6A07EE4E
:10333000101A37EEE56AB8EEC75A012F86EE057A05
:1033400037EE257A77EEC77A84ED1C7AE7EE866A47
:1033500084ED1B7AF0EE667AC4ED1E6AC4ED1D6A38
:1033600003F06A86D4F890E0B4F93A20636E0EF167
:10337000010107EE902A13440129C4F890106366F6
:10338000F8EEE77A03F0ED81D4ED205AD4ED226A0D
:1033900007EE101A37EEE56AB8EEC75A012F86EE2F
:1033A000057A37EE257A77EEC77A84ED217AE7EE53
:1033B000866A84ED207AF0EE667AC4ED236AC4ED65
:1033C000226A03F01186D4F8A4E0B4F93C20A36E7D
:1033D0000EF1010107EE902A13440129C4F8A4104C
:1033E000A366F8EEE77A03F0D581D4ED255AD4ED43
:1033F000276A07EE101A37EEE56AB8EEC75A012FB2
:1034000086EE057A37EE257A77EEC77A84ED267A4E
:10341000E6EE276A84ED257AF0EE667AC4ED286A36
:10342000C4ED276A03F0D385DFF858A2A8F8060098
:10343000B4F8A830049A013B1578A4F8A83007998D
:103440000023072D4B608B60CB6040F05781FDF768
:1034500035FB049BDFF828821D78069BC01A9AF87A
:103460002131A8F800000993002B40F04D816E4BEC
:103470005B79002B01F00A836D4B1B78013BDBB2BB
:10348000072D8AF8213102F0EC8300230A93694A60
:10349000DAF82C31D2ED006A674A9FED686AD2F8FB
:1034A00000B0604A0792069ADAED4AAADFF8D8819E
:1034B0009AED499A9FED62AADFED62BA9FED62CA6A
:1034C0009FED62BADFF8C491614FCAF82C21D31A7C
:1034D00007EE903AF8EE677AB7EE007AC6EE279AD2
:1034E00008F11C03002508935A4B05932E4677EEEE
:1034F0006A8A68EEA68AF4EEC78AF1EE10FA88BFEF
:10350000F0EE478A544B98ED008A2B44D3ED007AB5
:10351000F5EE407AF1EE10FA17D0504B2B4493EDB4
:10352000007A78EE476AB0EEE66AF4EEC67AF1EE1B
:1035300010FA08D5F5EEC06AF1EE10FACCBF37EEFE
:10354000878A37EE678A83ED008A454B1A8893078E
:103550003FD0022E3DD0434B9BF82E1033F916304E
:1035600007EE103A089B07EE901A2B44F8EEE76A34
:10357000B8EEC77AD3ED007A4B42A6EEA77A700078
:1035800007EE903AF8EEE77AB4EEE77AF1EE10FA49
:103590000AD407EE901AF8EE677AF4EEC77AF1EEE5
:1035A00010FA88BFF0EE477A2F4B30490344085E8B
:1035B000B3F90C30C01A07EE100AB8EEC77AD0077C
:1035C000E7EE4A7A41F1F881294B93ED008A27EE24
:1035D000888A079B9AF864212B4493ED01DA78EEF0
:1035E0004DCA002A00F0E780224BDAF868210699DC
:1035F0001B688A1A9A4240F3DE809BF84830022BFF
:1036000002F07883022E04F079851B4B1B68990722
:1036100000F19280194B87ED00CA1B689342C0F2FB
:10362000C48035E0A8630020B85B0020EC8F002048
:10363000E030002014390020A08E002000247449BE
:10364000CDCCCC3DAE47813F000000000000C84219
:10365000942E0020882E00200839002034230020DA
:103660009C8E002040230020EC3000204C8E002057
:10367000F03800201C390020408E0020183900202E
:10368000F08F0020F821002028230020A02E002009
:10369000F7EE007AF4EEE7AAF1EE10FA40F18B8033
:1036A00007991F4BD1ED017A93ED007AF0EEE77A9E
:1036B000F4EEC77AF1EE10FA7DD5D1ED027AF0EE94
:1036C000E77AB4EEE77AF1EE10FA74DDD1ED037A21
:1036D000F0EEE77AB4EEE77AF1EE10FA6BDD114B1B
:1036E0001B689A0761D51049104B45E0104BDFF875
:1036F00044A01D780493072D3FF4A9AE9AF8213118
:103700000993002B3FF4B3AE581E8AF82101012D16
:1037100001F0BE8317B0BDEC0C8BBDE8F08F00BF8D
:1037200024390020408E00204C8E0020EC300020F8
:10373000EC8F0020F8210020D64BD749DFF8CCE3EE
:1037400031F916C09EED008ADFF8C4E387ED00CAA8
:1037500003EB460028EE0A8AB0F90C00A0EB0C003F
:1037600007EE900AF8EEE77ADEF8000027EE888A86
:10377000904278EE4DCA8BDAB3F90C20B1F900E033
:10378000C648AEEB020E00688EEAEE72A2EBEE7255
:10379000824210DAB3F90E30B1F90220D21A82EA6D
:1037A000E273A3EBE273984205DD002318468AF822
:1037B0006431FDF7E1FABA4B2B4493ED000A059B07
:1037C00029EE000A022E20EE2C0AA3EC010A059332
:1037D00004F05184B34BD7ED006A93ED007AB24BFD
:1037E000D3ED007AB14B93ED006AB14B67EE277AC7
:1037F0002B4427EEA87AD3ED007A67EE277AF0EE15
:10380000665AECEEA75AB1EE467AB4EEE57AF1EEDE
:1038100010FA08DCB4EEE56AF1EE10FA8CBFB0EEF7
:10382000657AB0EE467A9AED4A6AF7EE007AB4EE1F
:10383000E76AF1EE10FAACBF0123002343B1F0EECA
:10384000E66AF0EEC77AF4EEE67AF1EE10FA01D508
:1038500087ED007A022E04F0CC83964A964B52F8FC
:1038600026001B68B0EE4D0A9847944A944B52F8D4
:1038700026001B6898479BF8373023B1914B1B8873
:10388000002B01F00681B0EE4C8A8F4B38EE400AD7
:103890002B4493ED008A83ED000A9BF8483030EE0C
:1038A000480A20EE298A53B3884B1B78DB0741F185
:1038B0007680F7EE007AF4EEE7AAF1EE10FA9AF8C5
:1038C0006431C1F2C986002B01F08881DAF86831D1
:1038D000069AD31A7E4A12689A4210DD7D4BD3EDC8
:1038E000007AF0EEECCAF4EEE7CAF1EE10FA42F11B
:1038F0000A82002318468AF86431FDF73DFA764BB8
:103900009AF874212B4493ED000A29EE000A20EE68
:10391000088A89ED008A32B9059B87ED00CA03ED5C
:1039200001CA89ED00CA0136032E08F1040809F125
:10393000040907F1040705F104057FF4E3AD049BD6
:103940001B78072B01F08D86012B02F07781002375
:1039500008939AF87C31002B41F0A7825F4B604AB4
:1039600007931B681668D90496F82C7001F1AC8097
:103970005C4B5D4A059319465C4B498B5C4D92ED5F
:10398000005AD3ED004A5B4A5B4BD5ED036AD3ED99
:10399000005AD2ED007A92ED014A92ED026A8AED68
:1039A000635A07EE101AB8EEC77A74EEC53A0123CF
:1039B00036EEC77A8AED615ACAED603ACAED644ABA
:1039C0008AF89431C7EE258A338D5A4206EE902A42
:1039D0004A4A9FED4B5AD2ED005A4A4AD2ED004A6C
:1039E000B7EE007AF4EEC78A75EEA45AF1EE10FA3B
:1039F00088BFF0EE478A75EEA75AF8EEE66AF4EE55
:103A0000C58AF1EE10FA07EE903AF4EEE65AB8BF26
:103A1000F0EE458AF1EE10FACAED678AB8EE677AE1
:103A200001F13A84F4EEC75AF1EE10FA88BFF0EED5
:103A3000475A324B9FED345AD3ED017A314BD3EDD7
:103A4000014A77EEA47A65EE855A77EE847AF4EE31
:103A5000E76AF1EE10FA08DCB4EEE77AF1EE10FA5C
:103A60008CBFF0EE676AF0EE476A244A738DD2EDA0
:103A7000027A9FED257A5A4204EE902A76EE277A52
:103A8000F8EEE44A66EE876AF4EEE47AF1EE10FAB4
:103A900040E000BFEC3000204C8E00202039002098
:103AA000C4380020940000206834002038390020F9
:103AB000D0380020703400206C340020C434002042
:103AC000C03400209C8E0020642300204841002048
:103AD0001C39002028390020DC380020B863002081
:103AE000A08E0020905A00204C2F0020BC300020D7
:103AF000F8900020942E002080420020882E002084
:103B000000000000A02E00206F12833AF038002041
:103B1000183900200AD407EE103AF8EE474AF4EEBE
:103B2000E74AF1EE10FA88BFF0EE674AE94BDFEDA5
:103B3000EA7A5B7864EEA74A0BB9F1EE644A002F8B
:103B400041F0E587F7EE003AE44F3E78002E03F0AF
:103B5000D580E34B9FEDE36A93ED025A93ED017A32
:103B6000D3ED037A26EE855AA5EE875AA4EEA75A1E
:103B700023EE855AB4EEC65AF1EE10FAB4BFB0EE99
:103B8000464AB0EE454A98BFB0EE456A012E8DED2B
:103B90000E5A03F0F280D3ED067A93ED053A93EDD9
:103BA000077A66EEA77AE5EE837AE4EE877A23EE6B
:103BB000A77AB4EEC67AF1EE10FAB4EEC47A8CBFEE
:103BC000F0EE467AF0EE477AF1EE10FA98BFB0EEDA
:103BD000676AB4BFF0EE447AF0EE477A022E8DEDBC
:103BE0000F7A00F0DE8093ED0A7A93ED093A93EDB7
:103BF0000B4A26EE877AA5EE837AA4EE847A23EE2A
:103C0000877AB4EEC67AF1EE10FAB4EEE77A8CBF9A
:103C1000B0EE464AB0EE474AF1EE10FA98BFB0EE69
:103C2000446AA8BFF0EE477A032E8DED107A00F0BB
:103C3000B88093ED0E7A93ED0D3A93ED0F4A26EE90
:103C4000877AA5EE837AA4EE847A23EE877AB4EE9F
:103C5000C67AF1EE10FAB4EEE77A8CBFB0EE464ABF
:103C6000B0EE474AF1EE10FA98BFB0EE446AA8BF32
:103C7000F0EE477A042E8DED117A00F0928093EDEC
:103C8000124A93ED113A93ED137A26EE844AA5EE8B
:103C9000834AA4EE874A23EE844AB4EEC64AF1EE84
:103CA00010FAB4EEE74A8CBFB0EE467AB0EE447A32
:103CB000F1EE10FA98BFB0EE476AA8BFF0EE447A72
:103CC000052E8DED124A6CD093ED164A93ED153A00
:103CD00093ED177A26EE844AA5EE834AA4EE874A2E
:103CE00023EE844AB4EEC64AF1EE10FAB4EEE74A87
:103CF0008CBFB0EE467AB0EE447AF1EE10FA98BF7F
:103D0000B0EE476AA8BFF0EE447A062E8DED134A56
:103D100047D093ED1A4A93ED193A93ED1B7A26EEAC
:103D2000844AA5EE834AA4EE874A23EE844AB4EE81
:103D3000C64AF1EE10FAB4EEE74A8CBFB0EE467A0E
:103D4000B0EE447AF1EE10FA98BFB0EE476AA8BF21
:103D5000F0EE447A072E8DED144A22D093ED1E7AB0
:103D600093ED1D3A93ED1F4A26EE877AA5EE837AEE
:103D7000A4EE247A27EE237AB4EEC67AF1EE10FA96
:103D8000B4EEE77A8CBFF0EE466AF0EE476AF1EEE9
:103D900010FA8DED157A98BFB0EE666AA8BFF0EE06
:103DA000477A77EEC67AF7EE006AF4EEE67AF1EE3D
:103DB00010FACAED4A7A43F3F18786EEA77A022E0B
:103DC000DDED0F7A27EE055A67EE877A8DED0E5AF4
:103DD000CDED0F7A2DD0DDED107A67EE877A032EC8
:103DE000CDED107A25D0DDED117A67EE877A042EBD
:103DF000CDED117A1DD0DDED127A67EE877A052EB2
:103E0000CDED127A15D0DDED137A67EE877A062EA6
:103E1000CDED137A0DD0DDED147A67EE877A072E9B
:103E2000CDED147A05D0DDED157A27EE877A8DED8C
:103E3000157A2D4B1B68DA0041F1C583F6EE008A36
:103E4000CAED678A002E02F07D87284B264AD97872
:103E5000DFF8A0B09AF994310A919AED646A244986
:103E60001068BBF906200978DFF88CC0DAED635AD8
:103E70000B9207EE103A079B059A1B68DFF87CE06F
:103E8000528B9CF800909EED005A0C92BDEEC66AD3
:103E900001F0010816EE10CA0A99DAED606ADAED4F
:103EA000617ABDEEE56A00F0805E03F4805203F0B3
:103EB000100003F480030D93B8EEC77A16EE103AA3
:103EC000002941F0B5800649DDED0E5A91ED006AFA
:103ED00016E000BF203100206F12833ACD8F002002
:103EE000F041002000000000342F00200893002043
:103EF00048410020EC790020F07A0020EC410020BD
:103F0000002841F0D08428EE866AC24AA5EE876A6E
:103F1000F0EE675AE6EE265ABDEEE56A16EE10EAB6
:103F200016EE100AE645A8BF60467345C8BF18469E
:103F300006EE100AB8EEC66A012E82ED006A00F0A5
:103F4000DC8091ED046ADDED0F5A28EE866AA5EE5D
:103F5000876AF0EE675AE6EE265ABDEEE56A16EE7F
:103F600010EA16EE100AE645A8BF60467345C8BFC2
:103F7000184606EE100AB8EEC66A022E82ED016AF5
:103F800000F0BB8091ED086ADDED105A28EE866ADC
:103F9000A5EE876AF0EE675AE6EE265ABDEEE56AB0
:103FA00016EE10EA16EE100AE645A8BF6046734505
:103FB000C8BF184606EE100AB8EEC66A032E82ED98
:103FC000026A00F09A8091ED0C6ADDED115A28EE3C
:103FD000866AA5EE876AF0EE675AE6EE265ABDEECF
:103FE000E56A16EE10EA16EE100AE645A8BF60462E
:103FF0007345C8BF184606EE100AB8EEC66A042E0E
:1040000082ED036A79D091ED106ADDED125A28EE47
:10401000866AA5EE876AF0EE675AE6EE265ABDEE8E
:10402000E56A16EE10EA16EE100AE645A8BF6046ED
:104030007345C8BF184606EE100AB8EEC66A052ECC
:1040400082ED046A59D091ED146ADDED135A28EE21
:10405000866AA5EE876AF0EE675AE6EE265ABDEE4E
:10406000E56A16EE10EA16EE100AE645A8BF6046AD
:104070007345C8BF184606EE100AB8EEC66A062E8B
:1040800082ED056A39D091ED186ADDED145A28EEFB
:10409000866AA5EE876AF0EE675AE6EE265ABDEE0E
:1040A000E56A16EE10EA16EE100AE645A8BF60466D
:1040B0007345C8BF184606EE100AB8EEC66A072E4A
:1040C00082ED066A19D091ED1C6ADDED155A68EE95
:1040D000868AE7EE258AE6EEA87AFDEEE77A17EE05
:1040E000901A8C45A8BF8C468B42D8BF634607EE1A
:1040F000903AF8EEE77AC2ED077AB8F1000F01F0D6
:10410000A580454B1B68002B41F0AD80434B1B78CD
:104110009BB1387870B1DFF8FC80DFF81891002689
:10412000F0B2D9F80030B8EC010A98473878013677
:104130008642F5DB3A4B1B689847049B1B78072B9C
:1041400001F0A48200230B93079B1B680A935E0572
:1041500001F1B181334B1F683C0701F14E81324BB5
:10416000B3F80090314B0893314BBBF906801C68C3
:104170006289904580F201864FF07E53CAF824315F
:10418000089A059992F904300E8BBBF9000011785A
:1041900092F801E0002BA0EB060383EAE37CACEB92
:1041A000E37C14BF01224FF0FF32BCF5FA7FA8BFB9
:1041B0004FF4FA7C614580F2DC85ACEB010307EE3D
:1041C000903AF8EEE77A8642C5ED007A03DDF1EE2B
:1041D000677AC5ED007ABBF90200831B83EAE37CB2
:1041E000ACEBE37CBCF5FA7FA8BF4FF4FA7C6145E9
:1041F00080F2BB85ACEB010307EE903AF8EEE77A6C
:10420000B042C5ED017A17DAF1EE677AC5ED017AB1
:1042100012E000BFEC2E002064340020187E002045
:10422000EC7A0020408E00209C8E0020E43000209C
:10423000A48E0020E47A0020BBF904108B1B83EAD3
:10424000E370A0EBE370B0F5FA7FA8BF4FF4FA700B
:104250007045CCBFA0EB0E0E4FF0000E02FB0EFE21
:1042600007EE90EAF8EEE77AB1420A9BC5ED027AD2
:10427000BCBFF1EE677AC5ED027A13F4805B00F003
:104280004F85B8F5FA6F4246A8BF4FF4FA62B2F50F
:104290007A7F9AF8A431B8BF4FF47A72A2F57A7295
:1042A000002B40F05685CD49DFF850E381FB02300A
:1042B000D317C3EB6013581C6FF0630C3EF910006A
:1042C0003EF913E00CFB0323A0EB0E0003FB00F30D
:1042D00081FB0321DB17C3EB61139E440FFA8EFEB3
:1042E00007EE90EAB8EEE78A85ED038ABBF1000F8E
:1042F00041F0468019F040030C9300F0DD80B84B8C
:10430000B849D3ED019A93ED026AD1ED028A91ED9D
:10431000043A93ED030AD3ED003A91ED039AD1EDFF
:10432000015AD5ED011A95ED002AAF4B38EEC35A6C
:1043300039EEC67A73EE807A25EE077A75EEC94AB1
:1043400075EE890A33EEC0AA24EEA71AB0EE474AEA
:10435000A0EE8A4A19F00302B0EE415A79EE867A4D
:1043600078EE836AA0EE8A5AA6EEA74AA6EEE75A2E
:10437000F0EE474AD6EEA74A34EE014AF6EE006A5E
:1043800073EEA9AA26EEC44A35EE475A35EEA87A4E
:10439000F0EE647AE0EECA4AA7EE2A4A77EEC17AD6
:1043A00036EE407A73EE49AA25EE265AE0EE8A7A76
:1043B000AAEE875A74EE814A24EE047A73EEE93A43
:1043C00033EE093A64EEA64A67EEA66AF0EE477A43
:1043D000E3EE234A75EEE85A36EE006AD5EE057A2A
:1043E000A5EE057AE5EE866AF1EE648AB0EE476ADC
:1043F000B0EE677AA8EEA47AF1EE663A26EEA43A19
:10440000A3EEA66A64EE260AF0EE665AB1EE450AFD
:10441000A6EEA67AB0EE431AF0EE606AE3EEA57A55
:1044200064EE243AE5EE246AA0EE041AA8EEA46A2B
:10443000F0EE638A71EEA19AE0EE240AE5EE258A99
:1044400027EE217A32EE029AA5EE043A61EE211AA5
:1044500066EEA96AE4EEA47AE0EE253A0CBFD5ED4B
:10446000022ADFED622A83ED005AE2EE066AA0EE30
:10447000897AE2EE281A33EE033A67EEA27A73EEF7
:10448000A33AB0EE006AA3EE227AE2EEA36AE1EE6E
:10449000867A8AED6C7A85ED017ACAED6B6AC5ED94
:1044A000006ACAED6D7A83ED014AC3ED025AC3ED8D
:1044B000034A0AB9C5ED027A17F0140F03D019F4B4
:1044C000027F41F010804A4B1B789BB1059B5B8BB0
:1044D00043450FDB474B1B78012B01F0CF83192B92
:1044E00001F0CC830E2B05D0082B03D00023AB604A
:1044F000CAF838319AF8DA611EB119F0030F41F0A9
:104500005C839AF8E061002E40F0CA86059B9B7F91
:10451000002B00F0BF83022B01F02A83032B41F014
:104520002E83059B93F82030C3EB431203EB8202EA
:10453000D20092B2059BDB7F0233DBB2002E00F08B
:10454000CC84002A00F0C9842B490968B2FBF1F23F
:104550000FFA82F8AAF81082ABB307EE908AF8EE51
:10456000E77AF7EE006A86EEA77A012BD5ED007A9E
:10457000DAED896A77EEE67A67EE877ACAED857AB0
:1045800021D0D5ED017ADAED8A6A77EEE67A022B50
:1045900067EE877ACAED867A15D0D5ED027ADAED24
:1045A0008B6A77EEE67A032B67EE877ACAED877A15
:1045B00009D0D5ED037ADAED8C6A77EEE67A67EE0C
:1045C000877ACAED887A049A1278092A03F06282FF
:1045D000B8F1000F40F3648322E000BF1F85EB5168
:1045E000C80E002094000020000F002000000000F2
:1045F000100F002020310020183100209C420020A4
:104600000000C842D7A368416F12033B0000484333
:104610000AD7233CA4707D3F00C0F94400C0F9C410
:104620009BB39AED897ADAED857A77EE877A012B5A
:10463000CAED897AC5ED007A21D09AED8A7ADAED51
:10464000867A77EE877A022BCAED8A7AC5ED017AEF
:1046500015D09AED8B7ADAED877A77EE877A032B8D
:10466000CAED8B7AC5ED027A09D0DAED8C7A9AED33
:10467000887A77EE877ACAED8C7AC5ED037A013BAA
:10468000022BB8BF0223DBB20993002E099818BF92
:10469000022023785FED226AA27807EE903AF8EEC6
:1046A000E77AB0EE007A67EEA67A049BF4EEC77A5A
:1046B000F1EE10FA197840F3DA855FED2E6A37EEE5
:1046C000C77AB0EE676AA7EE266AF0EE466A95ED05
:1046D000007A1FED336A27EE066AF0EEC65A8AEDBD
:1046E000536ACAED565A9AB107EE102AB8EEC75A65
:1046F0001FED397A66EE064A25EE075AB7EE007AC4
:1047000037EE457A64EEA54AA4EE857A26EE076A6E
:104710001FED427A637926EE877A27EE067ACBB1CF
:104720005FED456A1FED456A65EEA65A06EE903AC2
:10473000F8EEE66A65EEA65AF4EEC65AF1EE10FA05
:1047400001F3D881B7EE006A76EE655AC6EE256AA7
:1047500027EE267A0C291FED508A5FED506A00F093
:104760006087B4EEC87AF1EE10FA98BFB0EE478ACF
:10477000B4EEE68AF1EE10FAB8BFB0EE668A8AEDC2
:104780004C8A002800F0DC80B0EE007AF4EEC77AA4
:10479000F1EE10FA05DD37EEC77A5FED666AE7EEF7
:1047A000267A95ED017A5FED686A27EE267AF0EEBB
:1047B000C75A8AED547ACAED575A9AB106EE902A32
:1047C0001FED6D6AF8EEE66A27EE075A66EE866A16
:1047D000B7EE006A36EE666A25EE255AA5EE266A21
:1047E00027EE067A5FED776AA37967EEA67A67EE21
:1047F000877AABB107EE103AB8EEC77A1FED7C6A44
:104800005FED7C6A27EE257A27EE067AB4EEE67A2B
:10481000F1EE10FA41F34F815FED876A67EEA67AF9
:104820000C2900F0D7865FED846A1FED847AF4EEE0
:10483000E67AF1EE10FA88BFF0EE667AF4EEC77A07
:10484000F1EE10FAB8BFF0EE477A0128CAED4D7AC2
:1048500076DD63785FED926A07EE903AF8EEE77ADC
:10486000B0EE007A67EEA67A637AF4EEC77AF1EEDC
:1048700010FA05DD37EEC77A5FED9E6AE7EE267A1D
:1048800095ED027A5FEDA06A27EE267AF0EEC75A20
:104890008AED557ACAED585A9BB106EE903A1FED53
:1048A000A46AF8EEE66A27EE075A66EE866AB7EE65
:1048B000006A36EE666A25EE255AA6EE856A27EE70
:1048C000067A5FEDAE6AE37967EEA67A67EE877ADD
:1048D000FBB107EE103AB8EEC77A1FEDB36A5FED91
:1048E000B36A27EE257A27EE067AB4EEE67AF1EE81
:1048F00010FA01F3DC80B5EEC07AF1EE10FA02F1A5
:10490000C383B7EE006A36EE477AC6EE076A67EEF3
:10491000A67A0C2900F07D865FEDC16A1FEDC17A91
:10492000F4EEE67AF1EE10FA88BFF0EE667AF4EE75
:10493000C77AF1EE10FAB8BFF0EE477ACAED4E7AB8
:10494000092900F03286059B93F82140002C40F0A5
:10495000E785D44B1F6800238AF8E031B80607D5F5
:1049600019F0300F04D0D04B1B78D90702F12E81FB
:10497000CE4B1B7823B9CE4CA678002E41F008818F
:10498000049B1D78072D7EF4C2AEFCF797F8049ABD
:10499000C84B15780B9A801AD880FEF7B8BE9AF8E3
:1049A0006431002B3EF4ABAF002318468AF8643123
:1049B000FCF7E2F9FEF7A3BFB1F900209AED567AB1
:1049C000B1F90200DAED576ABB4982EAE273A3EB60
:1049D000E273F4EEC76A80EAE072F1EE10FAA2EB3D
:1049E000E072B4BFB0EE476AB0EE666A9342B8BFF9
:1049F000134607EE103A0B78B8EEC77A27EE0A7A1C
:104A0000002B40F0BC80AD4BD3ED005AF4EEEB5AD6
:104A1000F1EE10FA41F1B780B7EE005A75EE654A33
:104A2000DFEDA76A9FEDA75AA74B36EEC77A24EEB3
:104A3000855AD3ED006AE5EE075A65EEA65AF5EE03
:104A4000C05AF1EE10FA40F2BA85CBEE256AB7EE05
:104A5000007AF0EE475AE6EE665AF0EE656AF4EE3A
:104A6000C76AF1EE10FA88BFF0EE476AF5EEC06A49
:104A7000F1EE10FAB8BFF0EE4C6A944B93ED007A69
:104A800067EE877AA7EEA68AFEF7A3BD0123FEF79D
:104A9000F7BC8F4B8F4A2B4493ED007AD2ED007A0E
:104AA0008D4B67EE277AF7EE006AF4EEE67AF1EEC8
:104AB00010FA93ED007A88BFF0EE667A67EE877A97
:104AC00027EE888AFEF7E1BE844B854D1B78D5ED35
:104AD000037A13F0010F834B059304BF1B8BAAF8D5
:104AE0008831814B1B8807EE103AB8EEC77AF4EE96
:104AF000C77AF1EE10FA41F2DF877C4A128807EE9E
:104B0000102AB8EEC77AF4EEC77AF1EE10FAC1F2C5
:104B1000BC80774B774A93ED006AD2ED006A9AF930
:104B20009431CAED636A76EE665A012BCAED616A6A
:104B3000CAED605A8AED646A01F0EB85069BCAF8FB
:104B40009831002237EEC77AFCEEE77A6A498AED9F
:104B5000677A17EE903AAAF888310123D1ED005A0E
:104B60008AF89431654B9A4241F29387644BD3EDB6
:104B7000007A93ED014A93ED026AFEF723BF524B90
:104B800093ED005AB5EEC05AF1EE10FA40F31785D6
:104B90005C4BD3ED006AF5EEC06AF1EE10FA40F31B
:104BA0000E8536EEC77A66EE4B5A87EE266AC5EE5C
:104BB000856AB7EE007AB4EEC76AF1EE10FA88BFE4
:104BC000B0EE476AB5EEC06AF1EE10FA76EE876A8B
:104BD000B8BFB0EE4C6A66EE266A40E74A4AD2EDAC
:104BE000007AB0EEC87AB4EEE77AF1EE10FA7EF70A
:104BF00086AE464AD2ED007AB0EEEC7AB4EEE77AB1
:104C0000F1EE10FA7EF77BAE414AD8ED007A92EDD4
:104C1000007AF0EEE77AF4EEC77AF1EE10FA7EF55C
:104C20006EAE01220699CAF868118AF86421FEF76F
:104C300051BECAF80C71374A374F384E04920AF504
:104C400080754FF0000B4FF0010807EE903A95ED9C
:104C5000007AF8EEE77A384687EE270AF3F760FB2A
:104C6000BAF8103108F1FF3103EB411206EB820272
:104C700082ED000A002903F06982B8F1030FC5F83C
:104C800000B000F0F387D9F800300435243708F17C
:104C90000108DAE7AAF810329846002E3FF45EAE1B
:104CA0000220F6E4408E00209E8E0020819200209B
:104CB0003A2C0020F08F0020FC380020043900201E
:104CC00000003443610BB63BF8380020F438002074
:104CD00050230020EC380020E83800204841002014
:104CE000F8900020905A0020844200208642002044
:104CF000BC300020704200208C4200208FD0030086
:104D0000942E0020003900202C3900202839002062
:104D100030390020EC8F0020483C0020DC39002096
:104D2000059B5A8B9045C0F2DC83B8F5FA6FD4BF6F
:104D3000C2EB0803C2F5FA634FF47A7101FB03F189
:104D40009AF8A401C2F5FA63B1FBF3F200283FF42C
:104D5000AAAA9AF8A5319F4902FB03F281FB02132C
:104D6000D217C2EB6312FFF79EBADFED9B7AFFF713
:104D700047BADFED997AFFF726BAB8F5FA6F80F2F5
:104D8000AC83217AA8EB020303FB01F3C2F5FA62BC
:104D900093FBF2F3C3F1640307EE903A9FED8F7A31
:104DA000F8EEE77A67EE877ACAED497AFFF7E8B955
:104DB000DAF81801BAF81031894FDFF86C82894AA5
:104DC000C3F1200603EB4010F6B2334607EB800038
:104DD0004146F5F721FABAF81031002B42F00D8365
:104DE000049B1B78142B02F0FC85DAF814217E4B0F
:104DF000013283FB02139918D317C3EBA103C3EB52
:104E0000C303D21ACAF814217849DAF81C21069D86
:104E100077480B680078CAF81C51AA1A13440B6033
:104E200000286AD107EE902A724EDFF8F891724F8F
:104E3000B8EEE78A06F2447506F5F668F6EC017AF4
:104E400094ED070AD4F86C37F8EEE77A284627EE97
:104E5000800A9847A5F1E000D4F88C369847A5F170
:104E60007000D4F8FC369847D6F85006D4F8AC3029
:104E70009847D7ED007AA9EC010AE0EE087A2435CC
:104E8000A845E7EC017AD9D1049B1D78FEF733BC25
:104E90005A4B5B4A196812885A4BC96919805A8063
:104EA00017B0BDEC0C8BBDE8F08F574B574F1B78FC
:104EB000D80700F123843A78002A00F01F86544B6B
:104EC00007939200534B544954480593544DDFF8CF
:104ED0005CB129F0FCFDFFF714B9BAF8108208F1B3
:104EE000FF380FFA88F8B8F1000FAAF810823FF7E0
:104EF00097AB002E7FF4D4AE30E5DFF808813D4D4E
:104F0000484BCDF8208007EE902AC346DFF8E890A2
:104F1000DDF81C80CDF814A0F8EEE78A05F2D4661F
:104F200000279A46049BD4ED077A1B78172B00F0D4
:104F3000A78195ED007AB8EEC78A082B28EE278A5C
:104F400007D1B0EE480A079328F020FE079BABF884
:104F50000000D8F8002092000BD5002F03F0068146
:104F6000B0EE480AD4F86C3706F170009847B0EEFE
:104F7000408AB0EE480AD4F88C36A6F17000984703
:104F8000D4F8FC3630469847049B1B78032BB0EED0
:104F9000408A00F07081D5F85406D4F8AC30B0EEF9
:104FA000480A9847D9ED007AAAEC010AE0EE287A7F
:104FB0000137032F06F124060BF1020B05F104055E
:104FC000E9EC017AAED1049BDDF814A01D78FEF760
:104FD00092BB00BF1F85EB51000000000AD7233CA5
:104FE000DC390020F82100209324499290410020D0
:104FF000B0390020F85B002094410020948F0020FD
:10500000DE3D0020F08F002048410020CD8F0020A1
:10501000B8630020905A0020B4400020EC2E0020FD
:10502000F8900020AC6300205C3B0020EC7900206D
:10503000002800F05D87B8F1000F42F09D83C7495A
:10504000B9F1000F42F01C8291ED006ADDED0E5ABD
:10505000C34A28EE866ABDEEC55AA5EE876AF0EE11
:10506000675AE6EE265A15EE103ABDEEE56A16EEE0
:1050700010EA16EE100AE645A8BF60467345C8BFA1
:10508000184606EE100AB8EEC66A012E82ED006AD6
:1050900000F0DF8091ED046ADDED0F5A28EE866A9C
:1050A000A5EE876AF0EE675AE6EE265ABDEEE56A8F
:1050B00016EE10EA16EE100AE645A8BF60469E45B9
:1050C000B8BF184606EE100AB8EEC66A022E82ED88
:1050D000016A00F0BE8091ED086ADDED105A28EEFD
:1050E000866AA5EE876AF0EE675AE6EE265ABDEEAE
:1050F000E56A16EE10EA16EE100AE645A8BF60460D
:105100009E45B8BF184606EE100AB8EEC66A032ED2
:1051100082ED026A00F09D8091ED0C6ADDED115A7E
:1051200028EE866AA5EE876AF0EE675AE6EE265A02
:10513000BDEEE56A16EE10EA16EE100AE645A8BFC7
:1051400060469E45B8BF184606EE100AB8EEC66A1D
:10515000042E82ED036A7CD091ED106ADDED125AC7
:1051600028EE866AA5EE876AF0EE675AE6EE265AC2
:10517000BDEEE56A16EE10EA16EE100AE645A8BF87
:1051800060469E45B8BF184606EE100AB8EEC66ADD
:10519000052E82ED046A5CD091ED146ADDED135AA0
:1051A00028EE866AA5EE876AF0EE675AE6EE265A82
:1051B000BDEEE56A16EE10EA16EE100AE645A8BF47
:1051C00060469E45B8BF184606EE100AB8EEC66A9D
:1051D000062E82ED056A3CD091ED186ADDED145A79
:1051E00028EE866AA5EE876AF0EE675AE6EE265A42
:1051F000BDEEE56A16EE10EA16EE100AE645A8BF07
:1052000060469E45B8BF184606EE100AB8EEC66A5C
:10521000072E82ED066A1CD091ED1C6ADDED155A51
:1052200068EE868AE7EE258AE6EEA87AFDEEE77A52
:1052300017EE901A8C45A8BF8C468B42D8BF6346A8
:1052400007EE903AF8EEE77AC2ED077A002E3EF4C8
:1052500058AFB2004349424829F039FC424B1B6821
:10526000002B3EF453AF10F001FFFEF74FBFF0EEFE
:10527000676AFFF72CBA28F089FCABF800008AE6D1
:1052800095ED007A04EB4702B8EEC78A128FABF8AF
:10529000002028EE278A5CE6F0EE665AFEF7C9BBCE
:1052A000324A334BD2F8EC201B6844F620618A4224
:1052B000A8BF0A46B2F57A7FB8BF4FF47A7292B2AD
:1052C000D906AAF8E22144D5BBF1000F01F0F0861F
:1052D000284BD3F800E0BEF8320040082649DAF83F
:1052E000E431D5ED037AA1FB02129109642292FB0D
:1052F000F1F2142ABDEEE77A0AEB430CA8BF1422A0
:1053000001339A42CAF8E43117EE108ADCBF002359
:10531000CAF8E4310AEB4303ACF8E881B3F9E831A9
:1053200007EE103AB8EEC77A77EEC77AFDEEE77A65
:10533000CDED087ABDF9202082EAE273A3EBE27397
:10534000834202F366800D4A4FF07E531360FFF7ED
:10535000DDB80A9BDB00B7D4FFF7D8B8F0410020D6
:10536000EC2E0020B44000206434002014120020F1
:10537000342F0020A08E0020D34D62109400002016
:105380001D21CA48F4F712FF002841F0C5832620EA
:1053900017F030FC00283EF4ADAFC54BDB78002B96
:1053A0007EF4A8AF2621C148F4F700FFDFEDC17AF3
:1053B000C149002802F0BA8438EE678AC6F57A72CD
:1053C000FDEEC87A12B2CDED0C7ABDF930301B0378
:1053D00081FB0301DB17C3EBA11302FB03F343F3D0
:1053E0000F33334407EE903AB8EEE78A012385ED98
:1053F000038A8AF8A031FEF77DBFD5ED027AAF4B64
:10540000B2EE0E7AF0EEE76AF4EEC76AF1EE10FA49
:10541000B3F80090AA4B40D519F0040F3DD0B3F972
:105420000430A84AA84982FB03020988DB17C3EBB2
:10543000A2035B1A9BB219B211F1B30FBCBF03F503
:10544000B47319B2B329C4BFA1F5B47319B29F4B99
:105450009F4A08931B791278002B4FF6FF7318BFF1
:10546000012310077EF580AE9A4A126811FB03F300
:10547000117E994A9BB211FB03F382FB03121A447B
:10548000DB17C3EB221307EE103AB8EEC77A77EEBC
:10549000C77AC5ED027AFEF767BEB3F904308949D1
:1054A000894A81FB0301DB17C3EBA10387490891FC
:1054B0001380FEF759BEA368002B3EF44BAE87491C
:1054C000A1F14C009847079B1B680A93FEF742BE68
:1054D000834B0493DFF820A296E4237AC3F164039C
:1054E0005AE459462CE47A4B1B7813F0100301F070
:1054F000E2839AF8B821DAF8BC3195ED017A002AF6
:105500000CBF01224FF0FF3203FB02F307EE903A8B
:10551000F8EEE77A77EE877AC5ED017AFEF7D3BF2A
:105520001E216248F4F742FE00283FF412AA0C9BA9
:10553000002B7FF40EAA9AF83432A34242F08F82F5
:10554000684B9AED8E0AD3ED058ADAED4E5A9FED3F
:10555000666ADFED666A20EE657A68EE007AA8EE8C
:10556000287AE5EEA87AB4EEC67AF1EE10FA88BF92
:10557000B0EE467AB4EEE67AF1EE10FAF4EEC67AC0
:10558000B8BFB0EE667AF1EE10FA88BFF0EE467A58
:10559000F4EEE67AF1EE10FAB8BFF0EE667A8AED34
:1055A0004C7ACAED4E7AFFF7D4B9FDEEC87A504A6C
:1055B00017EE903AA2F80480D380FFF7C4B9DFED6C
:1055C0004D6AFFF75ABA079B1B685B023EF536AC83
:1055D000FEF738BC9FED447ADFED446A444AF4EEAE
:1055E000C77AF1EE10FA98BFB0EE677AFDEEE77A6F
:1055F000B4EEE67AF1EE10FA17EE903AB8BFB0EEDC
:10560000667A01288AED4D7A53803FF722A9FFF789
:105610009AB9BDEEE77A364B17EE102A9A80FFF75B
:105620007BB9B4EEC87AF1EE10FA98BFB0EE478AB3
:10563000BDEEC77AB4EEE68A2D4EF1EE10FA17EE03
:10564000103AB8BFB0EE668A8AED4C8A33800028E3
:105650007FF49AA8FFF777B9002B3EF450A9FEF724
:1056600035B9FBF72BFA049B0A9A1B78DFF8808088
:10567000801A012BA8F8020000F0E282072B7EF4CA
:1056800066A9FBF71BFA0890FEF763B9FBF716FA59
:10569000049B08991B78164A401A072B90807EF4C9
:1056A00051ADFBF70BFA0B90FEF74EBD342F0020E7
:1056B0000893002000007A44D34D62109C8E002095
:1056C0004C8E002067666666448B0020E430002024
:1056D0009E8E0020A08E002089888888185C00207B
:1056E000EC8F00209400002000C0F94400C0F9C4F1
:1056F000F08F002000000000F82100203B78002BF4
:1057000000F0FC81DAED573A9AED566AF14ADAED8B
:10571000617AD2ED005A9AED607A9AED544ADAED48
:10572000534AED49ED4AF4EEC63AF3EE046AF1EE5F
:1057300010FA37EEA65A00F1258391ED026A26EEA3
:10574000446AF0EE674AE6EE074AF4EEC54A34EEE4
:10575000E66AF1EE10FA48BFB0EE656A012B82ED01
:10576000006A00F0CB8191ED066A26EE446AF0EE05
:10577000674AE6EE074AF4EEC54A34EEE66AF1EE11
:1057800010FA48BFB0EE656A022B82ED016A00F0A4
:10579000B58191ED0A6A26EE446AF0EE674AE6EEBC
:1057A000074AF4EEC54A34EEE66AF1EE10FA48BF55
:1057B000B0EE656A032B82ED026A00F09F8191EDE5
:1057C0000E6A26EE446AF0EE674AE6EE074AF4EE09
:1057D000C54A34EEE66AF1EE10FA48BFB0EE656AEB
:1057E000042B82ED036A00F0898191ED126A26EEA6
:1057F000446AF0EE674AE6EE074AF4EEC54A34EE34
:10580000E66AF1EE10FA48BFB0EE656A052B82ED4C
:10581000046A00F0738191ED166A26EE446AF0EE98
:10582000674AE6EE074AF4EEC54A74EEE66AF1EE20
:1058300010FA48BFF0EE656A062BC2ED056A00F06B
:105840005D81D1ED1A6A66EEC46AF0EE674AE6EE53
:10585000874AB3EE046AF4EEC54A74EEC66AF1EE06
:1058600010FA48BFF0EE656A072BC2ED066A00F039
:105870004581D1ED1E6A9A4B079326EEC44A994B97
:105880000593E4EE077A984DDFF860B2F4EEC57A3E
:1058900077EEC67AF1EE10FA48BFF0EE657AC2ED07
:1058A000077AFEF72EBCB8F1000F41F08D8228EE8A
:1058B000866A8A4AA5EE876AF0EE675AE6EE265AAD
:1058C000BDEEE56A16EE10EA16EE100AE645A8BF30
:1058D00060467345C8BF184606EE100AB8EEC66AA1
:1058E000012E82ED006A3FF4B4AC91ED046ADDED67
:1058F0000F5A28EE866AA5EE876AF0EE675AE6EE42
:10590000265ABDEEE56A16EE10EA16EE100AE645D6
:10591000A8BF60467345C8BF184606EE100AB8EE29
:10592000C66A022E82ED016A3FF493AC91ED086ADB
:10593000DDED105A28EE866AA5EE876AF0EE675A0A
:10594000E6EE265ABDEEE56A16EE10EA16EE100AED
:10595000E645A8BF60467345C8BF184606EE100A64
:10596000B8EEC66A032E82ED026A3FF472AC91ED86
:105970000C6ADDED115A28EE866AA5EE876AF0EE14
:10598000675AE6EE265ABDEEE56A16EE10EA16EE06
:10599000100AE645A8BF60467345C8BF184606EE24
:1059A000100AB8EEC66A042E82ED036A3FF451ACC9
:1059B00091ED106ADDED125A28EE866AA5EE876A2F
:1059C000F0EE675AE6EE265ABDEEE56A16EE10EAEC
:1059D00016EE100AE645A8BF60467345C8BF1846D4
:1059E00006EE100AB8EEC66A052E82ED046A3FF490
:1059F00030AC91ED146ADDED135A28EE866AA5EEFF
:105A0000876AF0EE675AE6EE265ABDEEE56A16EEB4
:105A100010EA16EE100AE645A8BF60467345C8BFF7
:105A2000184606EE100AB8EEC66A062E82ED056A22
:105A30003FF40FAC91ED186ADDED145A28EE866A3A
:105A4000A5EE876AF0EE675AE6EE265ABDEEE56AE5
:105A500016EE10EA16EE100AE645A8BF604673453A
:105A6000C8BF184606EE100AB8EEC66A072E82EDC9
:105A7000066A3FF4EEAB91ED1C6ADDED155A68EE57
:105A8000868AE7EE258AE8EEA67AFDEEE77A17EE3B
:105A9000901A8C45A8BF8C468B42C8BF9C4607EE27
:105AA00090CAF8EEE77AC2ED077AFFF7CFBBDFEDD9
:105AB000106AFEF72CBFB5EEC07AF1EE10FA01F1D4
:105AC000E782B7EE006A36EE477AC6EE076AFEF75F
:105AD000A5BE00BFEC410020F0410020EC2E0020CC
:105AE000B8630020905A0020F8900020EC79002044
:105AF0000000C8425FED026AFEF72ABE894B079399
:105B0000894B0593894DDFF874B2FEF7FABA884ADB
:105B10005379002B3EF416A8864B1B78002B3EF4DD
:105B200011A812789FED845A07EE902A834AB8EEA6
:105B3000677A128807EE903A06EE102AF8EEE77AB6
:105B4000B8EE466A67EE277AB7EE007AC7EE863A75
:105B5000F4EEC53AF1EE10FA88BFF0EE453AF4EEF5
:105B6000C73AF1EE10FAB8BFF0EE473AFDF7ECBFD6
:105B7000BAF8E22102F57A7292B2FEF7DBBC704B02
:105B80005A88FEF7D7BC6F4BD3ED005AFEF757BFCC
:105B90006D4D2B78013B0D2B39D8DFE813F0B9069A
:105BA0006E07C6061007F7063307A30699067406A4
:105BB00023005F06620759074F07644B9FED647A25
:105BC000D3ED087AF4EEC77AF1EE10FA00F22D85E3
:105BD0009FED607AD5ED037A77EE877AC5ED037A8B
:105BE000FEF78FBC5C4B1B78002B02F011811A2052
:105BF00017F05CF8002842F00B81584B1B78002B03
:105C000042F0068109232B700DF076F8A678012E5C
:105C100000F0F5842379012B01F08685022B7EF4B8
:105C2000AFAE2B78012B7EF4ABAE4C4B1B78002B28
:105C30007EF4A6AE0DF0ECFFFEF7A2BEDFF84081C9
:105C4000FAF73CFF464ADAF8783112680890C31A2E
:105C50009A1ACAF87801A8F80430A8F80620FDF7C7
:105C600078BEFAF72BFF0A90FDF711BC013303F061
:105C70001F03AAF81031049BFDF70BBB394B9B7B2C
:105C8000002B3EF433ACFEF735BCBAF888219A42BB
:105C900000F21685262016F0ADFF002840F0108592
:105CA000314B324AD3ED007A314B92ED007A1B78BA
:105CB000CAED637A8AED647A002B01F0988377EE5F
:105CC000676A9AF99431CAED606A0133CAED617A64
:105CD00001F09A86069BCAF8983100229FED1D7A42
:105CE00024498AED677AFF23D1ED005A8AF894316E
:105CF000FEF738BF0120FBF73FF8DAF86821069B72
:105D00009A1AFDF77FBC1C4BD8ED007A93ED007A10
:105D1000F0EEE77AF4EEC77AF1EE10FA7DF7EFAD28
:105D2000FDF7E7BDB8630020905A0020F8900020EE
:105D3000308E0020F6900020713DAA3FE0900020B8
:105D4000E4920020F8380020382C00206841002020
:105D50008FC2753C0000000022310020233100205A
:105D600018310020E45A00204C2F002074420020FB
:105D7000F07A00208842002030390020EC790020A1
:105D8000F08F002091ED016A26EE646AB0EE674A5A
:105D9000A6EE074AB4EEC54A34EE666AF1EE10FA92
:105DA00048BFB0EE656A012B82ED006A3FF4A6AEF3
:105DB00091ED056A26EE646AB0EE674AA6EE074AE0
:105DC000B4EEC54A34EE666AF1EE10FA48BFB0EEA2
:105DD000656A022B82ED016A3FF490AE91ED096A8B
:105DE00026EE646AB0EE674AA6EE074AB4EEC54AEC
:105DF00034EE666AF1EE10FA48BFB0EE656A032B26
:105E000082ED026A3FF47AAE91ED0D6A26EE646A85
:105E1000B0EE674AA6EE074AB4EEC54A34EE666AAB
:105E2000F1EE10FA48BFB0EE656A042B82ED036A0A
:105E30003FF464AE91ED116A26EE646AB0EE674AF3
:105E4000A6EE074AB4EEC54A34EE666AF1EE10FAE1
:105E500048BFB0EE656A052B82ED046A3FF44EAE92
:105E600091ED156A26EE646AB0EE674AA6EE074A1F
:105E7000B4EEC54A74EE666AF1EE10FA48BFF0EE71
:105E8000656A062BC2ED056A3FF438AED1ED196A9A
:105E900066EEE46AB0EE674AA6EE874AB3EE046A9D
:105EA000B4EEC54A74EE466AF1EE10FA48BFF0EE61
:105EB000656A072BC2ED066A3FF420AED1ED1D6A7C
:105EC000B14B079366EEE44AB04B0593E4EE877A54
:105ED000AF4DDFF8D0B2F4EEC57A77EEC67AF1EEC8
:105EE00010FAB8BFF0EE657AC2ED077AFEF709B98D
:105EF000A849B9F1000F41F0E98091ED006ADDEDAC
:105F00000E5AA54A28EE866ABDEEC55AA5EE876AE6
:105F1000F0EE675AE6EE265A15EE103ABDEEE56A47
:105F200016EE10EA16EE100AE645A8BF6046734565
:105F3000C8BF184606EE100AB8EEC66A012E82EDFA
:105F4000006A3EF4DAA891ED046ADDED0F5A28EEFE
:105F5000866AA5EE876AF0EE675AE6EE265ABDEE2F
:105F6000E56A16EE10EA16EE100AE645A8BF60468E
:105F70009E45B8BF184606EE100AB8EEC66A022E55
:105F800082ED016A3EF4B9A891ED086ADDED105A80
:105F900028EE866AA5EE876AF0EE675AE6EE265A84
:105FA000BDEEE56A16EE10EA16EE100AE645A8BF49
:105FB00060469E45B8BF184606EE100AB8EEC66A9F
:105FC000032E82ED026A3EF498A891ED0C6ADDED95
:105FD000115A28EE866AA5EE876AF0EE675AE6EE59
:105FE000265ABDEEE56A16EE10EA16EE100AE645F0
:105FF000A8BF60469E45B8BF184606EE100AB8EE28
:10600000C66A042E82ED036A3EF477A891ED106A09
:10601000DDED125A28EE866AA5EE876AF0EE675A21
:10602000E6EE265ABDEEE56A16EE10EA16EE100A06
:10603000E645A8BF60469E45B8BF184606EE100A62
:10604000B8EEC66A052E82ED046A3EF456A891EDBC
:10605000146ADDED135A28EE866AA5EE876AF0EE23
:10606000675AE6EE265ABDEEE56A16EE10EA16EE1F
:10607000100AE645A8BF60469E45B8BF184606EE22
:10608000100AB8EEC66A062E82ED056A3EF435A8FF
:1060900091ED186ADDED145A28EE866AA5EE876A3E
:1060A000F0EE675AE6EE265ABDEEE56A16EE10EA05
:1060B00016EE100AE645A8BF60469E45B8BF1846D2
:1060C000FDF7F9BF354EDAED017A9AED006A3188B5
:1060D000736977EEA77AF0EE006AB0EE677AA6EE03
:1060E000267A4E1E0AEBC601D6EE267A0839103300
:1060F000F6EE003A27EE237A67EEA37A8AED207A4D
:10610000CAED217ADFF898A057460AF1800091ED98
:10611000027A91ED036AD7ED036AD7ED027A53ED67
:10612000014A13ED025A37EE674A76EEC65A77EE09
:10613000277AE4EE845A013EA1F10801E5EE047AE3
:1061400007F1080703F1080336EE267A00F108008C
:10615000E4EE877AE5EE475A67EEA37A25EEA37A56
:10616000C0ED007A80ED017AD1D1BCF1140F7EF43C
:106170003EAEFAF7A3FCDFF83080DAF81421401BBA
:10618000A8F80200FEF733BEB8630020905A002042
:10619000F8900020F0410020EC2E0020C4390020AF
:1061A000F8210020EC790020F08F0020A64B197810
:1061B000DAF81801A54F9FEDA67AC600BB1983ED4A
:1061C000007A002901F03E81A24AB0EE476AF0EE63
:1061D000476A0023F2EC017A013367EEA77A05EEF5
:1061E000903AB4EEE77AF1EE10FAF8EEE55AB8BF5D
:1061F000B0EE677A8B4276EEA76AA7EEA56AE9D180
:10620000F5EEC06ABB19F1EE10FA83ED007A41F3A6
:10621000198186EE268A904BDFF85882B8F8002064
:10622000F7EE007A38EE678AD3ED007A68EE277AC7
:10623000FDEEE77A17EE903A812B40F335879342D3
:10624000A8BF134607EE903AB8EEE70A834B3044F6
:1062500003EB8000F2F764F8FDEEC07AB8F8003086
:1062600017EE902A812A40F31C879342A8BF134659
:1062700007EE903AF8EEE77AFCEEE77ACDED057A94
:10628000BDF81430DAF81801C600BA199380049BDF
:106290001B7810B9132B01F06D85152B01F0C88008
:1062A000142B7EF4A2AD64E7DAF818216C4B674931
:1062B0006C4E1846D30019441A448B88016800EECE
:1062C000103A10EE103A643BC82BA8BFC823782BB5
:1062D000B8BF782307EE903AB8EEC07AF8EEE77AC6
:1062E00006EB820677EE670A77EE876A67EE877AB3
:1062F00020EEA67AB8EE400AC7EE870A3046D6F8F6
:1063000014B0D6F81890D6F81C80376A19F068FFD8
:10631000049BC6F814B01B78C6F81890142BC6F866
:106320001C80376201F04D85DAF818214E48DAF802
:106330001411013280FB0230A0EBE27000EB400050
:10634000101A0131CAF81801CAF81411FEF732BD4B
:10635000464E4048B268B18926F046FB049B93F84C
:1063600000C0BCF1140F01F04785DAF814210132A6
:10637000CAF81421A7E6344F39785FEA910E01F08C
:1063800096853B4E0EF101094FEA491906EB0908C3
:1063900006F12003A6F1700013ED076A53ED056ABC
:1063A00013ED037A53ED017A53ED025A13ED084AC7
:1063B00053ED064A13ED045A26EE066A66EEA66A07
:1063C00027EE077A67EEA77AA4EE046A2033984591
:1063D000E4EEA46A00F11000A5EE057AE5EEA57AD8
:1063E000F1EEC65AB1EEE66AF1EEC76AB1EEE77AAF
:1063F00040ED085A00ED076A40ED066A00ED057AA7
:10640000CAD1A9F1200333440AEB0E1611F00300A0
:1064100018BF08330FD053ED017A13ED027A67EEFF
:10642000A77A0138E7EE077A03F10803B1EEE77ABD
:10643000A6EC017AEFD1BCF1140F01F0CD8401324A
:10644000CAF81421B4E600BFBE390020B43C0020D5
:1064500000000000F8210020C0390020DC3B0020B3
:10646000A86300203C63002056555555C4390020D0
:1064700078220020BC390020E64E3288D6F80490FD
:106480004FEA52084FEA88015FEAD20C0AEB010397
:106490000AEB820700F0A18001F110020CF1010C5F
:1064A000DD4803EB0C1C3A44103309F1100E07F1E0
:1064B000100151ED032A51ED043A10ED043A10EDAC
:1064C000032A51ED026A11ED016A10ED021A50ED36
:1064D000010A12ED044A12ED035A53ED044A53ED3A
:1064E000035A13ED027A53ED017A52ED021A12EDBE
:1064F000010A73EE238A32EE228A40ED048A00ED0F
:10650000038A71EE268A30EE868A40ED028A00ED1B
:10651000018A74EE848A35EE858A43ED048A03EDA0
:10652000038A77EE218A37EE808A43ED028A03EDF3
:10653000018A73EE633A75EE655A1EED035A32EE28
:10654000623A74EE644A25EE638A1EED044A23EE35
:10655000052A64EE652AA3EE048A10339C4524EED6
:10656000843AA3EE842A00F110000EF1100EA5EE7D
:10657000853A01F1100102F11002E4EE852A01EDE5
:10658000078A01ED082A02ED073A42ED082A5EED7E
:10659000055A1EED065A71EE666A30EEC66A31EE95
:1065A000C77A70EE677A26EE253A65EEE63A25EE72
:1065B000674A67EE054AE6EE053AA6EE853AA7EE8B
:1065C000254AE7EEA54A01ED063A41ED053A02ED0E
:1065D000064A42ED054A7FF46CAF1FFA88F84A4636
:1065E00041468E4819F014F841467268384619F051
:1065F0000FF8049B1B78142B7EF4F7ABB9E5884A9F
:10660000884B92681B689A423FF604AB2B780C3B90
:10661000022B7EF6B5A9844B2E701A78002A3EF420
:10662000AFA900221A70FEF7ABB9F0EEE76AB7EE39
:10663000005A35EE665A9FED7D4ADFED7D5A9FED9B
:106640007D6A9FED7D7A9AED770AF1EEC54AE6EE16
:10665000845AF5EEC07AA6EEA56AF1EE10FAA6EE1F
:10666000867A48BFDFED757A27EE247A48BF37EE89
:10667000C77A27EE000A27F089FAB0F5617F00F3A8
:10668000AA8607EE900AB8EEE70ADFED6D7A20EEF3
:10669000270A07EE906AB8EEE78AFDEEC07A17EE99
:1066A000903A2033402B40F29C869FED660A27F0FB
:1066B0006DFA00B207EE900AB8EEE77AFFF78ABAF1
:1066C0009AF8A021002A7FF4EBAA5F4B5F4993ED73
:1066D000007AD1ED007A9AF99431CAED637A77EEB7
:1066E000676A012BCAED617ACAED606A8AED647A45
:1066F00001F04E83069BCAF89831554B9FED517AB5
:10670000D3ED005A8AED677A01238AF89431FEF7B7
:1067100029BADAF89821069B9A1AFEF713BAB4F947
:106720003830226207EE903A0122F8EEE77A2366CB
:10673000E2670023012FC4ED1C7AC4ED1B7A636766
:1067400001F0F082B7427CF40DAEB4F93A306366E2
:1067500007EE903A00220123F8EEE77A6262C4F86D
:1067600090300023012FC4ED217AC4ED207AC4F8C3
:10677000883001F0FB82B7427CF425AEB4F93C309E
:10678000A36607EE903A00220123F8EEE77AA262B0
:10679000C4F8A4300023012FC4ED267AC4ED257A75
:1067A000C4F89C307CF440AE9FED268A032D2AD09D
:1067B000B9F1000F09D007EE909AF8EEE77AF4EEFF
:1067C000C87AF1EE10FA01F17783224BDFF84CA082
:1067D0001A68A36E9AF82011A8F8060003EB560376
:1067E00093FBF6F60023A66293621363D36229B18A
:1067F000194B1B6833F480637CF41AAE012025F03A
:10680000C5F8FCF715BEB0EE480A27F0BFF900B294
:10681000CEE700BFC439002008220020F821002064
:106820000C1100201C31002023310020306E99BC57
:106830002716983D843459BEA40DC93FDB0F49404B
:10684000D06D393A00000000BC30002070420020BA
:106850008C420020948F0020988E0020C44BC54AA3
:106860005B681268C833934205D30BF0CDFBA67862
:1068700000283FF4CCA9032E01F0AC8301232B7038
:10688000A678FFF7C4B91A2016F010FA00283FF4D2
:10689000BBA9B94B1B88002B7FF4B6A9B74B452089
:1068A0001E680BF0E5FB0E200BF0E2FB30460BF010
:1068B000B5FD069E30460BF0B1FDB14AB14B1268F2
:1068C0001A6030460A232B700BF0B8FEFFF79CB914
:1068D0000BF076FB0CF046FA002841F05283A678C4
:1068E000FFF795B90BF06CFBA74B002105208DE855
:1068F0000300A3F10802029153200CF02BFF0028A3
:10690000EDD19B4BA678186008232B70FFF77FB959
:106910009E4B1B78DA0701F142831F2016F0C6F95F
:106920000028DCD00C232B70D9E7914E0BF048FBEC
:10693000904A7368126864339342D0D240200BF0BF
:1069400017FB0028CBD13368DFF87C92DFF84C824C
:1069500040270CE00BF08CFBD8F800203368013A9C
:106960000133013FC8F80020336001F02C8319F88F
:1069700003301846002BEDD1002333604FF0FF3277
:10698000042372602B70A678FFF741B90BF018FB57
:106990007F4B002102208DE80300A3F10802029141
:1069A00048200CF0D7FE002899D1714BA6781860CA
:1069B0004FF0FF325A6006232B70FFF728B90BF017
:1069C000FFFA744A0292A2F10C032921019300916B
:1069D000A2F10A035021163A49200CF0BBFE002810
:1069E0007FF47DAF079B1B6813F0800301F0E18209
:1069F0005F4BA67818604FF0FF325A6005232B706A
:106A0000FFF705B90BF0DCFA634A0292A2F10C031E
:106A1000072601930096A2F108030021143A4720AB
:106A20000CF098FE00287FF45AAF514B2E704FF0B7
:106A3000FF3283E80500A678FFF7E9B81F2016F0BB
:106A400035F900287FF4E3A801232B70FFF7DFB8A6
:106A5000012E01F045820E2313202B7024F096FFA7
:106A60003DE7012E01D1F3F7C7FF0D2313202B7053
:106A700024F08CFFA678FFF7CAB83E4B3C4A1B684F
:106A8000536046490023136003220B602A70FFF70E
:106A9000BEB8DFED437A434B9AED677AC3ED007AD7
:106AA000C3ED017AC3ED027A3F4BB0EE676AB0EEF8
:106AB000674A1E68FCF786BF3C4B3D4AD3ED006A2F
:106AC0003C4B92ED006A1B78CAED636A8AED646AFA
:106AD000002B00F0E18276EE665A9AF99431CAED05
:106AE000605A0133CAED616A00F01886069BCAF845
:106AF0009831002237EE677AFCEEE77A2E498AED6C
:106B0000677A17EE903AAAF88831FF23D1ED005A40
:106B10008AF89431FEF726B8284BDB78002B7DF4F9
:106B2000E9ABDFED277A274938EE678AC6F5FA63C5
:106B3000FDEEC87A1BB2CDED0C7ABDF93020120300
:106B400081FB0201D217C2EBA11203FB02F343F354
:106B50000F33334407EE903AB8EEE78A262085EDEE
:106B6000038A16F047F800283DF4C4ABFEF71ABCC0
:106B7000C030002014540020402F00203C2F002063
:106B8000282F0020242F0020D8F30308484100209C
:106B900074F3030896F1030890F30308F42C002023
:106BA00000000000942E0020A08E00204C2F00201A
:106BB00074420020F07A00208842002008930020D0
:106BC00000007A44D34D621030F10308744B754ACB
:106BD000B3F90430DFED747A82FB0312DB17C3EBE9
:106BE000A2031BB208EE103AB8EEC88A28EE278A34
:106BF000B0EE480AF3F70EF9F0EE408AB0EE480A1C
:106C0000F3F78EF8694BD878002800F09D83684A26
:106C1000BAF93E12B2F9023044F250645B1AA34250
:106C200040F3FB86A3F50C43A03B44429C4200F397
:106C3000F1868342A8BF0346B2F90020BAF93C525C
:106C40000B4419B2531B44F250629342AAF83E120D
:106C500040F3D286A3F50C43A03B9C4203DC984250
:106C6000A8BF184604462B191BB207EE903A07EE50
:106C7000101AF8EEE77AF8EEC76A27EEE87A60EEC7
:106C8000277AA0EE267AAAF83C32E8EEA67ADFED63
:106C9000496A27EE267A67EEA67ABDEEC77AFDEE40
:106CA000E77A17EE102A17EE903AAAF84821AAF8C8
:106CB0004A31FDF75DBE0898C178002900F0608375
:106CC000BAF9C0218178A8EB020686EAE670A0EB4B
:106CD000E670884240F3A9869045C8BF494207EE56
:106CE000901AF8EEE77A012037EE888ACAF8C431A4
:106CF0008AF8C80185ED038AFDF7E5BB9FED2E8A72
:106D00008AED4A8A15F0C4FFF0EE487A002840F078
:106D10009D83B6EE007AF4EEC78AF1EE10FA7DF7A5
:106D200091A8B6EE008A67EE887AF4EEE87AF1EE82
:106D300010FAC8BFF0EE678A40F38883CAED678A0D
:106D4000FDF780B81D4BDFF878B0197801F0010825
:106D5000FDF7D3B9F9F7B2FE049B93F800C0BCF17C
:106D6000140F05BFDFF85C80DAF81421DAF814217B
:106D7000A8F800200546FCF795BA74EE467AB7EEFF
:106D8000007AF4EEC77AF1EE10FACAED4A7A41F3CE
:106D9000058085EE277A8DED0E7AFDF74AB800BFA3
:106DA0004C8E00206766666635FA8E3CC88A0020E5
:106DB000248B0020CDCCCC3D000000804841002039
:106DC000EC790020F08F0020002A00F0918628EE58
:106DD000866ABB4AA5EE876AF0EE675AE6EE265A47
:106DE000BDEEE56A16EE10EA16EE100AE645A8BFFB
:106DF00060467345C8BF184606EE100AB8EEC66A6C
:106E0000012E82ED006A3DF47CA991ED046ADDED6E
:106E10000F5A28EE866AA5EE876AF0EE675AE6EE0C
:106E2000265ABDEEE56A16EE10EA16EE100AE645A1
:106E3000A8BF60467345C8BF184606EE100AB8EEF4
:106E4000C66A022E82ED016A3DF45BA991ED086AE3
:106E5000DDED105A28EE866AA5EE876AF0EE675AD5
:106E6000E6EE265ABDEEE56A16EE10EA16EE100AB8
:106E7000E645A8BF60467345C8BF184606EE100A2F
:106E8000B8EEC66A032E82ED026A3DF43AA991ED8E
:106E90000C6ADDED115A28EE866AA5EE876AF0EEDF
:106EA000675AE6EE265ABDEEE56A16EE10EA16EED1
:106EB000100AE645A8BF60467345C8BF184606EEEF
:106EC000100AB8EEC66A042E82ED036A3DF419A9D1
:106ED00091ED106ADDED125A28EE866AA5EE876AFA
:106EE000F0EE675AE6EE265ABDEEE56A16EE10EAB7
:106EF00016EE100AE645A8BF60467345C8BF18469F
:106F000006EE100AB8EEC66A052E82ED046A3DF45C
:106F1000F8A891ED146ADDED135A28EE866AA5EE05
:106F2000876AF0EE675AE6EE265ABDEEE56A16EE7F
:106F300010EA16EE100AE645A8BF60467345C8BFC2
:106F4000184606EE100AB8EEC66A062E82ED056AED
:106F50003DF4D7A891ED186ADDED145A28EE866A43
:106F6000A5EE876AF0EE675AE6EE265ABDEEE56AB0
:106F700016EE10EA16EE100AE645A8BF6046734505
:106F8000C8BF184606EE100AB8EEC66A072E82ED94
:106F9000066A3DF4B6A891ED1C6ADDED155A68EE5F
:106FA000868AE5EE878AE8EEA67AFDEEE77A17EEA6
:106FB000901A8C45A8BF8C468B42D8BF634607EE1B
:106FC000903AF8EEE77AC2ED077AFDF79AB8012910
:106FD0007FF7EAAB07EE10EAB8EEC77AC7EE876A2A
:106FE000B1EEE68AFFF7E2BB012940F3BF8607EE68
:106FF00010EAB8EEC77AC7EE876AB1EEE68A032DCB
:1070000014D0B9F1000F09D007EE909AF8EEE77AA4
:10701000F4EEC87AF1EE10FA00F14E87636E03EBDE
:10702000560393FBF6F36362FFF7A5BBB0EE480A85
:1070300026F0ACFD00B2E4E7012940F3738607EEC9
:1070400010EAB8EEC77AC7EE876AB1EEE68A032D7A
:1070500014D0B9F1000F09D007EE909AF8EEE77A54
:10706000F4EEC87AF1EE10FA00F12687236E03EBF6
:10707000560393FBF6F32362FFF764BBB0EE480AB6
:1070800026F084FD00B2E4E7F7EE006AFDF73FBCAE
:10709000F7EE006AFDF7C2BB76EEC65AF0EE466A1E
:1070A0001BE58223FFF7EEB89FED060AFFF7CEB887
:1070B000054BD3F800E0BEF93200FEF70FB900BF70
:1070C000EC2E002000000243A08E002091ED006A0B
:1070D000DDED0E4AE34A28EE866ABDEEC54AA4EE0F
:1070E000876AF0EE674AE6EE264A14EE103AF4EEAE
:1070F000E45AF1EE10FAB0EE646A88BFB0EE456A69
:10710000BDEEC66A16EE10EA16EE100AE645A8BFF6
:1071100060467345C8BF184606EE100AB8EEC66A48
:10712000012E82ED006A3CF4E8AF91ED046ADDEDDA
:107130000F4A28EE866AA4EE876AF0EE674AE6EE0A
:10714000264AF4EEE45AF1EE10FAB0EE646A88BF13
:10715000B0EE456ABDEEC66A16EE10EA16EE100AEB
:10716000E645A8BF60469E45B8BF184606EE100A21
:10717000B8EEC66A022E82ED016A3CF4BEAF91ED14
:10718000086ADDED104A28EE866AA4EE876AF0EE02
:10719000674AE6EE264AF4EEE45AF1EE10FAB0EE53
:1071A000646A88BFB0EE456ABDEEC66A16EE10EAA4
:1071B00016EE100AE645A8BF60469E45B8BF1846C1
:1071C00006EE100AB8EEC66A032E82ED026A3CF49F
:1071D00094AF91ED0C6ADDED114A28EE866AA4EEBB
:1071E000876AF0EE674AE6EE264AF4EEE45AF1EEDC
:1071F00010FAB0EE646A88BFB0EE456ABDEEC66AAA
:1072000016EE10EA16EE100AE645A8BF60469E4547
:10721000B8BF184606EE100AB8EEC66A042E82ED14
:10722000036A3CF46AAF91ED106ADDED124A28EE74
:10723000866AA4EE876AF0EE674AE6EE264AF4EE26
:10724000E45AF1EE10FAB0EE646A88BFB0EE456A17
:10725000BDEEC66A16EE10EA16EE100AE645A8BFA5
:1072600060469E45B8BF184606EE100AB8EEC66ADC
:10727000052E82ED046A3CF440AF91ED146ADDED19
:10728000134A28EE866AA4EE876AF0EE674AE6EEB5
:10729000264AF4EEE45AF1EE10FAB0EE646A88BFC2
:1072A000B0EE456ABDEEC66A16EE10EA16EE100A9A
:1072B000E645A8BF60469E45B8BF184606EE100AD0
:1072C000B8EEC66A062E82ED056A3CF416AF91ED63
:1072D000186ADDED144A28EE866AA4EE876AF0EE9D
:1072E000674AE6EE264AF4EEE45AF1EE10FAB0EE02
:1072F000646A88BFB0EE456ABDEEC66A16EE10EA53
:1073000016EE100AE645A8BF60469E45B8BF18466F
:1073100006EE100AB8EEC66A072E82ED066A3CF445
:10732000ECAE91ED1C6ADDED154A68EE868AE7EE5B
:10733000248AE6EEA87AF4EEE75AF1EE10FAC8BF16
:10734000F0EE457AFCF7C9BE474B9FED486AB3F9AA
:107350000020B3F9023007EE902A06EE903AF8EEDC
:10736000E77AF8EEE66A27EEE87A60EE277AA0EE92
:10737000267AE8EEA67A27EE067A67EE867A8CE41D
:10738000BAF9C0318078A8EB030282EAE276A6EB74
:10739000E276864240F3558302EBD272012152100D
:1073A000CAF8D0218AF8D4118AF8C811DAF8BC21B9
:1073B0001344B3F5FA6FA8BF4FF4FA63B3F57A7FBD
:1073C000B8BF4FF47A7307EE903AF8EEE77AC5ED5E
:1073D000037AFDF778B807EE906A9FED250AB8EEBC
:1073E000E78AF2F7A5FB20EE080AFFF760B977EE0F
:1073F000C76AF0EE477AFEF764BCDAF81801B2000B
:1074000008EB020107EBC0105244F2F705FFFDF74D
:10741000E7BCBEF834309FED177A07EE903AF8EEED
:10742000E77A154B67EE877AC3ED007AFDF76EB801
:107430003E44DFF84880B38828F81030DAF8142189
:10744000FDF7D5BC049B1B78FEF727BFB7EE007A8B
:1074500077EE677AF4EEE78AF1EE10FA88BFF0EE85
:10746000678A6BE4EC2E0020248B0020CDCCCC3D31
:1074700084F9223F6F12833A94000020F08F00209D
:1074800091ED006ADDED0E4AB74A28EE866ABDEE40
:10749000C54AA4EE876AF0EE674AE6EE264A14EE85
:1074A000100AF4EEE45AF1EE10FAB0EE646A88BF06
:1074B000B0EE456ABDEEC66A16EE10EA16EE103A58
:1074C000E645A8BF63467045C8BF034606EE103ABE
:1074D000B8EEC66A012E82ED006A3DF4BAAE91EDB7
:1074E000046ADDED0F4A28EE866AA4EE876AF0EEA4
:1074F000674AE6EE264AF4EEE45AF1EE10FAB0EEF0
:10750000646A88BFB0EE456ABDEEC66A16EE10EA40
:1075100016EE103AE645A8BF63468645B8BF034657
:1075200006EE103AB8EEC66A022E82ED016A3DF40C
:1075300090AE91ED086ADDED104A28EE866AA4EE61
:10754000876AF0EE674AE6EE264AF4EEE45AF1EE78
:1075500010FAB0EE646A88BFB0EE456ABDEEC66A46
:1075600016EE10EA16EE103AE645A8BF63468645C9
:10757000B8BF034606EE103AB8EEC66A032E82ED97
:10758000026A3DF466AE91ED0C6ADDED114A28EE1B
:10759000866AA4EE876AF0EE674AE6EE264AF4EEC3
:1075A000E45AF1EE10FAB0EE646A88BFB0EE456AB4
:1075B000BDEEC66A16EE10EA16EE103AE645A8BF12
:1075C00063468645B8BF034606EE103AB8EEC66A73
:1075D000042E82ED036A3DF43CAE91ED106ADDEDC0
:1075E000124A28EE866AA4EE876AF0EE674AE6EE53
:1075F000264AF4EEE45AF1EE10FAB0EE646A88BF5F
:10760000B0EE456ABDEEC66A16EE10EA16EE103A06
:10761000E645A8BF63468645B8BF034606EE103A66
:10762000B8EEC66A052E82ED046A3DF412AE91ED05
:10763000146ADDED134A28EE866AA4EE876AF0EE3E
:10764000674AE6EE264AF4EEE45AF1EE10FAB0EE9E
:10765000646A88BFB0EE456ABDEEC66A16EE10EAEF
